:100000000C94BC300C94B6330C94E1330C940C3447
:100010000C9437340C9462340C948D340C94B834B2
:100020000C94E3340C94ED300C94ED300C94ED30E2
:100030000C94ED300C94ED300C94ED300C94ED30CC
:100040000C94ED300C9422DB0C94ED300C94ED30DC
:100050000C94ED300C94ED300C94A4C90C94EF305A
:100060000C94ED300C9456A10C9402A20C94ED303B
:100070000C94ED300C94ED300C94ED300C94ED308C
:100080000C94ED300C94ED300C94ED300C94ED307C
:100090000C94ED300C94ED300C94ED300C94ED306C
:1000A0000C94ED300C94ED300C94ED300C94ED305C
:1000B0000C94ED300C94ED300C94ED300C94ED304C
:1000C0000C94ED300C94ED300C94ED300C94ED303C
:1000D0000C94ED300C94ED300C94ED300C94ED302C
:1000E0000C94ED302C323132363240324A32C33247
:1000F00054325C3264326E327832823291329B32C8
:10010000C332A532AF32B932E732EA32D932DD3208
:10011000E3322133EE32F232F832FC32003306336E
:100120000A330E332133143318331C331568FB673D
:10013000F867FE67016804681068076821680A6844
:100140000D6889A18FA1A0A1ABA1B3A1C8A1B7A13E
:10015000C8A1BBA1BFA1C8A1C5A100B005B00AB08C
:1001600012B017B01CB021B026B043B043B02BB0D2
:1001700043B030B035B03EB05EB063B068B070B080
:1001800075B07AB07FB084B0A1B0A1B089B0A1B091
:100190008EB093B09CB0BCB0C1B0C6B0CEB0D3B03E
:1001A000D8B0DDB0E2B0FFB0FFB0E7B0FFB0ECB068
:1001B000F1B0FAB01AB11FB124B12CB131B136B1DE
:1001C0003BB140B15DB15DB145B15DB14AB14FB137
:1001D00058B124B229B234B23FB24AB255B260B279
:1001E0006BB2A0B2A0B2A0B2A0B276B2BFB2CBB294
:1001F000DCB2EDB2FEB20FB320B331B369B369B371
:1002000069B369B33FB388B394B3A5B3B6B3C7B307
:10021000D8B3E9B3FAB332B432B432B432B408B4B6
:1002200051B45AB469B474B47FB48AB495B49FB469
:10023000CEB4CEB4CEB4CEB4A7B410B516B527B5EF
:1002400033B53FB556B566B549B676B549B686B548
:1002500049B697B5A3B5B8B5C4B5F6B507B616B6E1
:1002600022B62EB63DB670B679B68DB69CB6ABB694
:10027000C5B6D8B6EDB7EBB6EDB7FEB6EDB712B76B
:1002800024B73CB756B78BB79FB7B1B7C0B7CFB796
:10029000E1B714B81DB831B840B84FB869B87CB8E8
:1002A00091B98FB891B9A2B891B9B6B8C8B8E0B849
:1002B000FAB82FB943B955B964B973B985B9B8B9A2
:1002C000BEB9CDB9D7B9DFB9F4B902BADFBA10BA3D
:1002D000DFBA1EBADFBA2DBA3CBA4DBA64BA99BABF
:1002E000A8BAB7BABFBAC7BAD6BA02C402C409C458
:1002F00009C409C410C410C410C41DC417C417C451
:1003000017C4084AD73B3BCE016E84BCBFFDC12F4A
:100310003D6C74319ABD56833DDA3D00C77F11BEF6
:10032000D9E4BB4C3E916BAAAABE000000803F05F9
:10033000A84CCDB2D44EB93836A9020C50B991862A
:1003400088083CA6AAAA2ABE000000803F000D949F
:1003500051660D9446610D946A3F0D9422194E41E9
:100360004E494E495459494E46CDCCCC3D0AD7232F
:100370003C17B7D13877CC2B329595E6241FB14F77
:100380000A000020410000C84200401C4620BCBEBC
:100390004CCA1B0E5AAEC59D7400000A0B02090C14
:1003A0000D0E08070304010000000000000000001B
:1003B000000000000000000000000000000000003D
:1003C00000000000001211100000000000000000FA
:1003D000000000000000000000000000000000011C
:1003E0000210202008081020401020408002010246
:1003F000010804020101020408102040808040200E
:100400001008040201800402018040201008040248
:1004100001080402010102040810204080010204C6
:100420000810204080050505050705080808080292
:100430000202020A0A08080404040401010101017D
:100440000101010303030303030303040707070C6C
:100450000C0C0C0C0C0C0C02020202060606060622
:100460000606060B0B0B0B0B0B0B0B0000200023DF
:1004700000260029002C002F00320000010000039C
:10048000010601090100002200250028002B002E92
:10049000003100340002010000050108010B0100D9
:1004A000002100240027002A002D00300033000125
:1004B000010000040107010A0101060D00FE090107
:1004C0006602D620FFFE0BFE0AFE0D0060221969AF
:1004D000808080808080800080183363A0A0A0038B
:1004E00057675050F850F850500259692078A0A032
:1004F000702828F02002596948A85010204050A8C0
:100500009002586840A0A040A0989068281363808B
:100510008080113B6B204040808080808040402064
:10052000113B6B8040402020202020404080065519
:100530006520A870A8200455652020F820201133DC
:1005400063604080065161F811336340E040025916
:1005500069080810102040408080025969205088A6
:100560008888888850200259692060A02020202097
:1005700020F80259697088880810204080F80259D4
:1005800069F8081020700808887002596910103046
:10059000505090F81010025969F88080B0C80808CF
:1005A000887002596970888080F088888870025944
:1005B00069F808101020204040400259697088886E
:1005C00088708888887002596970888888780808D7
:1005D000887011386840E040000040E04011386801
:1005E00040E04000006040800259690810204080CF
:1005F00040201008045464F80000F8025969804053
:100600002010081020408002596970888808102046
:1006100020002002596970888898A8A8B0807802C4
:1006200059692050888888F8888888025969F04874
:10063000484870484848F002596970888080808036
:10064000808870025969F048484848484848F00294
:100650005969F8808080F0808080F8025969F880BC
:100660008080F080808080025969708880808098C6
:1006700088887002596988888888F88888888812EC
:100680003969E040404040404040E002596938103C
:1006900010101010109060025969888890A0C0A0B6
:1006A0009088880259698080808080808080F802EC
:1006B00059698888D8A8A88888888802596988C80C
:1006C000C8A8A898988888025969708888888888F6
:1006D000888870025969F0888888F080808080015D
:1006E0005A6A70888888888888A87008025969F0D2
:1006F000888888F0A0908888025969708880807006
:1007000008088870025969F8202020202020202025
:100710000259698888888888888888700259698819
:10072000888888505050202002596988888888A875
:10073000A8A8A8500259698888505020505088882D
:10074000025969888850502020202020025969F8D9
:1007500008101020404080F8113B6BE080808080C2
:100760008080808080E002596980804040201010A5
:100770000808113B6BE0202020202020202020E0D2
:10078000085363205088015161F82A226280400298
:100790005666700878889868025969808080F08869
:1007A000888888F00256667088808088700259694F
:1007B0000808087888888888780256667088F880E3
:1007C000887002596930484040F04040404000582D
:1007D000687088888878088870025969808080B03D
:1007E000C8888888881238684000C040404040E08F
:1007F000004A6A1000301010101090906002596981
:1008000080808090A0C0A09088123969C04040408C
:1008100040404040E0025666D0A8A8A8A8880256EA
:1008200066B0C8888888880256667088888888700C
:10083000005868F0888888F0808080005868788840
:10084000888878080808025666B0C88080808002D0
:1008500056667088601088700258684040F04040CA
:1008600040483002566688888888986802566688AC
:1008700088885050200256668888A8A8A85002563A
:1008800066885020205088005868888888986808B2
:100890008870025666F810204080F8015B6B1820C3
:1008A000202020C0202020201822196980808080EC
:1008B0008080808080015B6BC02020202018202059
:1008C0002020C008536348A890FFFFFFFFFFFFFFF1
:1008D000FFFFFFFFFFFFFFFFFFFFFFFFFFFFFFFF28
:1008E000FFFFFFFFFFFFFFFFFFFF0D006022196901
:1008F0008000808080808080800358682070A8A05D
:10090000A0A8702002596930484040E0404048B0FB
:100910000356668870505070880259698888505014
:10092000F820F82020221969808080800080808053
:1009300080124A6A609080609090601090601A32D5
:1009400062A0A00359697088A8D8C8D8A888700484
:100950005767700878887800F80356662850A0A07A
:100960005028045363F80808163161E00359697090
:1009700088E8D8D8E8D888700A5161F817446460CC
:100980009090600357672020F8202000F807356515
:1009900040A02040E007356540A04020C02A2262E8
:1009A00040800058688888888898E8808002596963
:1009B00078E8E8E8E868282828262161C020226233
:1009C000408007356540C04040E004576770888824
:1009D000887000F8035666A050282850A0025A6A72
:1009E00040C04040E00818283808025A6A40C04019
:1009F00040E01028081038025A6A40A04020A04861
:100A00001828380802596920002020408088887002
:100A1000025A6A40200020508888F88888025A6A62
:100A200010200020508888F88888025A6A304800D0
:100A300020508888F88888025A6A285000205088F8
:100A400088F88888025A6A50500020508888F888B0
:100A500088025A6A20502020508888F888880259D5
:100A60006958A0A0A0B0E0A0A0B8005B6B7088801F
:100A70008080808088702040025A6A402000F88080
:100A800080F08080F8025A6A102000F88080F080A0
:100A900080F8025A6A304800F88080F08080F802BE
:100AA0005A6A505000F88080F08080F8123A6A80CC
:100AB0004000E04040404040E0123A6A204000E000
:100AC0004040404040E0124A6A609000E0404040B0
:100AD0004040E0123A6AA0A000E04040404040E0C0
:100AE000025969F0484848E8484848F0025A6A28DC
:100AF00050008888C8A8988888025A6A40200070E8
:100B0000888888888870025A6A10200070888888CF
:100B1000888870025A6A304800708888888888708F
:100B2000025A6A28500070888888888870025A6A39
:100B300050500070888888888870035565885020D8
:100B40005088015B6B08709898A8A8A8C8C87080E6
:100B5000025A6A40200088888888888870025A6A09
:100B600010200088888888888870025A6A30480077
:100B700088888888888870025A6A505000888888D7
:100B800088888870025A6A102000888850202020A7
:100B90002002596980F0888888F080808002596935
:100BA000609090A0A0908888B002596940200070A1
:100BB0000878889868025969102000700878889829
:100BC0006802596930480070087888986802596945
:100BD0002850007008788898680259695050007051
:100BE0000878889868025A6A304830007008788817
:100BF0009868025666702870A0A8500058687088DF
:100C00008080887020400259694020007088F880F8
:100C100088700259691020007088F8808870025925
:100C2000693048007088F880887002596950500017
:100C30007088F8808870123969804000C040404058
:100C400040E0123969204000C040404040E0124975
:100C500069609000C040404040E0123969A0A000A7
:100C6000C040404040E0025A6A50206010708888BE
:100C7000888870025969285000B0C888888888021E
:100C8000596940200070888888887002596910204E
:100C90000070888888887002596930480070888898
:100CA0008888700259692850007088888888700286
:100CB00059695050007088888888700357672020D1
:100CC00000F8002020015868087098A8A8C8708013
:100CD00002596940200088888888986802596910FC
:100CE0002000888888889868025969304800888878
:100CF0008888986802596950500088888888986860
:100D0000005B6B1020008888889868088870005AFB
:100D10006A8080B0C88888C8B08080005B6B505003
:100D200000888888986808887001050700FE05001B
:100D3000FB01F220FFFE05FE05FE02004002152524
:100D40008080800080053242A0A002556550F85096
:100D5000F8500146562070C030E0200255659010D2
:100D600020404802556560806890680512228080A6
:100D700002253540808080400225358040404080FB
:100D8000043343A040A003334340E04001223240FB
:100D900080043141E0021121800255650810204095
:100DA000800245556090909060022535C0404040DB
:100DB00040024555E0106080F0024555E01060109B
:100DC000E00245552060A0F020024555F080E0107B
:100DD000E00245556080E09060024555F0102040EB
:100DE00040024555609060906002455560907010DB
:100DF0006003132380008002142480008080023569
:100E0000452040804020033343E000E00235458028
:100E100040204080024555E010600040025565705A
:100E200088B8A870024555609090F090024555E052
:100E300090E090E00235456080808060024555E09A
:100E4000909090E0023545E080E080E0023545E09A
:100E500080E080800245557080B0907002455590CA
:100E600090F09090023545E0404040E0024555301A
:100E70001010906002455590A0C0A09002354580AA
:100E8000808080E002556588D8A888880245559002
:100E9000D0B090900245556090909060024555E02A
:100EA0009090E08001465660909090601002455509
:100EB000E09090E09002455570806010E00235456A
:100EC000E04040404002455590909090600245556A
:100ED0009090A0A04002556588A8A8A8500245554A
:100EE000909060909002455590907010600235454A
:100EF000E0204080E0022535C0808080C00255653A
:100F00008040201008022535C0404040C0053242D4
:100F100040A0024151F005223280400244547090BA
:100F2000907002455580E09090E0023444608080EB
:100F300060024555107090907002445460B0C060DB
:100F40000235452040E040400046567090907010B9
:100F50006002455580E090909002152580008080C9
:100F60008000273740004040404080024555809037
:100F7000A0E0900215258080808080025464F0A853
:100F8000A8A8024454E0909090024454609090606D
:100F9000004656E09090E080800046567090907039
:100FA0001010023444A0C0808002445470C030E06D
:100FB00002354540E0404020024454909090700239
:100FC00044549090A040025464A8A8505002344465
:100FD000A04040A00046569090907010600244548B
:100FE000F02040F0023545604080406002152580C9
:100FF00080808080023545C0402040C0054252506C
:10100000A0FFFFFFFFFFFFFFFFFFFFFFFFFFFFFF4F
:10101000FFFFFFFFFFFFFFFFFFFFFFFFFFFFFFFFE0
:10102000FFFF020040FFFFFFFFFFFFFFFFFFFFFF8B
:10103000FFFFFFFFFFFFFFFFFFFFFFFFFFFFFFFFC0
:10104000FFFFFFFFFFFFFFFFFFFFFFFFFFFFFFFFB0
:10105000FFFFFFFFFFFFFFFFFFFFFFFFFFFFFFFFA0
:10106000FFFFFFFFFFFFFFFFFFFFFFFFFFFFFFFF90
:10107000FFFFFFFFFFFFFFFFFFFFFFFFFFFFFFFF80
:10108000FFFFFFFF01050800FF060121023520FFD9
:10109000FF07FF06FF09005022165680808080005F
:1010A00080153353A0A0A00257575050F850F85065
:1010B000500257572070A07028702013355580A01B
:1010C00040A02002475740A0A040A0A050251353A5
:1010D0008080801226564080808080401226568074
:1010E00040404040800245559060F0609002555568
:1010F0002020F82020113353604080044151F0112A
:10110000335340E040024656101020408080123693
:101110005640A0A0A0A04012365640C0404040E03B
:101120000246566090106080F0024656F020601033
:1011300090600246562060A0F02020024656F080C3
:10114000E01090600246566080E090906002465643
:10115000F01020204040024656609060909060025F
:101160004656609090701060122555C0C000C0C0F7
:1011700011365660600060408012365620408080F4
:101180004020034353F000F01236568040202040A8
:101190008012365640A020400040015858304898F0
:1011A000A8A8904030024656609090F09090024679
:1011B00056E090E09090E00246566090808090600B
:1011C000024656E090909090E0024656F080E08013
:1011D00080F0024656F080E08080800246566090A3
:1011E00080B090600246569090F0909090123656E3
:1011F000E040404040E002465670202020A04002DF
:10120000465690A0C0A0A090024656808080808064
:10121000F002465690F0F090909002465690D0F032
:10122000B0B090024656609090909060024656E0B2
:101230009090E08080014757609090D0B06010029D
:101240004656E09090E09090024656609040209084
:1012500060123656E0404040404002465690909022
:101260009090600246569090909060600246569032
:101270009090F0F0900246569090606090900256E8
:1012800056888850202020024656F010204080F0DA
:10129000123656E080808080E002465680804020F2
:1012A0001010123656E020202020E016325240A0C6
:1012B000014151F0162252804002445470909070C7
:1012C0000246568080E09090E01234546080806046
:1012D00002465610107090907002445460B0C06086
:1012E000024656205040E040400145556090701045
:1012F000600246568080E09090901236564000C0C2
:101300004040E01137572000202020A040024656E0
:10131000808090E09090123656C040404040E002FD
:101320005454D0A8A8A8024454E090909002445489
:1013300060909060014555E090E0808001455570D7
:1013400090701010024454A0D0808012345460C0B9
:1013500020C00246564040E0405020024454909045
:101360009070123454A0A0A04002545488A8A850F1
:1013700002445490606090014555909070906002D6
:101380004454F02040F0024757304020C020403005
:10139000221656808080808080024757C0204030CF
:1013A0004020C006425250A0FFFFFFFFFFFFFFFF9B
:1013B000FFFFFFFFFFFFFFFFFFFFFFFFFFFFFFFF3D
:1013C000FFFFFFFFFFFFFFFFFF09005022165680BF
:1013D00000808080800146562070A0A070200246C8
:1013E000562050E04050A002555588705070880239
:1013F00056568850F820F8202217578080800080A9
:1014000080800247577080E0907010E0173151A043
:1014100002565670A8C8C8A87014355560A0600060
:10142000E003435350A050123353E02020143151B5
:10143000E002565670E8D8E8D870173151E01533FD
:101440005340A04012355540E04000E0143555406F
:10145000A02040E0143555C020C020C016225240C4
:1014600080014555909090E08002565678E8E868F3
:10147000282824115180112252408014355540C033
:101480004040E014355540A04000E0034353A050D5
:10149000A0024757808080A060F0200247578080DC
:1014A000A0D010207002475780408060A0F020122A
:1014B000365640004080A04002475740206090F0E0
:1014C000909002475720406090F0909002475760FC
:1014D000906090F0909002475750A06090F09090EC
:1014E00002475790006090F09090024757609060DC
:1014F00090F0909002465670A0A0F0A0B00147571F
:10150000609080809060400247574020F080E080EB
:10151000F00247572040F080E080F002475760908B
:10152000F080E080F00247579000F080E080F012F9
:1015300037578040E0404040E01237572040E040BD
:101540004040E012375740A0E0404040E01237579B
:10155000A000E0404040E00256567048E84848701D
:1015600002475750A090D0B090900247574020605B
:1015700090909060024757204060909090600247A2
:10158000576090609090906002475750A060909094
:10159000906002475790006090909060123353A083
:1015A00040A002465670B0B0D0D0E002475740206D
:1015B00090909090600247572040909090906002E9
:1015C000475760909090909060024757900090909D
:1015D00090906002575710208850202020024656D5
:1015E00080E09090E0800246566090A0A090A0021B
:1015F000475740200070909070024757204000707D
:10160000909070024757205000709090700247579A
:1016100050A00070909070024656500070909070EC
:1016200002475760906070909070025454F068B018
:101630007811355560808060400247574020006037
:10164000B0C06002475720400060B0C060024757FA
:1016500060900060B0C060024656500060B0C0604C
:10166000123757804000C04040E0123757204000FA
:10167000C04040E012375740A000C04040E0123662
:1016800056A000C04040E0024757A040A010709014
:101690006002475750A000E09090900247574020CA
:1016A0000060909060024757204000609090600278
:1016B00047576090006090906002475750A00060CC
:1016C00090906002465690006090906012355540B0
:1016D00000E0004002445470B0D0E0024757402080
:1016E00000909090700247572040009090907002B8
:1016F00047576090009090907002465690009090EE
:1017000090700148582040009090709060014757B9
:101710008080E090E080800147579000909070902A
:101720006025753A2530327500253032753A2530FE
:1017300032750020202020002520200025200025B3
:1017400031640025326400253364002534640025AB
:10175000356400253664000000007E0060006000F3
:1017600060F87ECC60CC60CC60F860CC00CC00CC63
:1017700000CC00000000000000FE7F0E70266472A6
:101780004E7A5E324C8241324C7A5E724E26640E44
:1017900070FE7F000000000000FE7F0E70C663C276
:1017A0004382411A58BA5D1A588241C243C6630E39
:1017B00070FE7F00000000000088088808101120DB
:1017C0002220221011880888081011000000000053
:1017D000000000000000000000202210118808888E
:1017E000081011202220221011880800000000009B
:1017F00000000000000000000000000000000000E9
:1018000000000000000000000000000000FE7FFE5D
:101810007F06600000000000000000F00FF81FF8D5
:101820001FF81FF00FF00FF81FF81FF81FE007C098
:1018300003800100000000304848304572723A20B1
:101840007574663820666F6E74206E6F7420696ED2
:10185000697469616C697A65642E004572723A2018
:101860007574663820666F6E74206E6F7420696EB2
:10187000697469616C697A65642E004572723A20F8
:101880007574663820666F6E74206E6F7420696E92
:10189000697469616C697A65642E00506C65617366
:1018A00065207265736574005052494E544552204C
:1018B00048414C544544007F80FFC0FFC0FFC07FBB
:1018C000807F80FFC0FFC0FFC03F001E000C00FFF4
:1018D000FFFF0E000E000E000E000E000E000E00A8
:1018E0000E007FC03F801F000E00040004000E00A9
:1018F0001F003F807FC00E000E000E000E000E0085
:101900000E000E000E0000FE0003FF800783C00ED5
:1019100001C00E00E01C00E07F00E03E00E01C0083
:10192000E00800E00000E00001C00E01C00F0780E9
:1019300007FF0001FC0003F8000FFE001E0F003837
:101940000700380380700380700FE07007C07003D9
:10195000807001007000003800003807001E0F0082
:101960000FFE0003F80000060C00FE07022603BC71
:10197000017FFE08FE08FE05080806000040F0C8CA
:101980008888987810050808060000C0F8888888BC
:101990008888F80505050600012030F83020050884
:1019A000080600002070F820202020E00509090624
:1019B00000FF2070A8A8B8888870200506060600D9
:1019C00001E08CEA8C8A0A0509090600FFF8A8885C
:1019D00088888888A8F8050A0A0600FE205050501A
:1019E0005088A8A8887003030306000340A040FFA6
:1019F000FFFFFFFFFFFFFFFFFFFFFFFFFFFFFFFFF7
:101A0000FFFFFFFFFF0000000605FF0107070602BA
:101A10000080808080800080030303060105A0A071
:101A2000A005060606000050F85050F850050909B8
:101A30000600FF2070A8A07028A8702005070706E0
:101A40000000C8C81020409898050707060000400D
:101A5000A0A040A8906801030306020580808003CF
:101A600009090601FF204040808080404020030992
:101A7000090601FF804040202020404080050707E4
:101A800006000020A8702070A820050505060001AA
:101A90002020F820200203030601FFC0408005013A
:101AA00001060003F8020202060100C0C005070794
:101AB00006000008101020404080050707060000BF
:101AC000708898A8C8887003070706010040C040C6
:101AD000404040E0050707060000708808102040DD
:101AE000F8050707060000F8081030088870050799
:101AF0000706000010305090F81010050707060088
:101B000000F880F0080888700507070600003040DC
:101B100080F0888870050707060000F8081010207C
:101B200020200507070600007088887088887005E7
:101B3000070706000070888878081060020505060F
:101B40000100C0C000C0C00206060601FFC0C00000
:101B5000C0408003050506010120408040200503A8
:101B600003060002F800F803050506010180402085
:101B7000408005070706000070881020200020051F
:101B800007070600007088B8A8B880700507070628
:101B90000000708888F8888888050707060000F02C
:101BA0004848704848F005070706000070888080A4
:101BB000808870050707060000F04848484848F04C
:101BC000050707060000F88080F08080F805070709
:101BD000060000F88080F08080800507070600007E
:101BE00070888080988870050707060000888888BC
:101BF000F8888888030707060100E040404040401D
:101C0000E005070706000038101010109060050767
:101C1000070600008890A0C0A0908805070706006E
:101C200000808080808080F805070706000088D843
:101C3000A8888888880507070600008888C8A898AB
:101C400088880507070600007088888888887005DE
:101C50000707060000F08888F080808005070706E7
:101C6000000070888888A89068050707060000F0C3
:101C70008888F0A0908805070706000070888070AB
:101C8000088870050707060000F820202020202083
:101C90000507070600008888888888887005070778
:101CA0000600008888888850502005070706000035
:101CB00088888888A8A850050707060000888850EB
:101CC00020508888050707060000888850202020BB
:101CD00020050707060000F80810204080F80309D7
:101CE000090601FFE080808080808080E005070792
:101CF000060000804040201010080309090601FF7B
:101D0000E020202020202020E005030306000520FD
:101D100050880501010600FEF80303030601058053
:101D2000402005050506000070087888780507073B
:101D30000600008080F0888888F005050506000010
:101D4000708080887005070706000008087888887A
:101D500088780505050600007088F0807005070783
:101D6000060000304840E04040400507070600FEFE
:101D7000708888887808700507070600008080F062
:101D8000888888880307070601004000C04040405B
:101D9000E00409090601FE100030101010109060D8
:101DA00005070706000080808890E09088030707F9
:101DB000060100C04040404040E005050506000027
:101DC000D0A8A8A8A8050505060000B0C88888887E
:101DD000050505060000708888887005070706005D
:101DE000FEF0888888F080800507070600FE788866
:101DF0008888780808050505060000B0C88080803E
:101E000005050506000078807008F0050707060044
:101E1000002020F8202020180505050600008888ED
:101E20008898680505050600008888885020050503
:101E3000050600008888A8A850050505060000884A
:101E4000502050880507070600FE888888502040EB
:101E500080050505060000F8102040F80309090672
:101E600001FF204040408040404020010909060217
:101E7000FF8080808080808080800309090601FFC8
:101E80008040404020404040800503030600024857
:101E9000A890FF1FFFFFFFFFFFFF60000000000191
:101EA000FF400000000000FF8000000000007F8372
:101EB000CF00000C303F87FF80000C301F867980F8
:101EC000000C000F8C30C7838C30E78C30CFC7CC30
:101ED00031F38C30DCECEC33B98C30D86C6C3319CA
:101EE0008C30D06C0C33198C30D86C0C33198C308E
:101EF000DC6C0E3B198C30CF7C079F198C30C77C73
:101F0000038F194000000000000260000000000084
:101F1000061FFFFFFFFFFFF80000000000000000A9
:101F200000000000000000000000000000000000B1
:101F300000000000000000000000000C0000000095
:101F40000000000C00000000000000120000000073
:101F5000000000230000000000000021000000003D
:101F60000000004C800000000000005E80000000C7
:101F70000000009240000000000000A140000000AE
:101F800000000121200000000000027F90000000FE
:101F90000000020010000000000007FFF800000031
:101FA0000000040008000000000008000400000019
:101FB0000000080006000000000010000200000001
:101FC0000000301E010000000000207F81000000A2
:101FD000000041FFE0800000000043FCF0800000B2
:101FE0000000873B7840000000018EDBFC600000B1
:101FF00000010FEBCC20000000021FEDB610000026
:1020000000021FDEB6100000000439CD7F0800007A
:10201000000436E0FF08000000087EC0BB8400001A
:1020200000187F005D86000000107FC0ED82000078
:1020300000203CC07301000000203B337F01000002
:1020400000701BE77E03800000C81DEEDE04C000A8
:1020500000880FDEDC04400001240FDF3C09200073
:10206000012607DBF8192000027203E7F013900045
:10207000025101FFE02290000489007F8024480083
:102080000904801E004824000BFE400000DFF4001D
:1020900010004000008002001FFFFFFFFFFFFE0056
:1020A0000000000000000000000000000000000030
:1020B00000000000000000001022103C3C0E1F0039
:1020C0001022100422110400102210082211040012
:1020D000102210083C1104001022101022110400DC
:1020E00010221020221104001E1C1E3C3C0E040075
:1020F00000000000000000000000000000000000E0
:1021000000000000000000000000000000000000CF
:1021100000000000000000000000000000000000BF
:1021200000000000000000000000000000000000AF
:10213000000000000000000000000000000000009F
:10214000000000000000000000000000000000008F
:1021500000000000000000060900FE06018902FEE2
:1021600020FFFE07FE06FE0000000600070106062F
:10217000060200808080800080030303060103A024
:10218000A0A00507070600FF5050F850F850500572
:1021900009090600FE2070A8A07028A87020060873
:1021A000080600FF40A84810204854080507070605
:1021B00000FF60909060989068010303060203801E
:1021C00080800207070602FF4080808080804002F6
:1021D00007070602FF804040404040800505050695
:1021E00000008850F850880505050600002020F8FA
:1021F00020200204040602FEC040408005010106C2
:102200000002F8020202060200C0C004060606012F
:1022100000101020408080040606060100609090A7
:1022200090906003060606010040C0404040E00474
:1022300006060601006090102040F0040606060124
:1022400000F020601010E005060606000010305077
:1022500090F810040606060100F080E01010E0047B
:1022600006060601006080E0909060040606060104
:1022700000F0101020404004060606010060906047
:102280009090600406060601006090907010600255
:102290000505060200C0C000C0C00207070602FE16
:1022A000C0C000C0404080050505060000186080E1
:1022B0006018050303060001F800F805050506008F
:1022C00000C0300830C004070706010060901060AD
:1022D0004000400506060600007090A8B08070051A
:1022E0000606060000205088F888880506060600C5
:1022F00000F088F08888F0040606060100609080EF
:10230000809060040606060100E090909090E00442
:102310000606060100F080E08080F0040606060153
:1023200000F080E080808004060606010060908056
:10233000B090600406060601009090F09090900323
:102340000606060100E040404040E00506060600A3
:102350000038101010906004060606010090A0C01E
:10236000A090900406060601008080808080F00521
:10237000060606000088D8A8A88888040606060174
:102380000090D0B0909090050606060000708888F6
:10239000888870040606060100E09090E0808004C2
:1023A00007070601FF609090D0B060100406060693
:1023B0000100E09090E09090040606060100609015
:1023C00040209060050606060000F820202020200E
:1023D00004060606010090909090906004060606A0
:1023E0000100909090F06060050606060000888865
:1023F000A8A8D88805060606000088502020508826
:1024000005060606000088885020202004060606DF
:102410000100F010204080F0030606060100E08075
:10242000808080E0040606060100808040201010B5
:10243000030606060100E020202020E00503030635
:1024400000032050880501010600FEF80202020682
:102450000204804004040406010070909070040699
:10246000060601008080E09090E00404040601006C
:102470007080807004060606010010107090907045
:1024800004040406010060B0C070040606060100E2
:10249000205040E040400406060601FE6090907027
:1024A00010600406060601008080E090909003060C
:1024B000060601004000C04040E00308080601FE97
:1024C000200060202020A040040606060100808035
:1024D000A0C0A090030606060100C040404040E0B6
:1024E000050404060000D0A8A8880404040601001E
:1024F000E09090900404040601006090906004064F
:10250000060601FEE09090E080800406060601FECB
:10251000709090701010040404060100A0D0808018
:1025200004040406010070C030E004060606010041
:102530004040E04050200404040601009090907058
:102540000404040601009090606005040406000085
:1025500088A8A85004040406010090606090040656
:10256000060601FE9090907090600404040601003D
:10257000F02040F003070706010020404080404063
:10258000200107070602FF8080808080808003078B
:1025900007060100804040204040800402020601FE
:1025A0000350A0FFFFFFFFFFFFFFFFFFFFFFFFFF45
:1025B000FFFFFFFFFFFFFFFFFFFFFFFFFFFFFFFF2B
:1025C000FFFFFFFF000000060007010606060200ED
:1025D0008000808080800406060601FF2070A0A095
:1025E00070200507070600FF304840F04040F8051E
:1025F0000505060000A8508850A80506060600003C
:102600008850F820F8200107070602FF808080002C
:102610008080800407070601FF708060906010E0F2
:10262000030101060105A00607070600007884944F
:10263000A494847803050506010160A06000E0050C
:1026400005050600002850A05028040303060100D9
:10265000F01010040101060102F006070706000051
:102660007884B4A4A48478040101060105F004036D
:10267000030601026090600507070600FF2020F8AE
:10268000202000F803050506010140A02040E003DA
:102690000505060101C0204020C002020206020416
:1026A00040800405050601FF9090B0D08005060625
:1026B00006000078E8E86828280101010602028087
:1026C0000202020602FE408003050506010140C029
:1026D0004040E003050506010140A04000E005057B
:1026E00005060000A0502850A00508080600FF407D
:1026F000C04050703078100508080600FF40C04008
:1027000050680810380508080600FFC0204030F067
:1027100030781004070706010020002060809060D8
:10272000050707060000402020507088880507072D
:10273000060000102020507088880507070600005A
:102740002050205070888805070706000028502078
:1027500050708888050707060000500020507088D8
:10276000880507070600002050205070888805065D
:102770000606000078A0F0A0A0B80408080601FE34
:102780006090808090602040040707060100402090
:10279000F080E080F00407070601002040F080E0B0
:1027A00080F00407070601002050F080E080F0046C
:1027B00007070601005000F080E080F003070706DD
:1027C00001008040E0404040E00307070601002090
:1027D00040E0404040E003070706010040A0E04021
:1027E0004040E0030707060100A000E0404040E051
:1027F0000506060600007048E8484870040707060A
:10280000010050A090D0B09090040707060100404E
:1028100020609090906004070706010020406090BF
:10282000909060040707060100205060909090602F
:1028300004070706010050A060909090600407070D
:1028400006010050006090909060050505060000AC
:1028500088502050880408080601FF1070B0B0D0DE
:10286000D0E080040707060100402090909090601F
:10287000040707060100204090909090600407072D
:102880000601002050909090906004070706010018
:102890005000909090906005070706000010208877
:1028A0005020202004060606010080E09090E08081
:1028B0000406060601006090A0A090A00407070689
:1028C000010040200070909070040707060100206E
:1028D00040007090907004070706010020500070BF
:1028E00090907004070706010050A000709090704F
:1028F0000406060601005000709090700407070659
:1029000001002050207090907005040406000070B3
:10291000A8B0780406060601FE708080702040048E
:10292000070706010040200060B0C07004070706DA
:10293000010020400060B0C07004070706010020BD
:10294000500060B0C070040606060100500060B080
:10295000C070030707060100804000C04040E0034C
:102960000707060100204000C04040E003070706BB
:10297000010040A000C04040E0030606060100A0A0
:1029800000C04040E004070706010030601070906E
:10299000906004070706010050A000E090909004AA
:1029A00007070601004020006090906004070706BA
:1029B000010020400060909060040707060100209D
:1029C00050006090906004070706010050A000606E
:1029D000909060040606060100500060909060052B
:1029E00005050600002000F800200404040601008C
:1029F00070B0D0E0040707060100402000909090DE
:102A000070040707060100204000909090700407B2
:102A10000706010020500090909070040606060101
:102A2000005000909090700409090601FE204000BB
:102A30009090907090600408080601FE8080E090FD
:102A400090E080800408080601FE5000909090708D
:102A500090605072696E742066726F6D20534400EE
:102A60005072696E742066726F6D20534400022E9E
:102A70002E004D61696E0046696C616D656E740073
:102A8000544D4320647269766572730053746570A7
:102A9000732F6D6D004A65726B00416363656C65F1
:102AA000726174696F6E0056656C6F63697479004A
:102AB000436F6E66696775726174696F6E00457306
:102AC000746570732F6D6D004573746570732F6D31
:102AD0006D005A73746570732F6D6D005A73746551
:102AE00070732F6D6D005973746570732F6D6D0069
:102AF0005973746570732F6D6D00587374657073BE
:102B00002F6D6D005873746570732F6D6D00416487
:102B100076616E6365642053657474696E677300D3
:102B200056652D6A65726B0056652D6A65726B007D
:102B3000567A2D6A65726B00567A2D6A65726B0043
:102B400056792D6A65726B0056792D6A65726B0035
:102B500056782D6A65726B0056782D6A65726B0027
:102B6000416476616E6365642053657474696E6751
:102B70007300416D6178204500416D61782045000A
:102B8000416D6178205A00416D6178205A00416D95
:102B90006178205900416D6178205900416D61785C
:102BA000205800416D6178205800412D7472617683
:102BB000656C00412D74726176656C00412D726503
:102BC000747261637400412D726574726163740084
:102BD000416363656C00416363656C0041647661C9
:102BE0006E6365642053657474696E677300565430
:102BF000726176206D696E005654726176206D693F
:102C00006E00566D696E00566D696E00566D617886
:102C1000204500566D6178204500566D6178205A38
:102C200000566D6178205A00566D61782059005623
:102C30006D6178205900566D6178205800566D619D
:102C400078205800416476616E6365642053657432
:102C500074696E6773004C6F6164206D6D004C6F1A
:102C60006164206D6D00556E6C6F6164206D6D0048
:102C7000556E6C6F6164206D6D00416476616E63AA
:102C800065204B00416476616E6365204B004164B2
:102C900076616E6365642053657474696E67730052
:102CA00044697361626C65207374657070657273DA
:102CB000004D3834004C6576656C205820417869A9
:102CC00073004D313137204C6576656C696E672035
:102CD0005820417869730A4732380A473020583102
:102CE00036302046393939390A4730205A3520469E
:102CF000363030300A4739310A4D323131205330C5
:102D00000A4D3430300A4D393036205A3630300AC8
:102D10004730205A2D313520463530300A47302093
:102D20005A3520463530300A4739300A4D34303074
:102D30000A4D393036205A3936300A4D3231312079
:102D400053310A4732380A4D313137204C657665A8
:102D50006C696E6720646F6E652E0A004175746F32
:102D600020686F6D6500473238004D6F76652061D1
:102D7000786973004D61696E004578747275646599
:102D80007220004175746F20686F6D65004732389E
:102D9000004D6F7665205A004D6F76652059004DC5
:102DA0006F76652058004D6F76656D656E740045D1
:102DB0007874727564657220004D6F766520302ED0
:102DC000316D6D004D6F766520316D6D004D6F7604
:102DD000652031306D6D004D6F76652061786973C7
:102DE00000486F74656E6420746F6F20636F6C644D
:102DF00000457874727564657220004D6F766520A9
:102E00005A004D6F76652059004D6F766520580049
:102E10004D6F7665205A004D6F76652059004D6FD5
:102E200076652058005761697420666F7200666984
:102E30006C616D656E742070757267650000506C12
:102E40006561736520776169742E005072657373D4
:102E500020627574746F6E00746F20726573756D87
:102E600065207072696E74005761697420666F72B4
:102E70000066696C616D656E74206C6F61640049F9
:102E80006E736572742066696C616D656E74006145
:102E90006E6420707265737320627574746F6E0057
:102EA000746F20636F6E74696E7565005072657320
:102EB0007320627574746F6E00746F20686561743E
:102EC000206E6F7A7A6C65004E6F7A7A6C65206836
:102ED000656174696E6700506C6561736520776128
:102EE00069742E2E2E005761697420666F72006619
:102EF000696C616D656E7420756E6C6F61640057EE
:102F000061697420666F720066696C616D656E74CC
:102F1000206368616E676500746F207374617274FA
:102F2000004368616E67696E672046696C616D6514
:102F30006E7400554E4C4F41442046494C414D451E
:102F40004E54004C4F41442046494C414D454E544F
:102F50000020204E6F7A7A6C653A20002000456E82
:102F6000642066696C616D656E74206368616E676C
:102F700065005075726765206D6F7265000043686B
:102F8000616E67652066696C616D656E7400556E73
:102F90006C6F61642066696C616D656E74004C6F66
:102FA00061642066696C616D656E74004D36303009
:102FB00020423020542564004D373032203B2564B8
:102FC000004D37303220542564004D3730312054C5
:102FD0002564005072656865617420437573746F71
:102FE0006D005072656865617420437573746F6D10
:102FF00000507265686561742041425300507265EB
:103000006865617420504C41004261636B004E6FF3
:103010002053442063617264005072696E742066AC
:10302000726F6D2053440041626F75742050726955
:103030006E746572004368616E67652066696C61D5
:103040006D656E74004368616E67652066696C61CA
:103050006D656E74004D36303020423000436F6E27
:1030600066696775726174696F6E0054656D70652D
:10307000726174757265004D6F76656D656E740072
:10308000526573756D65207072696E740054756E4B
:10309000650053746F70207072696E7400506175B2
:1030A0007365207072696E7400496E666F20736379
:1030B0007265656E005072696E746572205374613A
:1030C0007473004669726D7761726520566572731C
:1030D000696F6E004D61696E0053746F702070727D
:1030E000696E74004D61696E005072696E74206182
:1030F000626F72746564004D3234004D3235205079
:103100000A4D32340050726F6265205A204F666655
:10311000736574004261627973746570205900426E
:1031200061627973746570205800466C6F77004651
:103130006C6F770046616E20737065656400466150
:103140006E207370656564004265640042656400CA
:103150004E6F7A7A6C65004E6F7A7A6C65005370A8
:10316000656564005370656564004D61696E004279
:103170006162797374657020590042616279737479
:1031800065702058002569730025696D20256973D5
:10319000002569682025696D20256973002569640B
:1031A000202569682025696D2025697300256979C6
:1031B00020256964202569682025696D20256973AB
:1031C000003E2000457874727564656420746F74E5
:1031D000616C3A00256C642E25696D003E20004C20
:1031E0006F6E67657374206A6F622074696D653AEB
:1031F000003E2000546F74616C207072696E742000
:1032000074696D653A00436F6D706C657465643AFE
:1032100020005072696E7420436F756E743A2000FE
:10322000436F6F6C646F776E0046616E20737065DC
:1032300065640046616E2073706565640042656474
:1032400000426564004E6F7A7A6C65004E6F7A7A40
:103250006C65004D61696E00526573746F72652014
:103260006661696C73616665004C6F6164207365AB
:103270007474696E67730053746F7265207365743C
:1032800074696E67730050726F6265205A204F66D2
:103290006673657400416476616E6365642053658E
:1032A0007474696E6773004D61696E0050726F626D
:1032B00065205A204F66667365740053746570709C
:1032C000696E67206D6F64650053656E736F726C15
:1032D00065737320686F6D696E6700487962726903
:1032E00064207468726573686F6C640044726976F8
:1032F00065722063757272656E7400436F6E7472CE
:103300006F6C004530004F6666004F6E0045300020
:103310005A004F6666004F6E005A0059004F6666AD
:10332000004F6E00590058004F6666004F6E0058FF
:1033300000544D432064726976657273005374655E
:10334000616C746843686F7020656E61626C65645F
:10335000005900590058005800544D4320647269C8
:1033600076657273004530004530005A005A0059A6
:1033700000590058005800544D4320647269766526
:103380007273004530004530005A005A0059005908
:103390000058005800544D4320647269766572737A
:1033A000004D696E6920322072656164792E00508B
:1033B00072696E74696E672E2E2E005072696E747B
:1033C0002070617573656400436172642072656D7D
:1033D0006F766564004361726420696E7365727410
:1033E0006564004D33310043616E6E6F7420656E0D
:1033F000746572207375626469723A20006F70653B
:103400006E206661696C65642C2046696C653A20A3
:10341000006175746F25632E67006572726F72208C
:1034200077726974696E6720746F2066696C650ACB
:10343000004E6F74205344207072696E74696E6719
:103440000A005344207072696E74696E6720627955
:103450007465200044656C6574696F6E20666169EF
:103460006C65642C2046696C653A200046696C6581
:103470002064656C657465643A0057726974696E9E
:103480006720746F2066696C653A20006F70656E06
:10349000206661696C65642C2046696C653A200081
:1034A0006F70656E206661696C65642C2046696C7E
:1034B000653A200046696C652073656C65637465C8
:1034C000640A002053697A653A200046696C6520D9
:1034D0006F70656E65643A20002066696C653A20FD
:1034E00000667265736800646F696E67004E6F777F
:1034F0002000454E4420535542524F5554494E45A5
:103500000A002220706F73002220706172656E7451
:103510003A2200535542524F5554494E452043419B
:103520004C4C207461726765743A22007472796938
:103530006E6720746F2063616C6C207375622D67F9
:10354000636F64652066696C6573207769746820B1
:10355000746F6F206D616E79206C6576656C732E6B
:10356000204D4158206C6576656C2069733A310AAC
:10357000004D3234004D3233202573005344206314
:10358000617264206F6B0A006F70656E526F6F74AA
:10359000206661696C65640A00766F6C756D652ED6
:1035A000696E6974206661696C65640A0053442021
:1035B000696E6974206661696C0A00286E6F206606
:1035C000696C65290043616E6E6F74206F70656E63
:1035D0002073756264697220007C3C3E5E2B3D3F27
:1035E0002F5B5D3B2C2A225C004F4646004F4E006D
:1035F0006563686F3A004572726F723A0045727285
:103600006F722077726974696E6720746F20454508
:1036100050524F4D210A00507265737320627574C9
:10362000746F6E20286F72204D3130382920746FEE
:103630002068656174206E6F7A7A6C650A0050723A
:1036400065737320627574746F6E20286F72204DDD
:103650003130382920746F20726573756D650A00EA
:10366000496E736572742066696C616D656E742055
:10367000616E6420707265737320627574746F6E0E
:1036800020286F72204D313038290A004D363030F5
:103690003A20546F6F20636F6C6400486F74656EDE
:1036A0006420746F6F20636F6C640A00486F7465E8
:1036B0006E6420746F6F20636F6C640A00496E73D0
:1036C0006572742066696C616D656E7420616E64EC
:1036D00020707265737320627574746F6E20286F2A
:1036E00072204D313038290A004C4F570048494765
:1036F00048004F4B004572726F723A20416C6C204B
:103700000020636F6E6E656374696F6E2E2E2E20BF
:103710000054657374696E6720004C4F5700484928
:103720004748004F4B004572726F723A20416C6CF3
:10373000200020636F6E6E656374696F6E2E2E2E8F
:10374000200054657374696E6720004C4F57004821
:10375000494748004F4B004572726F723A20416CE6
:103760006C200020636F6E6E656374696F6E2E2E21
:103770002E200054657374696E6720004C4F57000B
:1037800048494748004F4B004572726F723A2041DA
:103790006C6C200020636F6E6E656374696F6E2EB3
:1037A0002E2E200054657374696E672000544D43BB
:1037B00020434F4E4E454354494F4E204552524FA1
:1037C00052004452565F53544154555309005057C8
:1037D0004D5F5343414C45090050574D434F4E46B2
:1037E0000900434F4F4C434F4E46090043484F504A
:1037F000434F4E460900544849474809090054437D
:103800004F4F4C5448525309005450574D5448524E
:10381000530900545354455009090054504F57451B
:1038200052444F574E0900494F494E09090047532A
:1038300054415409090049484F4C445F4952554E80
:10384000090047434F4E460909000900092042611B
:103850006420726573706F6E736521000920426188
:103860006420726573706F6E736521000920426178
:103870006420726573706F6E736521000920426168
:103880006420726573706F6E73652100303D2E3356
:10389000323500313D2E31380066616C736500743D
:1038A0007275650066616C73650074727565006D94
:1038B0006178002F3331002F3331002F3331006610
:1038C000616C7365007472756500303D2E3332355E
:1038D00000313D2E31380066616C7365007472757D
:1038E000650066616C73650074727565006D617862
:1038F000002F3331002F3331002F33310066616CDC
:103900007365007472756500303D2E3332350031B9
:103910003D2E31380066616C736500747275650008
:1039200066616C73650074727565006D6178002F57
:103930003331002F3331002F33310066616C7365F2
:1039400000747275650066616C73650074727565EC
:1039500000303D2E33323500313D2E313800666166
:103960006C736500747275650066616C73650074D4
:10397000727565006D6178002F3331002F3331008F
:103980002F33310066616C73650074727565004495
:103990007269766572207265676973746572733ACD
:1039A0000A006F7409006F747077090073326761E1
:1039B00009007332676209006F6C6109006F6C6205
:1039C00009007374737409006673616374697665C2
:1039D000090073675F726573756C740900737461B5
:1039E0006C6C6775617264090044525653544154BB
:1039F0005553005374616C6C677561726420746810
:103A00007273002D73746172740900687973746540
:103A100072657369730A2D656E640900626C616E6C
:103A20006B2074696D65006F66662074696D650949
:103A3000004F54207072657761726E206861730A5E
:103A40006265656E20747269676765726564004FB0
:103A500054207072657761726E005B6D6D2F735DBF
:103A6000090070776D0A7468726573686F6C640919
:103A700000747374657009006D7374657073090068
:103A8000737465616C746843686F70007673656EFB
:103A90007365090050574D207363616C6500435393
:103AA0002061637475616C0900486F6C64206375F4
:103AB0007272656E740052756E2063757272656EF7
:103AC00074004D41582063757272656E7400524DDA
:103AD000532063757272656E74005365742063754C
:103AE0007272656E7400456E61626C6564090009EE
:103AF00000617869733A70776D5F7363616C652FED
:103B000063757272656E745F7363616C652F6D654A
:103B100063685F6C6F61647C666C6167737C7761FE
:103B2000726E636F756E740A006D41290A0020641D
:103B30007269766572206F76657274656D706572F4
:103B40006174757265207761726E696E67212028D5
:103B5000003A20002063757272656E74206465639C
:103B600072656173656420746F20006D41290A00DD
:103B700020647269766572206F76657274656D7007
:103B800065726174757265207761726E696E672106
:103B90002028003A20002063757272656E742064DC
:103BA000656372656173656420746F20006D4129DF
:103BB0000A0020647269766572206F76657274659A
:103BC0006D7065726174757265207761726E696E71
:103BD00067212028003A20002063757272656E7498
:103BE0002064656372656173656420746F200025CD
:103BF000756420253032753A25303275006D4129C3
:103C00000A0020647269766572206F766572746549
:103C10006D7065726174757265207761726E696E20
:103C200067212028003A20002063757272656E7447
:103C30002064656372656173656420746F2000445D
:103C40007269766572206572726F7200636F696C5B
:103C50002073686F727420636972637569740A00F7
:103C60006F76657274656D70657261747572650AE0
:103C70000020647269766572206572726F722064CA
:103C8000657465637465643A2030780063616E63BF
:103C9000656C00726573756D656400726573756D32
:103CA000650070617573656400706F7765726F662B
:103CB00066002F2F616374696F6E3A0020573A00D7
:103CC00020573A00457874727564657220436F6FAF
:103CD0006C696E672E2E2E0045787472756465725D
:103CE0002048656174696E672E2E2E00202F0020FB
:103CF00042403A0020403A00546865726D616C2081
:103D000052756E6177617900453120544845524DB6
:103D1000414C2052554E4157415900424544205490
:103D20004845524D414C2052554E41574159002073
:103D30002D20496E76616C696420657874727564B3
:103D40006572206E756D62657220210A004865619A
:103D500074696E67206661696C6564004265642001
:103D600068656174696E67206661696C65640048A6
:103D7000656174696E67206661696C6564004531D0
:103D80002048656174696E67206661696C656400CE
:103D90004D494E54454D5020747269676765726590
:103DA00064004531204572723A204D494E54454DCC
:103DB00050004572723A204D494E54454D502042B4
:103DC0004544004D415854454D5020747269676711
:103DD00065726564004531204572723A204D415844
:103DE00054454D50004572723A204D415854454D4E
:103DF0005020424544006265640A002C20737973A8
:103E000074656D2073746F707065642120486561FE
:103E10007465725F49443A200023646566696E6583
:103E20002044454641554C545F004B6420004B698B
:103E300020004B702000006265640050494420411E
:103E400075746F74756E652066696E6973686564F4
:103E5000212050757420746865206C617374204B48
:103E6000702C204B6920616E64204B6420636F6E60
:103E70007374616E74732066726F6D2062656C6F0F
:103E80007720696E746F20436F6E66696775726123
:103E900074696F6E2E680A00504944204175746F32
:103EA00074756E65206661696C6564212074696D46
:103EB000656F75740A00546865726D616C20527587
:103EC0006E6177617900453120544845524D414C2F
:103ED0002052554E415741590042454420544845CF
:103EE000524D414C2052554E415741590048656151
:103EF00074696E67206661696C65640045312048AD
:103F0000656174696E67206661696C65640042650D
:103F1000642068656174696E67206661696C6564B8
:103F200000504944204175746F74756E6520666158
:103F3000696C6564212054656D7065726174757279
:103F40006520746F6F20686967680A00204B643AC7
:103F50002000204B693A2000204B703A20000A20B4
:103F6000436C617373696320504944200A002054F4
:103F7000753A2000204B753A2000206D61783A2078
:103F800000206D696E3A200020643A2000206269AA
:103F900061733A2000504944204175746F74756E06
:103FA000652073746172740A00504944204175742D
:103FB0006F74756E65206661696C65642120546557
:103FC0006D706572617475726520746F6F206869B9
:103FD00067680A001000AD0330016A0150022B012E
:103FE00070030A019004F500B005E500D006D80082
:103FF000F007CE001009C500300ABE00500BB70014
:10400000700CB100900DAB00B00EA600D00FA20056
:10401000F0109D001012990030139500501492007A
:1040200070158E0090168B00B0178700D018840092
:10403000F0198100101B7E00301C7B00501D7900A0
:10404000701E7600901F7300B0207000D0216E00AB
:10405000F0226B00102469003025660050266300B2
:104060007027610090285E00B0295C00D02A5900BA
:10407000F02B5600102D5400302E5100502F4E00C2
:1040800070304B0090314800B0324500D0334200D0
:10409000F0343E0010363B003037370050383300E4
:1040A00070392E00903A2900B03B2300D03C1B0011
:1040B000F03D1100103F0100F03F00001000C90268
:1040C00010012C014001220170011801B0010E0104
:1040D000F00104015002FA00B002F0003003E600E3
:1040E000D003DC009004D2007005C800A006BE001A
:1040F0000008B400B009AA00D00BA000600E960022
:1041000060118C000015820020197800C01D6E001F
:10411000A0226400B0275A00902C500000314600C5
:10412000E0343C0010383200903A2800603C1E0019
:10413000A03D1400803E0A00203F00006F70656EB5
:1041400000545249474745524544003A20007A5F9F
:104150006D6178007A5F6D696E00795F6D617800DE
:10416000785F6D696E005265706F7274696E67205A
:10417000656E6473746F70207374617475730A0074
:10418000456E6473746F707320256320256320254A
:104190006320256300205A3A0020593A0020583AFB
:1041A00000656E6473746F7073206869743A2000E0
:1041B000486F6D696E67206661696C656400466969
:1041C0006C616D656E7420757365643A200053747C
:1041D0006174733A20002C204C6F6E6765737420F5
:1041E0006A6F623A2000546F74616C2074696D6567
:1041F0003A200053746174733A20002C20466169A0
:104200006C65643A20002C2046696E6973686564A9
:104210003A20005072696E74733A200053746174CE
:10422000733A2000496E76616C6964206578747217
:10423000756465720A00205A3A0020593A002043FA
:104240006F756E7420583A00C23100001C260000C1
:10425000F4190000D80F0000EB080000C0040000B3
:10426000750200004001000024F4D43050C38E20B9
:10427000C2A24017828B7011127A910D816CD90AFB
:10428000A861E108C7586607615143061E4B5D05EA
:10429000C145A7041A411104093D9803713931033E
:1042A0004036DB0265339102D4305402802E1D0269
:1042B000632CEE01752AC501B028A00110278101E9
:1042C0008F2564012B244B01E0223401AC211F0116
:1042D0008D200D01801FFC00841EED00971DDF0066
:1042E000B81CD200E61BC600201BBC00641AB2003A
:1042F000B219A8000A19A0006A189900D1179100F4
:1043000040178B00B516840031167E00B315790076
:104310003A157300C7146F0058146A00EE13660054
:104320008813630025135E00C7125B006C125700F0
:1043300015125400C111510070114F0021114B0092
:10434000D61049008D10470046104400021042006C
:10435000C00F4000800F3E00420F3C00060F3B00A4
:10436000CB0E3800930E37005C0E3500270E34005C
:10437000F30D3200C10D3100900D3000600D2E00A4
:10438000320D2D00050D2C00D90C2B00AE0C290090
:10439000850C29005C0C2700350C27000E0C26002C
:1043A000E80B2400C40B2400A00B23007D0B23008A
:1043B0005A0B2100390B2100180B2000F80A1F00AE
:1043C000D90A1E00BB0A1E009D0A1D00800A1D009E
:1043D000630A1C00470A1B002C0A1B00110A1A0062
:1043E000F7091A00DD091900C4091900AB09190001
:1043F000920917007B091800630917004C09160081
:1044000036091600200916000A091500F5081500DE
:10441000E0081400CC081400B8081400A408140024
:10442000900813007D0812006B0813005808120052
:104430004608120034081100230811001208110068
:1044400001081100F0071000E0071000D00710006D
:10445000C0071000B0070F00A107100091070E0061
:1044600083070F0074070F0065070E0057070E0043
:1044700049070E003B070D002E070E0020070D0018
:1044800013070D0006070D00F9060C00ED060D00E0
:10449000E0060C00D4060C00C8060C00BC060C009C
:1044A000B0060C00A4060B0099060C008D060B004C
:1044B00082060B0077060B006C060B0061060A00F3
:1044C00057060B004C060A0042060A0038060A008E
:1044D0002E060A0024060A001A060A001006090021
:1044E00007060A00FD050900F4050900EB050900AF
:1044F000E2050900D9050900D0050900C705090032
:10450000BE050900B5050800AD050800A5050900B0
:104510009C050800940508008C0508008405080027
:104520007C050800740508006C0507006505080097
:104530005D050700560508004E0507004705070002
:104540004005080038050700310507002A05070067
:10455000230507001C050600160507000F050700C8
:104560000805060002050700FB040600F504070025
:10457000EE040600E8040600E2040700DB0406007F
:10458000D5040600CF040600C9040600C3040600D3
:10459000BD040600B7040600B1040500AC04060023
:1045A000A6040600A00405009B040600950405006F
:1045B000900406008A0405008504050080040600B6
:1045C0007A04050075040500700405006B040500FD
:1045D00066040500610405005C040500570405003D
:1045E000520405004D04050048040500430405007D
:1045F0003E0404003A0405003504050030040400BC
:104600002C04050027040400230405001E040400F4
:104610001A04040016040500110404000D0404002B
:10462000090405000404040000040400FC03040061
:10463000F8030400F4030400F0030400EC03040096
:10464000E8030400E4030400E0030400DC030400C6
:10465000D8030400D4030400D0030400CC030400F6
:10466000C8030300C503030024F404D9201BC40CB1
:104670005C0E9804C4095F0265077101F405F90036
:10468000FB04B30048048700C103690058035500C8
:1046900003034500BE023A008402310053022A009F
:1046A0002902250004022000E4011C00C8011900B1
:1046B000AF0117009801140084011300710110006C
:1046C0006101100051010E0043010D0036010B0085
:1046D0002B010B0020010B00150109000C01090042
:1046E00003010800FB000800F3000800EB000700CE
:1046F000E4000600DE000600D8000600D200060036
:10470000CC000500C7000500C2000500BD00040084
:10471000B9000400B5000400B1000400AD000400BD
:10472000A9000400A5000300A20003009F000400EC
:104730009B00030098000300950002009300030013
:10474000900003008D0002008B000300880002002F
:104750008600020084000300810002007F00020046
:104760007D0002007B00020079000200770001005A
:104770007600020074000200720001007100020065
:104780006F0002006D0001006C0002006A00010071
:104790006900020067000100660001006500010079
:1047A000640002006200010061000100600001007D
:1047B0005F0002005D0001005C0001005B00010081
:1047C0005A00010059000100580001005700010083
:1047D0005600010055000100540001005300000084
:1047E000530001005200010051000100500001007F
:1047F0004F0001004E0000004E0001004D0001007E
:104800004C0001004B0000004B0001004A00010079
:104810004900010048000000480001004700010075
:104820004600000046000100450000004500010070
:10483000440001004300000043000100420000006A
:104840004200010041000000410001004000010061
:104850003F0000003F0001003E0000003E0001005C
:104860003D0000003D0001003C0000003C00000055
:104870003C0001003B0000003B0001003A0000004A
:104880003A00010039000000390001003800000042
:104890003800000038000100370000003700010038
:1048A0003600000036000000360001003500000030
:1048B0003500000035000100340000003400000025
:1048C0003400010033000000330000003300010019
:1048D0003200000032000000320001003100000010
:1048E0003100000031000100300000003000000005
:1048F000300001002F0000002F0000002F000000FA
:104900002F0001002E0000002E0000002E000100EC
:104910002D0000002D0000002D0000002D000100E2
:104920002C0000002C0000002C0000002C000100D6
:104930002B0000002B0000002B0000002B000100CA
:104940002A0000002A0000002A0000002A000100BE
:1049500029000000290000002900000029000000B3
:1049600029000100280000002800000028000000A5
:104970002800000028000100270000002700000098
:10498000270000002700000027000100260000008B
:10499000260000002600000026000000260001007E
:1049A0002500000025000000250000002500000073
:1049B0002500000025000100240000002400000064
:1049C0002400000024000000240001002300000057
:1049D000230000002300000023000000230000004B
:1049E000230000002300010022000000220000003C
:1049F000220000002200000022000000220001002E
:104A00002100000021000000210000002100000022
:104A10002100000021000000210001002000000012
:104A20002000000020000000200000002000000006
:104A30002000000020000000200001001F000000F6
:104A40001F0000001F0000001F0000001F000000EA
:104A50001F0000001F0001001E0000001E000000DB
:104A60001E0000001E0000003A0A0020286D6D297B
:104A7000002055004C0046696C616D656E74206CB9
:104A80006F61642F756E6C6F6164206C656E677406
:104A900068733A0A0020204D393030204B004C69B1
:104AA0006E65617220416476616E63653A0A0054F6
:104AB00030204500205A00205900205800447269D7
:104AC000766572207374657070696E67206D6F64AF
:104AD000653A0A00205900205800544D43323133C2
:104AE00030205374616C6C47756172642074687215
:104AF0006573686F6C643A0A0020543020450020CA
:104B00005A00205900205800487962726964205484
:104B100068726573686F6C643A0A002054302045EF
:104B200000205A00205900205800537465707065A9
:104B300072206472697665722063757272656E7434
:104B40003A0A0020204D383531205A005A2D507233
:104B50006F6265204F6666736574002044002049CB
:104B60000020204D333034205000204400204900E4
:104B700020204D333031205000504944207365745B
:104B800074696E67733A0A0020460020420020488C
:104B90000020204D3134352053004D617465726919
:104BA000616C2068656174757020706172616D65FB
:104BB000746572733A0A0020204D3432302053005D
:104BC0004175746F20426564204C6576656C696E32
:104BD000673A0A00204500205A002059002058005A
:104BE00020540020530020204D3230352042002038
:104BF000453C6D61785F655F6A65726B3E00205869
:104C00003C6D61785F785F6A65726B3E20593C6DE0
:104C100061785F795F6A65726B3E205A3C6D61789E
:104C20005F7A5F6A65726B3E00416476616E6365B0
:104C3000643A20423C6D696E5F7365676D656E74A2
:104C40005F74696D655F75733E20533C6D696E5F7F
:104C500066656564726174653E20543C6D696E5F83
:104C600074726176656C5F66656564726174653ED9
:104C70000020540020520020204D323034205000BB
:104C8000416363656C65726174696F6E2028756E2F
:104C90006974732F7332293A20503C7072696E74B4
:104CA0005F616363656C3E20523C72657472616340
:104CB000745F616363656C3E20543C747261766519
:104CC0006C5F616363656C3E0A00204500205A00FA
:104CD00020590020204D3230312058004D61786934
:104CE0006D756D20416363656C65726174696F6E8B
:104CF0002028756E6974732F7332293A0A00204593
:104D000000205A0020590020204D32303320580016
:104D10004D6178696D756D20666565647261746555
:104D2000732028756E6974732F73293A0A005374BF
:104D30006570732070657220756E69743A0A002080
:104D4000204D3134392043203B20556E6974732047
:104D5000696E2043656C736975730A0020204732C1
:104D600031202020203B20556E69747320696E200D
:104D70006D6D0020204D363033200020204D39311C
:104D8000340020204D3931330020204D3536392074
:104D900053310020204D3930360048617264636F12
:104DA0006465642044656661756C74205365747431
:104DB000696E6773204C6F616465640A0028230084
:104DC0000028230000C8000000E80300000000964F
:104DD000430000964300009643000020420000C8B4
:104DE000420000C842000048430000D243290A00A4
:104DF0002062797465733B206372632000207374B2
:104E00006F7265642073657474696E677320726570
:104E100074726965766564202800202863616C637C
:104E2000756C6174656429210A0020213D200045CC
:104E30004550524F4D20435243206D69736D61744C
:104E40006368202D202873746F7265642920002008
:104E500053697A653A2000496E6465783A200020EB
:104E60004D61726C696E3D563634290A00284545FD
:104E700050524F4D3D00454550524F4D2076657282
:104E800073696F6E206D69736D61746368200029AA
:104E90000A002062797465733B20637263200053BB
:104EA000657474696E67732053746F72656420282B
:104EB00000454550524F4D206461746173697A65B5
:104EC000206572726F722E0A0050726F62696E678F
:104ED000206661696C65640A0050726F62696E6772
:104EE000206661696C6564005761726E696E673A2D
:104EF00020486F6D696E672042756D702044697639
:104F000069736F72203C20310A00020204486F6D01
:104F100065202573257325732066697273740020DC
:104F200066697273740A005A0059005800486F6D20
:104F300065200020746F6F206C6F6E672065787439
:104F4000727573696F6E2070726576656E746564D4
:104F50000A0020636F6C6420657874727573696FE2
:104F60006E2070726576656E7465640A0020453A3D
:104F700000205A3A0020593A00583A0000004842AE
:104F80000000484200002042FF0101000000000034
:104F900000000000000040000030430000454300D6
:104FA000003743000040C00000404300003743008A
:104FB000002D430000404300003743000040C00084
:104FC00000A0C00000000020746F6F206C6F6E673F
:104FD00020657874727573696F6E2070726576657E
:104FE0006E7465640A0020636F6C64206578747267
:104FF0007573696F6E2070726576656E7465640A8C
:1050000000627573793A2070617573656420666F0C
:105010007220696E7075740A00627573793A207037
:10502000617573656420666F7220757365720A001E
:10503000627573793A2070726F63657373696E6716
:105040000A004D3131372050726F626520737563ED
:105050006365737366756C0A0020496E76616C69CE
:10506000642065787472756465722000205A3A2055
:105070000020593A200042656420583A20005072BE
:105080006F6265205A204F66667365743A20003F50
:105090005A206F7574206F662072616E67652028D4
:1050A0002D3220746F2035290A004D3134352053BC
:1050B0003C696E6465783E206F7574206F6620725F
:1050C000616E67652028302D31290A00436C6963C1
:1050D0006B20746F20726573756D652E2E2E0055D2
:1050E0006E6B6E6F776E20636F6D6D616E643A20CC
:1050F0002200454550524F4D204F4B0A004E6F2025
:105100006D6F76652E004543484F00494E464F006F
:105110004552524F52530044525952554E00434F3C
:105120004D4D554E49434154494F4E006F66660000
:1051300006510B51105117511E5144454255473AE3
:10514000004C756C7A426F74204D696E6920322074
:105150004F46462E00205A00205900580020204D6E
:1051600061783A2000205A00205900580020204D34
:10517000696E3A2000536F667420656E6473746FB5
:1051800070733A20005072696E742074696D653ACC
:1051900020004D3131332053002F2F200043617008
:1051A0003A004D4F54494F4E5F4D4F4445530054C4
:1051B0004845524D414C5F50524F54454354494F1E
:1051C0004E004155544F5245504F52545F53445F27
:1051D0005354415455530050524F4D50545F535502
:1051E00050504F525400454D455247454E43595F2C
:1051F00050415253455200434153455F4C49474843
:10520000545F4252494748544E45535300544F4708
:10521000474C455F4C494748545300534F465457F9
:105220004152455F504F574552004255494C445FEB
:1052300050455243454E54004C4556454C494E4707
:105240005F44415441005A5F50524F42450041551E
:10525000544F4C4556454C005052494E545F4A4FAE
:10526000420050524F4752455353004155544F52FC
:1052700045504F52545F54454D5000564F4C554D7C
:10528000455452494300454550524F4D00534552F5
:1052900049414C5F584F4E5F584F46460046495271
:1052A0004D574152455F4E414D453A4D61726C69D3
:1052B0006E20204649524D574152455F5645525344
:1052C000494F4E3A322E302E302E39342045585424
:1052D00052554445525F545950453A53696E676C74
:1052E0006545787472756465724165726F563220D7
:1052F000534F555243455F434F44455F55524C3AD7
:1053000068747470733A2F2F636F64652E616C65D7
:1053100070686F626A656374732E636F6D2F646962
:1053200066667573696F6E2F4D41524C494E205021
:10533000524F544F434F4C5F56455253494F4E3A8C
:10534000312E30204D414348494E455F5459504518
:105350003A4C756C7A426F74204D696E6920322028
:1053600045585452554445525F434F554E543A3177
:1053700020555549443A65353530323431312D6444
:105380003436642D343231642D626133612D6132E3
:10539000303132366437393330660A0020284E6F98
:1053A0007420796574206D65617375726564290078
:1053B000202041766572616765206D656173757245
:1053C0006564206261636B6C61736820286D6D2970
:1053D0003A002020536D6F6F7468696E6720286DE6
:1053E0006D293A202020202020202020202020204D
:1053F00020202020530020204261636B6C61736881
:105400002044697374616E636520286D6D293A20AC
:10541000202020202020200020202020202846316D
:105420002E30203D2066756C6C2C2046302E3020AE
:105430003D206E6F6E65290A002020436F727265F1
:105440006374696F6E20416D6F756E742F46616471
:10545000652D6F75743A202020202046006163740A
:105460006976653A0A00696E004261636B6C61732C
:105470006820636F7272656374696F6E2069732050
:1054800000205A0020506F736974696F6E616C2040
:105490004572726F723A0A004E6F7A7A6C652054C8
:1054A0006970204F757465722044696D656E73690B
:1054B0006F6E733A0A002020546F703A200020204B
:1054C00046726F6E743A200020204C6566743A2054
:1054D000004261636B6C6173683A0A00205A0043B2
:1054E000656E7465723A0A00202046726F6E743AD7
:1054F000200020204C6566743A20002020546F70F4
:105500003A200053696465733A0A00426564204C8E
:105510006576656C696E6720004661696C6564201C
:10552000746F20656E61626C6520426564204C6515
:1055300076656C696E670A00426564204C65766525
:105540006C20436F7272656374696F6E204D617475
:105550007269783A000A0A426564204C6576656C87
:1055600020436F7272656374696F6E204D6174724F
:1055700069783A00202B000A436F72726563746584
:105580006420426564204865696768742076732EDC
:105590002042656420546F706F6C6F67793A0A001F
:1055A000202B000A426564204865696768742054AE
:1055B0006F706F6772617068793A0A2020202B2D16
:1055C0002D2D204241434B202D2D2B0A2020207CC5
:1055D00020202020202020202020207C0A204C2059
:1055E0007C20202020282B29202020207C20520ACB
:1055F0002045207C20202020202020202020207CCE
:1056000020490A2046207C20282D29204E20282BA6
:1056100029207C20470A2054207C20202020202084
:1056200020202020207C20480A2020207C202020B0
:1056300020282D29202020207C20540A2020207C76
:1056400020202020202020202020207C0A20202014
:105650004F2D2D2046524F4E54202D2D2B0A202801
:10566000302C30290A003474682070726F62652013
:10567000706F696E742C2064697374616E63652049
:1056800066726F6D20706C616E653A200020284450
:10569000525952554E2900473239204175746F20B6
:1056A000426564204C6576656C696E67003F202812
:1056B0004C2C522C462C4229206F7574206F66208A
:1056C000626F756E64732E0A003F50726F626520C0
:1056D000706F696E74732028592920697320696D71
:1056E000706C61757369626C652028322D32292EC9
:1056F0000A003F50726F626520706F696E7473208C
:1057000028582920697320696D706C61757369620E
:105710006C652028322D32292E0A003F2856296533
:1057200072626F7365206C6576656C2069732069A1
:105730006D706C61757369626C652028302D342939
:105740002E0A0043757272656E742066696C653A44
:105750002000456E642066696C65206C6973740A6C
:1057600000426567696E2066696C65206C697374B8
:105770000A00416476616E6365204B3D003F4B201B
:1057800076616C7565206F7574206F662072616E2E
:1057900067652028302D3130292E0A004D313137F0
:1057A00020486F7420456E642048656174696E6797
:1057B0002E2E2E0A4D3130342053313730205430C4
:1057C0000A473238204F310A473120593235205AA2
:1057D00031302046353030300A4D313039205231A9
:1057E00037302054300A4D31313720526577697097
:1057F000696E67206E6F7A7A6C650A54300A473199
:105800002058343520593137342046353030300A6D
:105810004731205A310A4D31303920523137300A60
:105820004731205834352059313734204634303010
:10583000300A473120583435205931373420463426
:105840003030300A47312058343520593137342030
:1058500046343030300A47312058343520593137FA
:10586000342046343030300A4731205834352059FE
:105870003137342046343030300A473120583435FF
:1058800020593137342046343030300A47312058DF
:10589000343520593137342046343030300A4731DE
:1058A0002058343520593137342046343030300ACE
:1058B0004731205834352059313734204634303080
:1058C000300A473120583435205931373420463496
:1058D0003030300A473120583435205931373420A0
:1058E00046343030300A473120583435205931376A
:1058F000342046343030300A4731205A31350A4D91
:105900003130362053323535200A47302058302088
:1059100059300A4D31303920523136302054300A56
:105920004D3130370A007370726561644379636C7E
:105930006500737465616C746843686F70002064FF
:105940007269766572206D6F64653A0900737072D2
:105950006561644379636C6500737465616C746838
:1059600043686F700020647269766572206D6F64A1
:10597000653A09007370726561644379636C650010
:10598000737465616C746843686F70002064726939
:10599000766572206D6F64653A0900737072656197
:1059A000644379636C6500737465616C7468436803
:1059B0006F700020647269766572206D6F64653A5D
:1059C000090020686F6D696E672073656E73697476
:1059D00069766974793A200020686F6D696E672076
:1059E00073656E73697469766974793A20002073FF
:1059F0007465616C746843686F70206D61782073A2
:105A0000706565643A200020737465616C74684346
:105A1000686F70206D61782073706565643A20004E
:105A200020737465616C746843686F70206D617871
:105A30002073706565643A200020737465616C742E
:105A40006843686F70206D61782073706565643A93
:105A50002000207072657761726E20666C6167202D
:105A6000636C65617265640A0020707265776172AB
:105A70006E20666C616720636C65617265640A0004
:105A8000207072657761726E20666C616720636C4E
:105A900065617265640A00207072657761726E20BC
:105AA000666C616720636C65617265640A0066619B
:105AB0006C73650074727565002074656D70657235
:105AC0006174757265207072657761726E20747290
:105AD000696767657265643A200066616C7365008A
:105AE00074727565002074656D706572617475728D
:105AF00065207072657761726E2074726967676580
:105B00007265643A200066616C7365007472756535
:105B1000002074656D7065726174757265207072B5
:105B2000657761726E207472696767657265643A41
:105B3000200066616C736500747275650020746581
:105B40006D706572617475726520707265776172CF
:105B50006E207472696767657265643A200020641C
:105B600072697665722063757272656E743A200090
:105B7000206472697665722063757272656E743A1C
:105B80002000206472697665722063757272656E9A
:105B9000743A2000206472697665722063757272AF
:105BA000656E743A20004D6163726F20746F6F20D0
:105BB0006C6F6E672E0A0020466C6F773A200020CB
:105BC000643A0020693A0020703A00204500205ACB
:105BD00000205900204D393220580043290A006125
:105BE000626C656420286D696E2074656D7020009C
:105BF00064697300656E00436F6C6420657874722D
:105C00007564657320617265200020540020520085
:105C1000416363656C65726174696F6E3A20500010
:105C2000496E76616C69642065787472756465721A
:105C30000A0020643A0020693A0020703A00536C50
:105C40006565702E2E2E0047322F47332062616427
:105C500020706172616D65746572730A0050726FB5
:105C60006265205A204F66667365743A2000446F5F
:105C70006E6520736176696E672066696C652E0AB1
:105C80000053442072656164206572726F720A006D
:105C9000446F6E65207072696E74696E6720666904
:105CA0006C650A0053544F505045442E20005072EA
:105CB000696E7465722073746F70706564206475AA
:105CC0006520746F206572726F72732E204669783A
:105CD00020746865206572726F7220616E64207531
:105CE0007365204D39393920746F20726573746182
:105CF00072742E202854656D7065726174757265BA
:105D00002069732072657365742E20536574206951
:105D1000742061667465722072657374617274694F
:105D20006E67290A004E6F20436865636B73756D5B
:105D30002077697468206C696E65206E756D626588
:105D4000722C204C617374204C696E653A20004EB1
:105D50006F20436865636B73756D20776974682085
:105D60006C696E65206E756D6265722C204C617376
:105D700074204C696E653A2000636865636B7375C7
:105D80006D206D69736D617463682C204C61737450
:105D9000204C696E653A20004C696E65204E756D29
:105DA000626572206973206E6F74204C6173742079
:105DB0004C696E65204E756D6265722B312C204CDE
:105DC000617374204C696E653A20004D31313000AA
:105DD000526573656E643A20002042002050006FC7
:105DE0006B00656E7175657565696E672022005080
:105DF0004944204175746F74756E65206661696CE5
:105E000065642120426164206578747275646572EE
:105E1000206E756D6265720A0042656420636F6F63
:105E20006C696E672E2E2E00426564206865617471
:105E3000696E672E2E2E006F6B0030780047323867
:105E4000205A0A47302058383020593139302046FE
:105E5000333030300A4D313137205072696E742042
:105E600061626F727465642E002020506C616E6EEA
:105E7000657242756666657242797465733A200090
:105E80002046726565204D656D6F72793A2000433A
:105E90006F6D70696C65643A204665622032362009
:105EA000323031390A00207C20417574686F723AB3
:105EB0002028416C657068204F626A6563747320A6
:105EC000496E632E2C204C756C7A426F74204769A2
:105ED00074205265706F7369746F7279290A0000BB
:105EE000204C61737420557064617465643A2000BD
:105EF000322E302E302E39340A004D61726C696EAC
:105F00000020536F66747761726520526573657403
:105F10000A00205761746368646F67205265736577
:105F2000740A002042726F776E206F75742052657C
:105F30007365740A002045787465726E616C205236
:105F4000657365740A00506F77657255700A007347
:105F5000746172740A004B494C4C45442E20005029
:105F600072696E7465722068616C7465642E206B52
:105F7000696C6C28292063616C6C6564210A004B94
:105F8000494C4C20636175736564206279204B49EC
:105F90004C4C20627574746F6E2F70696E0A004BE2
:105FA000494C4C2063617573656420627920746F7D
:105FB0006F206D75636820696E6163746976652012
:105FC00074696D65202D2063757272656E7420632F
:105FD0006F6D6D616E643A20004D31303420533165
:105FE00037302054300A4D313137204C6576656C9E
:105FF000696E67205820417869730A4732380A472A
:106000003020583136302046393939390A47302066
:106010005A352046363030300A4739310A4D323150
:10602000312053300A4D3430300A4D393036205A41
:106030003630300A4730205A2D3135204635303041
:106040000A4730205A3520463530300A4739300A61
:106050004D3430300A4D393036205A3936300A4DF9
:106060003231312053310A4732380A4D313137202D
:106070004C6576656C696E6720646F6E652E0A47A5
:1060800031320A4D31303920523136300A4D3131FA
:10609000372050726F62696E6720626564007072AB
:1060A0006F62655F7265776970650050726F6269D3
:1060B0006E67206661696C6564004D31313720423E
:1060C0006564206C6576656C696E67206661696CD5
:1060D00065642E0A4730205A31300A473020453057
:1060E0000A4D3330302050323520533838300A4D85
:1060F000333030205035302053300A4D333030208B
:1061000050323520533838300A4D33303020503536
:10611000302053300A4D3330302050323520533840
:1061200038300A47342053310070726F62655F6601
:1061300061696C65640050726F7465637465642096
:1061400050696E0A0025311D402924301C45272343
:106150002F1B0A0743222B1A42043803FF36040878
:106160000606000159506084188EFDA406DAAD01C0
:10617000AB01A901A701388E11241FBECFEFD1E2D8
:10618000DEBFCDBF00E00CBF14E0A0E0B2E0EEE463
:10619000F5EE02E00BBF02C007900D92A837B107E1
:1061A000D9F728E1A8E7B4E001C01D92A43AB207EC
:1061B000E1F710E3CBEBD0E300E006C02197010943
:1061C000802FFE010F94B76AC23BD10780E0080719
:1061D000A9F70E941C440D9496720C9400001F9223
:1061E0000F920FB60F9211242F933F938F939F938B
:1061F000AF93BF938091790490917A04A0917B042E
:10620000B0917C043091780423E0230F2D3720F4E3
:106210000196A11DB11D05C026E8230F0296A11D00
:10622000B11D209378048093790490937A04A0930D
:106230007B04B0937C0480917D0490917E04A091B6
:106240007F04B09180040196A11DB11D80937D044F
:1062500090937E04A0937F04B0938004BF91AF918C
:106260009F918F913F912F910F900FBE0F901F9094
:1062700018952FB7F8946091790470917A04809101
:106280007B0490917C042FBF08953FB7F8948091D0
:106290007D0490917E04A0917F04B091800426B586
:1062A000A89B05C02F3F19F00196A11DB11D3FBF4E
:1062B000BA2FA92F982F8827820F911DA11DB11DDC
:1062C000BC01CD0142E0660F771F881F991F4A95D8
:1062D000D1F708958F929F92AF92BF92CF92DF92A3
:1062E000EF92FF926B017C01D0DF4B015C01C11486
:1062F000D104E104F104F1F091D3C7DFDC01CB015B
:1063000088199909AA09BB09883E9340A105B105DE
:1063100070F321E0C21AD108E108F10888EE880E76
:1063200083E0981EA11CB11CC114D104E104F10446
:1063300021F7DDCFFF90EF90DF90CF90BF90AF902F
:106340009F908F900895789484B5826084BD84B5C1
:10635000816084BD85B5826085BD85B5816085BD60
:10636000EEE6F0E0808181608083E1E8F0E0108279
:10637000808182608083808181608083E0E8F0E0BA
:10638000808181608083E1EBF0E0808184608083A4
:10639000E0EBF0E0808181608083E1E9F0E08081E2
:1063A00082608083808181608083E0E9F0E0808189
:1063B00081608083E1EAF0E0808182608083808177
:1063C00081608083E0EAF0E0808181608083E1E2A7
:1063D000F1E0808182608083808181608083E0E25F
:1063E000F1E0808181608083EAE7F0E08081846071
:1063F00080838081826080838081816080838081CE
:10640000806880831092C10008951F93CF93DF931B
:10641000182FEB0161E016D1209711F460E004C061
:10642000CF3FD10531F461E0812FDF91CF911F91F2
:1064300045C1E12FF0E0E756FC4FE4914E2F50E0CC
:10644000FA013197E231F10508F09DC08827EE5836
:10645000FF4F8F4F0D94B76A84B5806884BDC7BD68
:1064600097C084B5806284BDC8BD92C08091800011
:10647000806880938000D0938900C093880088C092
:1064800080918000806280938000D0938B00C093C5
:106490008A007EC080918000886080938000D093C5
:1064A0008D00C0938C0074C08091B0008068809390
:1064B000B000C093B3006CC08091B0008062809344
:1064C000B000C093B40064C0809190008068809355
:1064D0009000D0939900C09398005AC0809190008A
:1064E000806280939000D0939B00C0939A0050C02C
:1064F00080919000886080939000D0939D00C0931D
:106500009C0046C08091A00080688093A00080918C
:10651000A0008F7B8093A000D093A900C093A80017
:1065200037C08091A00080628093A000D093AB0020
:10653000C093AA002DC08091A00088608093A00025
:10654000D093AD00C093AC0023C08091200180683F
:1065500080932001D0932901C093280119C0809114
:106560002001806280932001D0932B01C0932A01E7
:106570000FC080912001886080932001D0932D016D
:10658000C0932C0105C0C038D1050CF04CCF46CFCC
:10659000DF91CF911F91089590E0FC013197E23196
:1065A000F10508F04EC08827EC57FF4F8F4F0D9430
:1065B000B76A809180008F7703C0809180008F7DC3
:1065C00080938000089580918000877FF9CF84B503
:1065D0008F7702C084B58F7D84BD08958091B0000F
:1065E0008F7703C08091B0008F7D8093B0000895B5
:1065F000809190008F7707C0809190008F7D03C0BD
:1066000080919000877F8093900008958091A000F2
:106610008F7707C08091A0008F7D03C08091A0007C
:10662000877F8093A0000895809120018F7707C015
:10663000809120018F7D03C080912001877F80930E
:1066400020010895CF93DF9390E0FC01E152FC4FCD
:106650002491FC01EB5DFB4F8491882361F190E074
:10666000880F991FFC01E156FB4FC591D491FC01A5
:10667000EB57FB4FA591B491611109C09FB7F894F6
:106680008881209582238883EC912E230BC0623071
:1066900061F49FB7F8943881822F80958323888393
:1066A000EC912E2B2C939FBF06C08FB7F894E881F6
:1066B0002E2B28838FBFDF91CF9108951F93CF9307
:1066C000DF93282F30E0F901E756FC4F8491F90160
:1066D000E152FC4FD491F901EB5DFB4FC491CC2307
:1066E000C1F0162F811158DFEC2FF0E0EE0FFF1FE5
:1066F000EB57FB4FA591B4918FB7F894111105C0DA
:106700009C91ED2FE095E92302C0EC91ED2BEC93E9
:106710008FBFDF91CF911F910895CF93DF93282FE3
:1067200030E0F901E756FC4F8491F901E152FC4F4A
:10673000D491F901EB5DFB4FC491CC2389F0811119
:106740002BDFEC2FF0E0EE0FFF1FE559FB4FA5917B
:10675000B491EC91ED2381E090E021F480E002C05F
:1067600080E090E0DF91CF91089508951F920F92FD
:106770000FB60F9211240BB60F922F933F934F93A6
:106780005F936F937F938F939F93AF93BF93EF9399
:10679000FF93E0910402F09105021995FF91EF91AA
:1067A000BF91AF919F918F917F916F915F914F9129
:1067B0003F912F910F900BBE0F900FBE0F901F9027
:1067C00018951F920F920FB60F9211240BB60F92CD
:1067D0002F933F934F935F936F937F938F939F93E9
:1067E000AF93BF93EF93FF93E0910602F0910702FE
:1067F0001995FF91EF91BF91AF919F918F917F91EB
:106800006F915F914F913F912F910F900BBE0F9021
:106810000FBE0F901F9018951F920F920FB60F92F8
:1068200011240BB60F922F933F934F935F936F9367
:106830007F938F939F93AF93BF93EF93FF93E091D9
:106840000802F09109021995FF91EF91BF91AF9164
:106850009F918F917F916F915F914F913F912F9178
:106860000F900BBE0F900FBE0F901F9018951F92A8
:106870000F920FB60F9211240BB60F922F933F93E6
:106880004F935F936F937F938F939F93AF93BF9338
:10689000EF93FF93E0910A02F0910B021995FF919B
:1068A000EF91BF91AF919F918F917F916F915F9188
:1068B0004F913F912F910F900BBE0F900FBE0F90F5
:1068C0001F9018951F920F920FB60F9211240BB6BE
:1068D0000F922F933F934F935F936F937F938F9379
:1068E0009F93AF93BF93EF93FF93E0910002F091DA
:1068F00001021995FF91EF91BF91AF919F918F91F7
:106900007F916F915F914F913F912F910F900BBEAF
:106910000F900FBE0F901F9018951F920F920FB6F9
:106920000F9211240BB60F922F933F934F935F93C7
:106930006F937F938F939F93AF93BF93EF93FF9347
:10694000E0910202F09103021995FF91EF91BF913E
:10695000AF919F918F917F916F915F914F913F91F7
:106960002F910F900BBE0F900FBE0F901F90189598
:106970001F920F920FB60F9211240BB60F922F9306
:106980003F934F935F936F937F938F939F93AF93B7
:10699000BF93EF93FF93E0910C02F0910D021995D4
:1069A000FF91EF91BF91AF919F918F917F916F91E7
:1069B0005F914F913F912F910F900BBE0F900FBEA3
:1069C0000F901F9018951F920F920FB60F921124DF
:1069D0000BB60F922F933F934F935F936F937F93D9
:1069E0008F939F93AF93BF93EF93FF93E0910E022A
:1069F000F0910F021995FF91EF91BF91AF919F9187
:106A00008F917F916F915F914F913F912F910F9057
:106A10000BBE0F900FBE0F901F90189508951F93F7
:106A2000CF93DF93EC011D821C821F821E82198688
:106A300081E0888782E28A871F861E86FE01B396E0
:106A4000CE01C1962FEF2193E817F907E1F711E086
:106A500018A3CE0165D51F8B188E198E80E48A8FFE
:106A60001B8E81E698E39AAB89ABDF91CF911F91A2
:106A70000895DB01ED91FC911994EF92FF921F9321
:106A8000CF93DF931F921F92CDB7DEB77C01DC015D
:106A9000D196ED91FC91D29782E069837A83199522
:106AA00020E030E04AE069817A81C701E2DF182FF7
:106AB000D701D196ED91FC91D29783E01995D7013A
:106AC000D196ED91FC91D29780E01995812F0F908E
:106AD0000F90DF91CF911F91FF90EF9008950F934A
:106AE0001F93CF93DF93EC018B01E9A9FAA982E010
:106AF0001995E9A9FAA981E0199520E030E044E16F
:106B0000B801CE01B6DF9E012D5C3F4F47E1B801D1
:106B1000CE01AFDFE9A9FAA980E0DF91CF911F9103
:106B20000F911994EF92FF921F93CF93DF93EC0193
:106B30007B01E9A9FAA982E01995E9A9FAA981E0FE
:106B4000199520E030E045E1B701CE0192DF182F22
:106B5000882339F09E012D5C3F4F47E1B701CE01FC
:106B600088DFE9A9FAA980E01995812FDF91CF91FB
:106B70001F91FF90EF900895CF93DF931F92CDB7B1
:106B8000DEB79E012F5F3F4F46E473DF89810F9090
:106B9000DF91CF910895CF93DF931F92CDB7DEB7EA
:106BA0009E012F5F3F4F47E464DF89810F90DF91A3
:106BB000CF91089520E030E048E45BCFCF93DF939E
:106BC000EC016A817B81D8DF88836A817B81CE0179
:106BD000E2DF89836A817B81CE01ECDF8B879E01B6
:106BE0002D5C3F4F6A817B8147E1CE01DF91CF91E0
:106BF00040CFCF93DF93EC016A817B813EDF882316
:106C000019F0CE01DBDF81E0DF91CF9108958F9203
:106C10009F92AF92BF92CF92EF920F93CF93DF9359
:106C20001F921F92CDB7DEB74C015B012A834983C7
:106C3000F6DEF401B382A282498147A32A8120A70C
:106C400005A3E4A2C3A2C4010F900F90DF91CF91DE
:106C50000F91EF90CF90BF90AF909F908F90C9CF42
:106C6000FC01628173813BCFCF93DF93EC01EE8512
:106C7000FF85309709F019956A817B81CE01DF91FC
:106C8000CF9150CF0F93FC0182819381648F458F08
:106C9000278F068F9F01245E3F4F4BE3BC01CF013E
:106CA0000F91E7CEFC0160A30895BF92CF92DF92CF
:106CB000EF92FF920F931F93CF93DF936C01D62F28
:106CC000B42EC22F7801CC2369F0F701049120E0A3
:106CD0004B2D6D2FC601D6DFFFEFEF1AFF0AC15013
:106CE000D85FF1CFDF91CF911F910F91FF90EF907F
:106CF000DF90CF90BF9008958F929F92AF92BF92F6
:106D0000CF92DF92EF92FF920F931F93CF93DF9377
:106D10005C01C62EC42FD22ED02F220F220F220F9D
:106D20001ED0882379F0DC0F8D2C912CCD1751F0DB
:106D300087012D2D4C2F6C2DC501B7DFE80CF91CF8
:106D4000CF5FF4CFDF91CF911F910F91FF90EF9024
:106D5000DF90CF90BF90AF909F908F9008950F934A
:106D6000FC010150040F84A996A9941718F0081784
:106D700028F402C0081750F0041740F42150260FE1
:106D800083A995A9961720F4281720F480E007C05E
:106D9000281720F481E0261710F0F8CF81E00F913A
:106DA000089581E008952EE93FE0009729F0F90168
:106DB0003197F1F70197F9CF0895FC011282808194
:106DC0008150838314820895FC0180819281980F01
:106DD00092832181921760F494819F5F94839381C1
:106DE000890F821710F08FEF820F838381E008955F
:106DF00080E00895FC0191E08381861708F490E01B
:106E000031E0461708F030E0832F892B21E05281D2
:106E1000451708F420E02823832F8923822B089527
:106E2000DC01FB01108212968C91129781831596DA
:106E30008C9115978150828313968C91838308954A
:106E4000FB0141812381213029F0233031F468EFA7
:106E5000640F04C0642F485F01C0642FCBCFDC01F6
:106E600015962C9115971696ED91FC911797CF01D9
:106E7000820F911D820F911D1192E817F907E1F71A
:106E80000895FC01A681B7818281481B8581483025
:106E900018F0A80FB11D4770382F369536953695E6
:106EA000562F577080E890E002C0959587955A95C7
:106EB000E2F7439F402D1124669566956695E62F6F
:106EC000F0E0E40FF11DEA0FFB1F3081222311F0E7
:106ED000832B02C08095832380830895FB01418129
:106EE000DC0112962C911297421760F013962C91A8
:106EF0001397241738F0608115962C91621710F4BF
:106F00002481BFCF0895CF92DF92FF920F931F93FA
:106F1000CF93DF936C01EB01FA809B81913051F0AC
:106F200030F0923049F0933051F41FEF09C010E077
:106F300001E007C011E004C010E00FEF02C010E054
:106F400000E0F7FE03C0BE01C601C8DF9881900FC4
:106F500098839981910F9983FF0C99F7DF91CF91D5
:106F60001F910F91FF90DF90CF9008950F931F9383
:106F7000CF93DF938901FB01C281D3814233D9F0E2
:106F800058F44531E1F0473109F1443141F5CE0182
:106F900066DFCE0112DF23C04634E1F04734E1F072
:106FA0004B33E9F4B901CE014BDF8823C1F0B801BE
:106FB000CE01A9DF14C0B901CE0190DF10C0CE010F
:106FC00003DF882369F0CE014ADF09C0B901CE0191
:106FD00027DF05C08D8101C08981F801808381E0B0
:106FE000DF91CF911F910F910895CF92DF92EF9291
:106FF000FF920F931F93CF93DF937C01D62FD42E54
:10700000C22F122FC62EC20E6C2D611B183038F005
:107010000FEF20E04D2DC70135DE1850F5CF6C2F56
:10702000687F6D0F2C2F277071F097E029272F5F55
:1070300027700FEF10E001C0000F2A95EAF720E05B
:107040004D2DC7011FDEDF91CF911F910F91FF9052
:10705000EF90DF90CF900895EF92FF920F931F93E0
:10706000CF93DF937C01D62F122FC42F040F212F33
:107070004C2F6D2FC701B9DFCF5F0C13F8CFDF9115
:10708000CF911F910F91FF90EF900895DF92EF92B3
:10709000FF920F931F93CF93DF93EC01162FF42EE3
:1070A000E22E5DDE882329F02E2D4F2D612FCE019B
:1070B000D3DFDF91CF911F910F91FF90EF90DF9081
:1070C00008950895FC01E60FF11D849190E0982F3A
:1070D00088273196E4918E0F911D0895FC018491CB
:1070E0000895FCDF882321F0823011F083E00895B9
:1070F00086E0089580E00895FC018081089566E0AF
:10710000E1CF68E0DFCF0A96FC01849108950B96E9
:10711000FC0184910895DC011496ED91FC91159782
:10712000319684910895BF92CF92DF92EF92FF92B1
:107130000F931F93CF93DF938C01E62EDC011496FF
:10714000CD91DC911597CE01C9DFF82EF80184812D
:107150009581C7DFC82EF1E0FF1203C02FE0B22EE9
:1071600002C0BB24BA94D80114968D919C911597B6
:10717000CADFF82EF80184819581C9DFD82ED801A5
:1071800014968D919C911597BCDFB0E6BE1538F42E
:10719000009729F0C80FD91F91E6F92E0FC0F8010A
:1071A00084819581ACDFF0E4FE1538F4009729F076
:1071B000C80FD91F81E4F82E01C06196DE1490F447
:1071C000D80150961C92509753961C925397549600
:1071D0001C92549751961C92519752961C9280E0A3
:1071E00090E066C0DF1460F38C2D90E0FE012491E6
:1071F0002F3F11F4219657C0FE104CC0D8011496B1
:107200008D919C9115976ADF9E012F5F3F4FFE0184
:10721000882311F08230E1F48491D80153968C9345
:107220005397F901249154962C935497FE01339669
:10723000E4915096EC935097FE013496E491519668
:10724000EC935197FE013596E4915296EC9320C051
:107250008491982F9F709250D80152969C93529788
:1072600082958F7051968C935197F9012491822FBA
:107270008F7054968C93549722952F7053962C931D
:107280005397FE013296E491E295EF705096EC939D
:10729000CE010EC0FE013296E491EB219C012E0F2F
:1072A000311DC20FD31FFD1409F48ACFF3949ECF72
:1072B000DF91CF911F910F91FF90EF90DF90CF90D2
:1072C000BF9008954F925F926F927F929F92AF927C
:1072D000BF92CF92DF92EF92FF920F931F93CF93C3
:1072E000DF931F92CDB7DEB72C01C62E942E622FEE
:1072F0001ADF7C01892B09F43AC0F201848195815F
:10730000F0DEB82EF201138904898189C80E8289C2
:10731000981AD92CD01A212F4D2D6C2DC2011FDDAA
:10732000882311F1EB0CF11C195F16951695169533
:10733000612E712CD914C1F03C2D57018A2D8E1964
:10734000811770F4F501049120E04D2D632FC201E7
:10735000398398DCFFEFAF1ABF0A3981385FEECF6F
:10736000E60CF71CD394E6CFF201808901C080E0DF
:107370000F90DF91CF911F910F91FF90EF90DF90D1
:10738000CF90BF90AF909F907F906F905F904F9005
:1073900008950F931F93CF93DF9300D0CDB7DEB73F
:1073A0008C01DC015596ED91FC9156972B834A8315
:1073B000698319954A81480F2B816981C8010F9013
:1073C0000F900F90DF91CF911F910F917BCFAF92D4
:1073D000BF92DF92EF92FF920F931F93CF93DF93B1
:1073E0001F921F92CDB7DEB77C01D62E042FDC0191
:1073F0005596ED91FC91569729833A831995080F7C
:107400002981A22E3A81B32E10E0F50121915F016E
:10741000222339F0402F6D2DC70154DFD80E180FED
:10742000F4CF812F0F900F90DF91CF911F910F918B
:10743000FF90EF90DF90BF90AF900895DF92EF92B2
:10744000FF920F931F93CF93DF937C01D62FD42EFF
:107450008901DC015596ED91FC9156971995D80E4E
:10746000C0E0F8012491222349F04D2D6D2FC70172
:1074700029DFD80FC80F0F5F1F4FF3CF8C2FDF917D
:10748000CF911F910F91FF90EF90DF900895DC0155
:1074900014962D913C9115972115310509F43FC0A3
:1074A00057968C915797F901811108C03596E49150
:1074B0005896EC935897F9013C9611C0813041F4ED
:1074C0003F96E4915896EC935897F901709607C04F
:1074D0003D96E4915896EC935897F9013E96E491C5
:1074E0005996EC93599758968C915897082E000C02
:1074F000990B59962C915997821B910927FD9395C9
:107500005A962C915A97203441F0829FC001112441
:1075100026E0969587952A95E1F75B968C930895DA
:107520002AE738E3FC01368B258B0895CF92DF9252
:10753000EF92FF920F931F93CF93DF938C017B0108
:107540006A01CB01FA011995D82F882311F1682F10
:10755000C801E9DDF801C189C195FFEFEF1AFF0A03
:10756000C701F6011995F801882351F08089C80FE9
:10757000C701F6011995D82F682FC801D4DDEDCFCA
:10758000D03221F091898389890F01C080898C0FC5
:1075900001C080E0DF91CF911F910F91FF90EF909C
:1075A000DF90CF9008954CE758E3C0CFCF93DF939F
:1075B000FC01248135812617370741F0EC017583E2
:1075C000648365DF8AE798E39E8B8D8BDF91CF9193
:1075D00008954F925F926F927F92AF92BF92CF9237
:1075E000DF92EF92FF920F931F93CF93DF93CDB76C
:1075F000DEB729013A019B01AC012419350946097E
:1076000057098A899B89AC89BD89BC01CD016A195A
:107610007B098C099D090F94376AA80197012419E9
:107620003509460957090F949B6ACA01B9016A0DC9
:107630007B1D8C1D9D1DDF91CF911F910F91FF90A0
:10764000EF90DF90CF90BF90AF907F906F905F9062
:107650004F90089580E090E008950895CF92DF92D2
:10766000EF92FF920F931F93CF93DF936C017A01F8
:107670008B01C0E0D0E0CE15DF0589F0D8016D9117
:107680008D01D601ED91FC910190F081E02DC601B4
:107690001995892B11F47E0102C02196ECCFC70108
:1076A000DF91CF911F910F91FF90EF90DF90CF90DE
:1076B0000895DC01ED91FC910190F081E02D199489
:1076C000CF93CFB7F89480918404811127C0EAE565
:1076D000F4E08491E4E1F4E09491E82FF0E0EE0F1F
:1076E000FF1FE156FB4FA591B491EC91E92321F4E2
:1076F00061E085E30E945E3361E085E30E9422330E
:107700008CB580618CBD8CB580648CBD61E084E3F8
:107710000E94223361E083E30E942233809184043B
:107720008F5F80938404CFBFCF910895CF92EF9263
:107730000F93FC0113AE14AE15AE049668DA0F91E8
:10774000EF90CF900895CF92DF92EF92FF921F9328
:10775000CF93DF93EC0180E090E00F94CF6725EDAD
:1077600034E045E352E40F946D6920E030E04AE7ED
:1077700054E40F9436676B017C012AE037ED43EA4D
:107780005CE369857A858B859C850F9456669B01A1
:10779000AC01C701B6010F946D6926E636E646EAEC
:1077A0005EE30F94366720E030E040E85FE30F943B
:1077B00055660F94A367162FE881F9810480F5813F
:1077C000E02D603118F561E0CE0119952AE037ED22
:1077D00043EA5CE369857A858B859C850F945666C0
:1077E0009B01AC01C701B6010F946D692CEE31E528
:1077F00048E35EE30F94366720E030E040E85FE363
:107800000F9455660F94A367162F03C060E0CE0156
:107810001995612FCE01C6D2612F70E080E090E013
:107820000F94D1672D853E854F8558890F946D69DA
:107830000F94A367CE01DF91CF911F91FF90EF903E
:10784000DF90CF9092C2FC01258736874787508B07
:107850007ACFCF92DF92EF92FF92CF93DF93EC013A
:10786000DED2682F70E06F5F7F4F072E000C880B11
:10787000990B0F94D16720E030E040E05DE30F9476
:107880006D696B017C01E881F9810680F781E02D4B
:10789000CE011995811105C026E636E646EA5EE37B
:1078A00004C02CEE31E548E35EE3C701B6010F9456
:1078B0006D696B017C012AE037ED43EA5CE3698581
:1078C0007A858B859C850F9456669B01AC01C70118
:1078D000B6010F94366725ED34E045EB5FE30F9476
:1078E000366720E030E04AE754E40F946D690F9466
:1078F000A367CB01DF91CF91FF90EF90DF90CF9006
:107900000895DC01ED91FC910084F185E02D19953D
:10791000611571058105910539F06F3F7F4F8F4FDC
:107920009F4F21F080E0089582E0089581E008955E
:10793000DC01ED91FC910484F585E02D19958350CF
:107940000895DC01ED91FC910088F189E02D1995F5
:107950008F5F08956031710509F441C088F4623089
:10796000710509F454C020F4672B09F458C0089538
:107970006430710509F443C068307105C1F10895A0
:1079800060347105E1F020F46032710501F1089571
:107990006038710561F06115714009F048C0DC0183
:1079A000ED91FC910288F389E02D60E03FC0DC019D
:1079B000ED91FC910288F389E02D61E037C0DC0194
:1079C000ED91FC910288F389E02D62E02FC0DC018B
:1079D000ED91FC910288F389E02D63E027C0DC0182
:1079E000ED91FC910288F389E02D64E01FC0DC0179
:1079F000ED91FC910288F389E02D65E017C0DC0170
:107A0000ED91FC910288F389E02D66E00FC0DC0166
:107A1000ED91FC910288F389E02D67E007C0DC015D
:107A2000ED91FC910288F389E02D68E019940895A6
:107A3000DC01ED91FC910488F589E02D19958930E0
:107A400048F4E82FF0E0EE0FFF1FEA51FD4F808170
:107A50009181089580E090E00895DC01ED91FC9122
:107A6000008CF18DE02D1995843030F4E82FF0E092
:107A7000EE51FD4F8081089580E00895DC01ED9185
:107A8000FC910280F381E02D61E01995862F089525
:107A9000FC0185810895DC0115966C931597ED9195
:107AA000FC91262F30E040E050E00190F081E02D85
:107AB00061E11994DC01ED91FC910280F381E02DEC
:107AC00062E11994FC01268137818085482F4F702F
:107AD000842FB90190E00895DC019A01462F4F7080
:107AE00016962C93169717963C931797942F9F7082
:107AF00018968C911897807F892B18968C931897DD
:107B0000ED91FC91119750E00190F081E02D63E13F
:107B1000CD011994FC0167A170A592A581A5917072
:107B20000895DC0197964C93979798965C93989755
:107B300099966C9399979A968C919A9770FB80F985
:107B40009A968C939A97ED91FC9111979A01AB01BB
:107B500051700190F081E02D6DE6CD011994DC01AA
:107B60006F7097962C919797207F262B97962C9342
:107B70009797ED91FC91119798963C9198979996CB
:107B80004C9199979A965C9151700190F081E02DFB
:107B90006DE61994DC016F7098963C919897307F50
:107BA000362B98963C939897ED91FC911197979668
:107BB0002C91979799964C9199979A965C915170C0
:107BC0000190F081E02D6DE61994DC016F779996B4
:107BD0004C9199974078462B99964C939997ED91B3
:107BE000FC91119797962C91979798963C9198971E
:107BF0009A965C9151700190F081E02D6DE6199498
:107C0000FC0191A5990F9595292F092E000C330B96
:107C100020743327220F331F892F8F77822B0895EB
:107C2000DC01ED91FC910280F381E02D6FE6199467
:107C3000DC01ED91FC910084F185E02D1995CB01DB
:107C400093700895DC01ED91FC910084F185E02DA5
:107C5000199577FB882780F90895DC01ED91FC9157
:107C60000084F185E02D19958F710895DC01ED9167
:107C7000FC910084F185E02D1995892F817008957C
:107C8000DC01ED91FC910084F185E02D199591FBCB
:107C9000882780F90895DC01ED91FC910084F1853D
:107CA000E02D199592FB882780F90895DC01ED916C
:107CB000FC910084F185E02D199593FB882780F9CC
:107CC0000895DC01ED91FC910084F185E02D19957A
:107CD00094FB882780F90895DC01ED91FC910084E4
:107CE000F185E02D199595FB882780F90895DC0131
:107CF000ED91FC910084F185E02D199596FB882784
:107D000080F90895DC01ED91FC910084F185E02D6E
:107D1000199597FB882780F90895FC01228133810A
:107D20008481482F4F70842FB90190E00895DC01C1
:107D30009A01462F4F7012962C93129713963C93EC
:107D40001397942F9F7014968C911497807F892B92
:107D500014968C931497ED91FC91119750E001903B
:107D6000F081E02D60E1CD011994DC016F71129674
:107D70008C911297807E682B12966C931297ED91DE
:107D8000FC911197262F13963C91139714968C9182
:107D90001497482F4F7050E00190F081E02D60E182
:107DA000CD011994DC016F7113968C911397807E2D
:107DB000682B13966C931397ED91FC911197129683
:107DC0002C911297362F14968C911497482F4F7040
:107DD00050E00190F081E02D60E1CD011994DC01CB
:107DE0006F7014968C911497807F682B14966C9307
:107DF0001497ED91FC91119712962C91129713966E
:107E00003C911397462F4F7050E00190F081E02D88
:107E100060E1CD011994FC0182818F710895FC010C
:107E200083818F710895DC016770962F9295907F02
:107E300092966C9192976F78692B92966C93929729
:107E4000ED91FC91119792962D913D914D915C9100
:107E500095970190F081E02D6CE6CD011994DC013D
:107E600092968C91929760FB87F992968C93929759
:107E70006695677093968C919397887F682B9396FD
:107E80006C939397ED91FC91119792962D913D9162
:107E90004D915C9195970190F081E02D6CE6CD01BC
:107EA0001994DC0193968C91939760FB87F99396D4
:107EB0008C93939761FB882780F994966C919497A3
:107EC0006E7F682B94966C939497ED91FC9111972B
:107ED00092962D913D914D915C9195970190F081F5
:107EE000E02D6CE6CD011994DC0194962C919497C9
:107EF00060FB21F994962C939497ED91FC91119746
:107F000092962D913D914D915C9195970190F081C4
:107F1000E02D6CE619946F70DC0195962C91959785
:107F2000207F622B95966C939597ED91FC9111971C
:107F300092962D913D914D915C9195970190F08194
:107F4000E02D6CE61994CF93DF93EC01E881F98181
:107F50000280F381E02D6CE619956AA37BA38CA3C4
:107F60009DA3DF91CF910895CF93DF93EC01EBDFD9
:107F70008AA182958770DF91CF910895CF93DF9387
:107F8000EC01E1DF9AA1991F9927991F8BA18770B6
:107F9000880F892BDF91CF910895CF93DF93EC0168
:107FA000D2DF9BA1991F9927991F8CA18170880FFF
:107FB000892BDF91CF910895CF93DF93EC01C3DF3D
:107FC0008CA186958170DF91CF910895CF93DF9337
:107FD000EC01B9DF8DA18F70DF91CF910895DC01A5
:107FE00092964D935D936D937C939597ED91FC9153
:107FF0000190F081E02D9A01AB016CE619946F704D
:10800000DC0192962C919297207F622B92966C9332
:108010009297ED91FC91119792962D913D914D91F2
:108020005C9195970190F081E02D6CE61994CF93C7
:10803000DF93EC0188DF8AA18F70DF91CF910895E3
:10804000CF92DF92EF92CF93DF93EC01E881F98139
:108050000280F381E02D60E019956B01E82E23E0AA
:10806000E222CA8ADB8A2E2D23709C899C7F922B68
:108070009C8B8E2DB60190E0DF91CF91EF90DF9039
:10808000CF900895DC019A01462F437052962C93AD
:10809000529753963C935397942F937054968C9188
:1080A00054978C7F892B54968C935497ED91FC9127
:1080B000119750E00190F081E02D60E0CD0119941E
:1080C000DC0152968C91529760FB82F952968C9308
:1080D0005297ED91FC911197282F53963C9153970D
:1080E00054968C915497482F437050E00190F08142
:1080F000E02D60E0CD011994DC0152968C915297ED
:1081000060FB84F952968C935297ED91FC911197F4
:10811000282F53963C91539754968C915497482FFF
:10812000437050E00190F081E02D60E0CD011994A2
:10813000DC0153968C91539760FB80F953968C9396
:108140005397ED91FC91119752962C915297382F9D
:1081500054968C915497482F437050E00190F081D1
:10816000E02D60E0CD011994CF93DF93EC0168DF3F
:108170008A8982FB882780F9DF91CF910895FC01DD
:1081800023A534A585A5482F4F73842FB90190E00E
:108190000895DC019A01462F4F739B962C939B9771
:1081A0009C963C939C97942F9F739D968C919D9742
:1081B000807C892B9D968C939D97ED91FC911197D6
:1081C00050E00190F081E02D60E7CD011994CF934C
:1081D000DF93EC0161E088810E94223361E08C81B1
:1081E0000E94223362E08A810E942233E881F98171
:1081F000E152FC4FE491EE83EA81FB81E152FC4FB6
:10820000E491EF83EC81FD81E152FC4FE491E8873A
:10821000DF91CF9108959F92AF92BF92CF92DF925C
:10822000EF92FF920F931F93CF93DF938C01942EC5
:1082300087E0C82ED12CE12CF12CC0E0A62EB12C69
:10824000C501911019C00E2C02C0959587950A940E
:10825000E2F780FF02C061E001C060E0F8018081C8
:108260000E945E3361E0F80184810E945E33F80170
:108270008281911016C007C00C2C02C0959587957D
:108280000A94E2F7E6CF0E948D3321E030E0892B9B
:1082900011F420E030E00E2C01C0220F0A94EAF71E
:1082A0000DC00E948D3321E030E0892B11F420E0D5
:1082B00030E00C2C01C0220F0A94EAF7C22B60E0D8
:1082C000F80184810E945E33FFEFEF1AFF0A81E01C
:1082D000C81AD108E8E0EE16F10409F0B1CF8C2FEE
:1082E000DF91CF911F910F91FF90EF90DF90CF9092
:1082F000BF90AF909F9008950F931F93CF93DF93FC
:108300008C01D62F672F41E086DFC82F41E06D2F0B
:10831000C80181DF2C2F30E0322F2227A901482B02
:10832000CA01DF91CF911F910F9108950F93FC0126
:1083300030E080E092E1AAE7B0E0481759076A0709
:108340007B0740F4B695A795979587953F5F3630A4
:10835000A1F737E091E09327222311F020E501C037
:1083600020E7892F86950C70082B022B00839170D3
:1083700091830F91089520918304222399F04FB7A0
:10838000F89420918304213059F42DB32093810473
:108390003DB320918204209523232DBB4FBF02C003
:1083A000409381048CBD9DBD08958EBD00000DB429
:1083B00007FEFDCF8EB508950CB405FC0DC09EBD23
:1083C00000000DB407FEFDCF9EB58EBD00000DB4BC
:1083D00007FEFDCF8EB508958EBD00000DB407FEDB
:1083E000FDCF8EB59EBD00000DB407FEFDCF9EB53E
:1083F000089580918304882361F09FB7F8942091B9
:10840000830480918104213019F48DBB9FBF0895AE
:108410008FBF0895CF93DF93FC0112821382848172
:10842000807F84831582168217828085807F808773
:10843000218732874387548780E090E0A0E0BFE344
:1084400085879687A787B08B8CEF92E09183808396
:10845000128A138A84898C7F848B158A168A87896D
:10846000807F878B108E118E828D807F828F138EFE
:10847000148E158E868D8E7F868F178E10A281A109
:10848000807881A3DF01929685E0ED0119928A95AB
:10849000E9F717A210A611A682A58E7F82A713A6C0
:1084A00014A685A5807C85A786A58C7F86A770AB42
:1084B00067A712AA11AADF91CF910895FC0187A5A1
:1084C0000C945E33AF92BF92CF92DF92EF92FF9205
:1084D0000F93CF93DF931F921F92CDB7DEB75C014E
:1084E000F62EFC0181A992A9892B09F44EC060E007
:1084F000C501E4DF41E06F2DF50181A992A98BDE72
:1085000060E070E0F50181A992A9F6DE60E070E01C
:10851000F50181A992A9F0DE61E0C501CFDF60E03D
:10852000C501CCDF41E06F2DF50181A992A973DE71
:10853000F501818B41E060E081A992A96CDEC82E33
:10854000D12CE12CF12CFE2CED2CDC2CCC2441E0A8
:1085500060E0F50181A992A95EDEC82AFE2CED2C0F
:10856000DC2CCC2441E060E0F50181A992A953DE26
:10857000C82AFE2CED2CDC2CCC2441E060E0F50177
:1085800081A992A948DEC82A41C0409110025091A9
:10859000110260911202709113020CE021E0CE01F1
:1085A0000196C4DE89819A81E6DE60E0C50186DF3E
:1085B0008F2DFBDE80E090E0FFDE80E090E0FCDECF
:1085C00061E0C5017BDF60E0C50178DF8F2DEDDE66
:1085D000F501818B80E0E9DEC82ED12CE12CF12C55
:1085E000FE2CED2CDC2CCC2480E0DFDEC82AFE2C17
:1085F000ED2CDC2CCC2480E0D8DEC82AFE2CED2C1F
:10860000DC2CCC2480E0D1DEC82AF3DE61E0C50199
:1086100055DFC701B6010F900F90DF91CF910F91F9
:10862000FF90EF90DF90CF90BF90AF9008954F9262
:108630005F926F927F928F929F92AF92BF92EF92D2
:10864000FF920F931F93CF93DF931F921F92CDB78B
:10865000DEB77C0149015A01162F1068FC0181A97F
:1086600092A9250166247724892BA9F060E0C7012F
:1086700025DF41E0612FF70181A992A9CCDDF70147
:10868000818BB20181A992A937DEB401F70181A9DA
:1086900092A932DE1CC040911002509111026091EB
:1086A0001202709113020CE021E0CE0101963EDE31
:1086B00089819A8160DE60E0C70100DF812F75DE6D
:1086C000F701818BC20178DEC40176DE92DE61E0C3
:1086D000C701F4DE0F900F90DF91CF911F910F91A2
:1086E000FF90EF90BF90AF909F908F907F906F9092
:1086F0005F904F900895CF93DF93EC0161E08FA5D9
:108700000E94223361E0CE01D9DE89A99AA900979F
:1087100009F05DDD8A899B892C89A22FA370AC01A9
:108720006A2F70E0CE01AEDC4AA15BA16CA17DA1F5
:10873000CE0155DC4FA158A569A57AA57170CE016F
:10874000F0D98BA59CA52DA5A22FAF73AC016A2FE4
:1087500070E0CE011EDD8A819B812C81A22FAF703B
:10876000AC016A2F70E0CE01E2DA68E0CE0147DCAE
:10877000E881F9810688F789E02D61E0CE01DF917B
:10878000CF911994DC01ED91FC910280F381E02DF1
:1087900064E01994F7DF64FB882780F90895CF938C
:1087A000DF93EC01F7DF811105C0CE0140DC91E0E1
:1087B000811101C090E0892FDF91CF910895FC01D4
:1087C000258936898789482F4F70842FB90190E019
:1087D0000895DC019A01462F4F7055962C935597BA
:1087E00056963C935697942F9F7057968C91579717
:1087F000807F892B57968C935797ED91FC91119719
:1088000050E00190F081E02D64E1CD011994FC016C
:10881000208D318D828D482F4F70842FB90190E0CB
:108820000895DC01ED91FC910280F381E02D61E778
:108830001995862F089508950E94A331FCDF0F94A7
:108840009465C0E0D0E00F942D662097E1F30E947C
:108850000000F9CF0E94697F4091540C909134023E
:108860002091550C3091560C609154027091550234
:108870002627372760914B0C70914C0C2627372701
:10888000949FA0011124440F452F441F550B51956F
:1088900024273527A9014827CA0120918A0430914D
:1088A0008B042817390731F090938B0480938A0446
:1088B00081E0089580E00895E3E6F6E080E091919C
:1088C000992311F08927FBCF90918C0491110BC053
:1088D00091E020918904281301C090E090938804CE
:1088E00091E090938C049091880491118093890475
:1088F00081E0911101C080E008950E94697F982F66
:1089000081E020918704291302C080E008959093AC
:10891000870408955D9A88E28A950000E9F78091BE
:1089200094048E7F8093940408955D9880919404BC
:108930008E7F80939404089588EF0E947C5088E293
:108940008A950000E9F708958AEF0E947C5088E23A
:108950008A950000E9F7089580919404982F937008
:10896000913029F081608D7F80939404EDCF08953C
:10897000CF93C82F807F0E947C508C2F8295807F60
:108980000E947C5088E28A950000E9F7CF91089513
:10899000CF93DF931F92CDB7DEB790919404292F28
:1089A0002370233039F0916092609093940489830E
:1089B000C3DF89810F90DF91CF91DACF1F93CF93DF
:1089C000DF931F92CDB7DEB7182F811102C080E26E
:1089D00001C084E2611102C090E001C092E0892BE5
:1089E0006983D6DF9091940410FB92F9892F6981F5
:1089F00060FB83F9809394040F90DF91CF911F91D6
:108A000008956091940462FB992790F9891721F0E9
:108A100063FB662760F9D2CF0895CF93C82F81E01A
:108A2000F0DFC11102C082E201C083E2B1DF9091A8
:108A30009404C0FB94F990939404CF91089590917D
:108A40009404929591708913E8CF089561E081E0D4
:108A5000B5DF61E081E0B2DF80E0DFCFCF93C82FE8
:108A600080E0CFDF8C2F8F738068CF9191CFCF9331
:108A7000C82F80E0C6DF8C2F8F738064CF9188CFA2
:108A80001F93CF93DF931F92CDB7DEB7182F81E0EE
:108A90006983B7DF6981862F80687ADF812F8F70C5
:108AA00080680F90DF91CF911F9172CF80E0A9DF96
:108AB00081E06EDF6FE070E080E090E00C946A315E
:108AC00029DFF4DF61E081E079DF2FCF23DFBEDF34
:108AD000EDDF61E081E072DF28CFCF93C82F85E022
:108AE000BDDF3ADFC11102C0C6E001C0C4E080E0D2
:108AF0003FDF8C2FCF913CCFCF92DF92EF92FF924E
:108B00001F93CF93DF931F921F92CDB7DEB7698378
:108B10007A83ADDF21DF6981C62E7A81D72E11E1FC
:108B2000115059F0F601E590F4908F2D21DF8E2D34
:108B30001FDF82E0C80ED11CF3CF0F900F90DF91A2
:108B4000CF911F91FF90EF90DF90CF900895CF933A
:108B5000DF93C0E06C2F80E093DFFEDED1E1D150E7
:108B600029F080E005DF80E003DFF9CFCF5FC0327E
:108B700089F7DF91CF910895CF92DF92EF92FF9224
:108B80000F931F93CF93DF931F92CDB7DEB7982F2C
:108B9000623010F06250985FC62EC29480EFC822F7
:108BA0008A01D12C6D2D6C0D892F998369DFD4DE5C
:108BB000F801E590F4908F2DDBDE8E2DD9DED39475
:108BC0000E5F1F4F998180E1D812ECCF0F90DF919B
:108BD000CF911F910F91FF90EF90DF90CF9008956C
:108BE00080E02DDF67ED77E180E090E085DF67EBE7
:108BF00077E180E190E080DF67E977E180E290E073
:108C00007BDF67E777E180E390E076DF47E158E1DB
:108C100060E080E0B1DF47EF57E161E080E0ACDF8A
:108C200047E557E161E085E0A7DF80E056CFCF93CD
:108C3000DF93EC018991882311F09ADEFBCFDF915D
:108C4000CF9108950F931F93CF93DF93CDB7DEB7E6
:108C500027970FB6F894DEBF0FBECDBF6330B1F0DB
:108C600038F46130B1F0623049F523E437E113C0E4
:108C7000653031F040F0663009F523E537E10BC08F
:108C80002FE437E108C02BE437E105C027E437E1E2
:108C900002C02FE337E19F938F933F932F938E0171
:108CA0000F5F1F4F1F930F930F947C6FC801BFDF9F
:108CB0000F900F900F900F900F900F9027960FB678
:108CC000F894DEBF0FBECDBFDF91CF911F910F9102
:108CD00008950F931F93CF938C01C62FF8018191B4
:108CE0008F01882329F0CC2319F042DEC150F6CF42
:108CF000CF911F910F910895CF92DF92EF92FF9243
:108D00000F931F93CF93DF93CDB7DEB727970FB69F
:108D1000F894DEBF0FBECDBF8C0188E09FDEF80166
:108D200060817181828193812CE3C22ED12CE12C50
:108D3000F12CA70196010F94796ACA01B901A70124
:108D400096010F94796A8E010F5F1F4F243631050B
:108D500098F47F936F933F932F9389E297E19F93CA
:108D60008F931F930F930F947C6F0FB6F894DEBF11
:108D70000FBECDBF85E012C07F936F933F932F93BB
:108D800081E297E19F938F931F930F930F947C6FD2
:108D90000FB6F894DEBF0FBECDBF86E0F801E80F36
:108DA000F11D80E28083D8DD66E0C80192DF27965E
:108DB0000FB6F894DEBF0FBECDBFDF91CF911F91EC
:108DC0000F91FF90EF90DF90CF900895CF93DF93B6
:108DD000FC018491EF012196882319F0C9DDFE0181
:108DE000F8CFDF91CF910895CF92DF92EF92FF926B
:108DF0000F931F93CF93DF93C42E623010F0625015
:108E0000805F982F9170D92EC82FC695D62FD295F6
:108E1000D07F87E3E82E88E1F82E01E0F701149176
:108E2000602F6D0F8C2F2CDE97DDCC2051F0D110F0
:108E300002C0812F01C080E09BDDDD2021F0812F69
:108E400003C080E095DD80E093DD0F5FFFEFEF1A58
:108E5000FF0A053019F7DF91CF911F910F91FF9015
:108E6000EF90DF90CF9008958F929F92AF92BF9234
:108E7000DF92EF92FF920F931F93CF93DF93D82E41
:108E800069E10F94466A20E1929FC001112469E1D3
:108E900070E00F94666A80E090E85C0102C0B594CF
:108EA000A7946A95E2F711E0ED2CF12C612F8CE08C
:108EB000E7DD52DD20E030E000E0490189E1880E85
:108EC000911CE814F90434F42E153F0534F0C0E089
:108ED000D0E004C0CFEFDFEF01C0E501113051F069
:108EE0001D3041F0033011F4C16006C0011104C00F
:108EF000D06802C0CFEFDFEF8D2F3ADD8C2F38DD49
:108F00000F5F940124363105C1F61F5F1E3071F6E4
:108F10008CE0A4DD21DD80E22BDD29E02D1530F48D
:108F200064E0C7018FDE8CE397E105C063E0C70111
:108F300089DE88E397E1DF91CF911F910F91FF9038
:108F4000EF90DF90BF90AF909F908F903FCFCF93E7
:108F5000C82F0E94A17FC11104C090918604981768
:108F600021F080938604CF917FCFCF9108951F93F6
:108F7000CF93DF931F92CDB7DEB7182F80E16983BF
:108F80006DDDEADC6981662349F0111102C012E04F
:108F900001C010E080E0ECDC812F03C080E2E8DC5F
:108FA00080E20F90DF91CF911F91E2CCCF92DF92C0
:108FB000EF92FF920F93CF93DF93C82F6B017A014B
:108FC000D22F813049F028F0823049F0833039F0D7
:108FD00008C081E043DD05C081E140DD02C089E0D9
:108FE0003DDDBADC63E0C6012DDEDD2341F08AE120
:108FF000BFDC63E0C70126DE011106C015C00023F7
:1090000099F083E397E1E2DE41E04D276C2F85E0A4
:10901000EBDE4D2F6C2F89E0DF91CF910F91FF9008
:10902000EF90DF90CF90E0CEDF91CF910F91FF9046
:10903000EF90DF90CF9008950F93CF936115710556
:1090400089F0C1E0681779073CF49C01261B370BB7
:109050002330310544F406C09B01281B390B233013
:1090600031050CF4C0E02091140221702C1711F08E
:1090700001E001C0042F2C2FAB01BC0180E096DF82
:1090800080911402C0FB80F980931402CF910F915C
:1090900008950F93CF936115710589F0C1E06817AA
:1090A00079073CF49C01261B370B2330310544F42F
:1090B00006C09B01281B390B233031050CF4C0E09E
:1090C0002091140222FB222720F92C1711F001E035
:1090D00001C0042F2C2FAB01BC0181E067DF809120
:1090E0001402C0FB82F980931402CF910F9108956E
:1090F000CF93C82F86E0B2DC2FDC63E08C2F90E0AA
:10910000A1DD85E2CF9134CCCF93DF93EC0186E1F2
:10911000A5DC22DC63E0CE0195DD85E2DF91CF9115
:1091200027CC4F925F926F927F928F929F92AF92D5
:10913000BF92CF92DF92EF92FF921F93CF93DF9374
:1091400000D01F92CDB7DEB7F82E811104C082DBAC
:10915000882309F467C00E94697F182F0F94A561C6
:1091600069837A838B839C83A0905402B0905502CC
:1091700060914F0C7091500C8091510C9091520C59
:109180000F949E672B013C01C0904B0CD0904C0C6F
:109190008090550C9090560C6091590C70915A0C1F
:1091A00080915B0C90915C0C0F949E67DC01CB016D
:1091B0004F2DB40141DF4F2DB601C2016ADF20916E
:1091C000540CE22EF12C11110DC09091340297FD38
:1091D00009C0929F900111247901EE0CEF2CEE1C36
:1091E000FF08F19424E62E9DC0012F9D900D1124BF
:1091F00081589F4F6FEF70E00F94666A862F78DF7B
:10920000CE01019679DDC5017FDFEF2811F0812FB6
:1092100064DC61E01C141D041CF060E080E001C00F
:10922000812FA5DE0F900F900F900F90DF91CF91BF
:109230001F91FF90EF90DF90CF90BF90AF909F90E5
:109240008F907F906F905F904F900895CF9388E1BB
:1092500005DC82DB83E696E00E94767EC82F66E11D
:1092600083E696E036DDC63120F480E281DBCF5F15
:10927000FACFCF910895811103C01EDB882311F02E
:10928000E5DF3BCB0895CF93C82F44DB8C2F49DF1C
:109290008C2FF1DF8C2F5BDECF9147CB3BDBD6DB16
:1092A00005DC55DC9DDC81E0EEDF3FCB80E0EBCFE1
:1092B00090918504981729F0809385048111EECF51
:1092C000FFCB0895E2EAF4E083AF64AF0895EF9234
:1092D000FF920F931F93CF93DF937A016F3F710536
:1092E0008105910509F058F482EA94E00E94593B07
:1092F00086EA94E00E948B38282F30E014C0C09199
:10930000DD04D091DE044D2F50E0EC2FF0E08B0116
:109310009C01BF0186EA94E0ADD1C80FC093DD0483
:10932000D093DE049C01C901DF91CF911F910F9171
:10933000FF90EF900895EF92FF920F931F93CF93BA
:10934000DF938B01C2EAD4E0FBACECAC4E2D50E0D5
:109350006F2D70E09C0186EA94E0E4D1F80EFBAE3C
:10936000ECAEDF91CF911F910F91FF90EF90089598
:10937000EF92FF920F931F93CF93DF938B01C2EA7B
:10938000D4E0FBACECAC4E2D50E06F2D70E09C01B6
:1093900086EA94E013D2F80EFBAEECAEDF91CF91EB
:1093A0001F910F91FF90EF9008950F931F93CF930C
:1093B000DF93CDB7DEB728970FB6F894DEBF0FBEA8
:1093C000CDBF8A0123E0660F771F2A95E1F7680F6A
:1093D000791F48E050E0CE0101960F94B06E2981CC
:1093E0003A81F801808191812817390790F082171E
:1093F000930760F09C818281981758F081E090E09B
:109400003B812381231738F080E005C081E090E0A4
:1094100002C08FEF9FEF28960FB6F894DEBF0FBE05
:10942000CDBFDF91CF911F910F910895EF92FF92E1
:109430000F931F93CF93DF93EC018B017A018A8501
:109440009B858617970731F0888199810E94D63ACB
:109450001B870A8788859985019689F00E811F816F
:10946000B701888199810E94D33A080F111D888520
:1094700099858017910718F481E090E011C06E8102
:109480008A81680F97014C81888199810E94E73910
:109490002E813F81280F311D3F832E8380E090E095
:1094A000DF91CF911F910F91FF90EF9008954F9210
:1094B0005F926F927F928F929F92AF92BF92CF9264
:1094C000DF92EF92FF920F931F93CF93DF93CDB76D
:1094D000DEB72D970FB6F894DEBF0FBECDBF6C017F
:1094E0002A013B01490158011B861C86CE010196C9
:1094F0007C0188E0F70111928A95E9F7DB01CA0146
:1095000027E0B695A795979587952A95D1F79A83E1
:109510008983F42FFF77FD878F2F80588B838C836F
:109520001A8619864F3F51056105710509F018F437
:1095300060E070E026C060919704709198048E01FD
:10954000075F1F4F970145ED59E480919504909175
:1095500096040E94C77C97FDEBCF69857A8583E0EE
:10956000660F771F8A95E1F7809195049091960494
:10957000680F791F48E050E0C7010F94B06E6F810B
:1095800078856115710519F44B86B60106C0C616BB
:10959000D70619F08D8580688B87AE01455F5F4FD8
:1095A000C401F50119952D960FB6F894DEBF0FBED4
:1095B000CDBFDF91CF911F910F91FF90EF90DF9082
:1095C000CF90BF90AF909F908F907F906F905F9063
:1095D0004F9008956F927F928F929F92AF92BF9219
:1095E000CF92DF92EF92FF920F931F93CF93DF936F
:1095F00000D01F92CDB7DEB76C017B013A01590153
:10960000480119821A821B821C82AE014F5F5F4F94
:10961000B301C7010E94277D7C0149815A816B817A
:109620007C81411551056105710529F08401950181
:10963000C6013DDFE6CF0F900F900F900F90DF91A6
:10964000CF911F910F91FF90EF90DF90CF90BF903F
:10965000AF909F908F907F906F90089521E020931E
:109660009904E5E9F4E0918380837383628380E069
:1096700090E008957F92AF92BF92CF92DF92EF92E7
:10968000FF920F931F93CF93DF93CDB7DEB72C9745
:109690000FB6F894DEBF0FBECDBF6C01762EF72F4C
:1096A000842FE52FB901A801D6011496AD90BC9086
:1096B00015979091990491110AC02BE738E1482F32
:1096C000672DC6010E941E3A80E090E019C0DA8240
:1096D000C9827B82FC838D83EE8318861F82FA8683
:1096E000E9861C861B8606E11AE49E012F5F3F4F28
:1096F000C501DDDEB501C6010E94D63A8F8198858D
:109700002C960FB6F894DEBF0FBECDBFDF91CF9180
:109710001F910F91FF90EF90DF90CF90BF90AF908F
:109720007F900895CF92DF92EF92FF920F931F9355
:10973000CF93DF93CDB7DEB72C970FB6F894DEBF8B
:109740000FBECDBF7C01C901F701C480D580209137
:109750009904211108C02BE538E1C7010E941E3A87
:1097600080E090E01CC0FA82E9826B837C834D83A9
:109770005E8318861F821A8709871C861B8606E16E
:109780001AE49E012F5F3F4F41EC5CE7BC01C6012C
:1097900021DFB601C7010E94D63A8F8198852C96A9
:1097A0000FB6F894DEBF0FBECDBFDF91CF911F91F2
:1097B0000F91FF90EF90DF90CF900895CF92DF92BE
:1097C000EF92FF920F931F93CF93DF93CDB7DEB746
:1097D0002C970FB6F894DEBF0FBECDBF7C01C90138
:1097E000F701C480D58020919904211108C02BE392
:1097F00038E1C7010E941E3A80E090E01CC0FA8266
:10980000E9826B837C834D835E8318861F821A876F
:1098100009871C861B8606E11AE49E012F5F3F4FD5
:1098200044EC5CE7BC01C601D5DEB601C7010E946D
:10983000D63A8F8198852C960FB6F894DEBF0FBE6E
:10984000CDBFDF91CF911F910F91FF90EF90DF90EF
:10985000CF900895CF93DF93EC01262F4CAD6BADE5
:1098600004960E94C9392BAD082E000C990B820F6B
:10987000911D8BAF81E090E0DF91CF9108950F9320
:109880009CE0899F802D112421E0280F2093A104C2
:10989000845F8093A00490E002964091DA0450E047
:1098A0008417950714F480E033C0822F90E0209154
:1098B000DC0430E082179307B4F76623A9F061E077
:1098C00086EA94E00E9452364091A1044E5F0BE07C
:1098D00020E860E086EA94E00E94463860E086EA8C
:1098E00094E00E94523605C061E086EA94E00E944E
:1098F00052366091A0048091DA046817A0F290912A
:10990000A1048091DC04891770F280E0DBDC81E047
:109910000F910895CF93DF93FC0185ADEF0124965D
:10992000811105C081E085AFCE010E94F935CE01DD
:10993000DF91CF910C9430366FEF7FEF19CD6FEF41
:109940007FEFF9CC4FEF5FEFC2CC482F50E0209172
:109950009F04022E000C330B4217530781F08093B3
:109960009F04813031F466E571E286EA94E00C945C
:10997000D63A66E679E186EA94E00C94D63A089500
:10998000EF92FF920F9382EA94E0C4DF88E1E82E21
:109990008FE1F82E00E428E040E060E086EA94E001
:1099A0000E947C3669EB74E086EA94E00E94D63A25
:1099B00026E133E041E169E386EA94E00E94E73979
:1099C00069E27DE086EA94E00E94D63A2DE133E038
:1099D0004CE16AE386EA94E00E94E73964E870E1CA
:1099E00086EA94E00E94D63A2DE233E049E26BE346
:1099F00086EA94E00E94E73964E870E186EA94E040
:109A00000E94D63A29E333E04EE36DE386EA94E020
:109A10000E94E7392BE333E04EE362E486EA94E008
:109A20000E94E73986EA94E00E9434368111AECF75
:109A300064EC79E080E090E00E94DC9B66E679E1EE
:109A400086EA94E00F91FF90EF900C94D63A61E093
:109A500088E19FE195DF64EC79E080E090E00C9490
:109A6000DC9BCF92DF92EF92FF920F931F93CF93E5
:109A7000DF93EDDFC091A6040091A704D0E0BE0102
:109A80006853710977FF02C06F5F7F4F75956795C7
:109A9000D62E82EA94E03EDFCE01C0979695879558
:109AA000182FC257D109D695C7954EEEC42EC00EB9
:109AB000DAEFD00F83E9E82E8EE1F82E03E127E0FC
:109AC0004CE06D2D86EA94E00E947C3683E03DDF19
:109AD0002BE333E04C2D612F86EA94E00E94E739B6
:109AE00024E433E04D2F6C2F86EA94E00E94E7399E
:109AF00086EA94E00E9434368111DCCF64EC79E090
:109B000080E090E0DF91CF911F910F91FF90EF9057
:109B1000DF90CF900C94DC9B60E070E086E591E2F2
:109B20009DCD1F93CF93DF930E946645C091A704FC
:109B3000C695C69582EA94E0EDDEDC2FDD0F1D2F81
:109B40001C0F83E002DF6C2F80E0BCDB83E696E035
:109B5000F6DE6D2F80E0B6DB88EA98E1EDDE612F5E
:109B600080E0B0DB8BE998E1E7DE86EA94E00E94D2
:109B700034368111E6CFDF91CF911F91089508957A
:109B8000CF939CE0899F802D112421E0280F209302
:109B9000A104845F8093A004E82FF0E03296409106
:109BA000DA0450E0E417F5070CF441C030E04091CE
:109BB000DC0450E0241735070CF039C0C62F682F9D
:109BC0008EE380DB65E470E080E090E0BBDE61E383
:109BD0006C0F062E000C770B880B990BB3DE60E23E
:109BE00070E080E090E0AEDE6091590C70915A0C0C
:109BF00080915B0C90915C0C0F949E67CB010E944E
:109C0000B89C9DDE6FE270E080E090E09BDE0E94F9
:109C1000697F811104C08091FF0B811108C0809180
:109C2000550C9091560C0E94B89CCF9188CECF9144
:109C30000895CF92DF92EF92FF920F931F93CF93ED
:109C4000DF931F921F92CDB7DEB77B01622F49834E
:109C500016DE4981882309F440C0442309F1011527
:109C60001105F1F4C7010E94977E26E130E0281B20
:109C7000310937FF02C02F5F3F4F3595279530E8F8
:109C80002158822F830F87FD0CC060E270E080E0D6
:109C900090E02A83398356DE398131502A81F1CF11
:109CA00030E8C32ED12CB601C70162DB7601E81A79
:109CB000F90A0115110511F41E2D06C0FF24B70184
:109CC000C80139DB1E2D181B173038F060E270E038
:109CD00080E090E037DE181BF7CF0F900F90DF91F8
:109CE000CF911F910F91FF90EF90DF90CF9008954B
:109CF0000F93CF93DF93982F862FEA01692FBFDD53
:109D0000882309F168E770E0CE0132DBC8E7C81BA1
:109D1000C73038F060E270E080E090E013DEC81BEE
:109D2000F7CF6091A0048AE7CDDA602F000F770BA0
:109D3000880B990B07DE60E270E080E090E0DF9135
:109D4000CF910F91FFCDDF91CF910F910895CF92D9
:109D5000DF92EF92FF920F931F93CF93DF93982F91
:109D6000862F6A017901692F8ADD882309F442C0B0
:109D7000C701002321F00E94977E182F03C00E9484
:109D8000767E182FC4E1D0E0C11BD1098C2F880F3B
:109D9000C80FCC0FD0E0BE01C601EADAC81B6AE3E7
:109DA00070E080E090E0CEDDC73038F060E270E037
:109DB00080E090E0C7DDC81BF7CF8AEF189F802DA9
:109DC00011246091A00480587DDAC701002349F076
:109DD000DF91CF911F910F91FF90EF90DF90CF9087
:109DE000ABCDDF91CF911F910F91FF90EF90DF905E
:109DF000CF90A5CDDF91CF911F910F91FF90EF9064
:109E0000DF90CF900895BF92CF92DF92EF92FF92B2
:109E10000F931F93CF93DF936C017B010E94977E7A
:109E2000C82FC7010E94767E04E110E0081B1109CB
:109E30008C2F90E0BB24B394081719071CF0B12CA9
:109E4000C5E201C0CFE12C2F30E0A9014E5F5F4F8A
:109E50008091DA0490E04817590744F029503109FD
:109E60008091DC0490E0821793079CF5D0E0E11428
:109E7000F104B1F16AE370E080E090E063DDBB20C3
:109E800081F0C45F8091DA04C81750F12C2F30E0C4
:109E9000295031098091DC0490E0821793071CF46B
:109EA0001FC0DD23E9F0802F880F800F6C2F880FF3
:109EB00009DA60E270E080E090E044DDC701DF9104
:109EC000CF911F910F91FF90EF90DF90CF90BF90B7
:109ED00036CD6C2F80E0F6D9C6012EDDD1E0C7CF9C
:109EE000DF91CF911F910F91FF90EF90DF90CF9076
:109EF000BF900895EF92FF920F93CF93DF93D82FE7
:109F0000C62F7901682F8C2FBADC8823D9F0002363
:109F100029F062E070E080E090E014DD2D2F4C2FFE
:109F200065E1C7010E941A7F6EE770E004DACEE7B0
:109F3000C81BC73038F060E270E080E090E002DDDE
:109F4000C81BF7CFDF91CF910F91FF90EF9008954D
:109F50008F929F92AF92BF92CF92DF92EF92FF9239
:109F60000F936B017C0180909B0490909C04A090C7
:109F70009D04B0909E04A50194010F942F6788233F
:109F800001F120E030E0A901C701B6010F942F676D
:109F9000882351F0A5019401C701B6010F942F67E2
:109FA00087FD04C081E003C080E001C08FEF809393
:109FB0009A04C0929B04D0929C04E0929D04F0927B
:109FC0009E048091DA04813128F48091DC0483308E
:109FD00008F048C08091DA04853128F48091DC04CF
:109FE000843108F04FC08091DA048F3308F057C0F5
:109FF0008091DC048F3208F452C086E0E82E89E1BB
:10A00000F82E00E123E04FE265E086EA94E00E944A
:10A010007C3696E3E92E99E1F92E23E04FE26AE5DA
:10A0200086EA94E00E947C3680919A0440E3481BC3
:10A030002CEEE22E28E1F22E0DE022E06EE686EA1A
:10A0400094E00E947C3680919A0441E3481B32EDF3
:10A05000E32E38E1F32E22E069E186EA94E00E94E3
:10A060007C361DC080919A0444E0481B57EBE52ED6
:10A0700058E1F52E0CE022E062E486EA94E00E94CA
:10A080007C36A8CF4FECE42E48E1F42E01E023E02B
:10A0900044E16CE386EA94E00E947C36A4CF0F9101
:10A0A000FF90EF90DF90CF90BF90AF909F908F90F8
:10A0B0000895CF92EF920F93CF93DF93C2EAD4E04B
:10A0C0001B821A828CE593E099838883CC24CA94FE
:10A0D000EE24EA9402E522E143E165E172E0CE017B
:10A0E0000E94963B88E693E099838883DF91CF9125
:10A0F0000F91EF90CF9008955A9887FD52C05B98CA
:10A1000000000000000000005A9A5A98282F220FE1
:10A1100086FD53C05B9800000000000000005A9AC2
:10A120005A98922F990F26FD46C05B9800000000B8
:10A13000000000005A9A5A98892F880F96FD39C05E
:10A140005B9800000000000000005A9A5A98982F6F
:10A15000990F86FD2CC05B980000000000000000F5
:10A160005A9A5A98892F880F96FD1FC05B98000055
:10A170000000000000005A9A5A98982F990F86FD07
:10A1800012C05B9800000000000000005A9A5A9824
:10A1900096FD15C05B9800000000000000005A9A70
:10A1A00008955B9AADCF5B9AEDCF5B9AE0CF5B9A57
:10A1B000D3CF5B9AC6CF5B9AB9CF5B9AACCF5B9A91
:10A1C000EACF2F923F925F927F929F92AF92BF927F
:10A1D000CF92DF92EF92FF920F931F93CF93DF9373
:10A1E0007C011B01942E69018AE0481709F47BC0A9
:10A1F000A5E14A134EC0DB011296ED91FC91139735
:10A200001281C681D7815D9A88E28A950000E9F7BC
:10A2100000EE010F80E1582E510E98E2792E88EF62
:10A220006BDF872D8A950000E9F7103208F046C0F1
:10A23000812F8077806860DF812F8295807F5CDF4F
:10A24000872D8A950000E9F780E856DF80E054DF2B
:10A25000872D8A950000E9F78AEF4EDF872D8A95D2
:10A260000000E9F75E01B0E1AB0EB11C8881807F90
:10A2700043DF89918295807F3FDFCA15DB05B1F707
:10A28000872D8A950000E9F71F5F0F5F1511C7CF73
:10A290005D989601492DB101C701DF91CF911F91C2
:10A2A0000F91FF90EF90DF90CF90BF90AF909F9075
:10A2B0007F905F903F902F900C94B637802F8077DF
:10A2C00080681ADF802F8295807F16DF872D8A9520
:10A2D0000000E9F780E810DF80E80EDF872D8A951F
:10A2E0000000E9F7B9CF559A5D98539A5B98529A56
:10A2F0005A9A5D9AC8E28C2F8A950000E9F788E7A0
:10A3000090E00E94D33688EFF7DE8C2F8A9500000C
:10A31000E9F780E2F1DE80E0EFDE8C2F8A95000025
:10A32000E9F780E0E9DE80E8E7DE8C2F8A9500001F
:10A33000E9F780E0E1DE80E1DFDE8C2F8A95000026
:10A34000E9F78FE090E00E94D33680E2D5DE80E42A
:10A35000D3DE8C2F8A950000E9F780E2CDDE80E61F
:10A36000CBDECA950000E9F710E0D8E208E2812FC1
:10A3700080778068C1DE812F8295807FBDDE8D2F42
:10A380008A950000E9F780E8B7DE80E0B5DE8D2F22
:10A390008A950000E9F78AEFAFDE8D2F8A950000DD
:10A3A000E9F7C0E280E0A8DE80E0A6DE9D2F9A9566
:10A3B0000000E9F7C150B1F788EF9EDE802F8A9543
:10A3C0000000E9F71F5F103209F0D1CF80E094DE82
:10A3D00080EC92DE88E28A950000E9F75D9859CF1B
:10A3E0000E94D98C41E050E060E070E0811103C030
:10A3F00040E050E0BA0140935506509356066093F2
:10A4000057067093580610922F0681E08093090634
:10A4100083E0809324020895CF92DF92EF92FF921F
:10A420000F931F93CF93DF930E94D68D6C0161E051
:10A4300081E00E948775C0912F06D0E081E0C81AA4
:10A44000D108C11117C08091F805811104C00E9484
:10A45000647F81119BC080912402882359F081E0A0
:10A460009091F805911180E004E024E042E75AE27F
:10A470006D2F3EDC6CEB78E083E498E00E94BD93A6
:10A480008091BC088F3201F18091C90883FF1CC004
:10A49000C130C1F48091F805813021F40E94647FBD
:10A4A00081117CC080912402882361F081E0909129
:10A4B000F805913009F080E000E22EE34EE65AE222
:10A4C0006D2F16DC92E001C091E080912402882378
:10A4D00009F454C0760111E01C0F8FEFE816F8065E
:10A4E00009F44CC0C91345C060E070E0C7010E9488
:10A4F000FF899091C9088091F80594FF22C08C13C0
:10A5000054C00E94647F882309F44FC08CEB98E00C
:10A510000E94838C10922F0682E090E0A0E0B0E0D1
:10A520008093550690935606A0935706B09358060D
:10A5300081E08093090610925A0683E080932402FA
:10A5400050C08C1304C00E94647F81113DC0809173
:10A550002402882361F081E09091F8059C1380E04B
:10A5600000E02DE938E142E55AE26D2FC3DC912F7E
:10A5700001C09F5F81E0E81AF108AFCFDF5FCF5FD6
:10A58000D53009F05ECF9093F7052BC00E94CC74B4
:10A5900080910906882309F45ECF23C021DF8091D2
:10A5A0000906882309F47ECF1CC0809124028823E9
:10A5B000F1F281E09091F8059C1380E001E02DE933
:10A5C00038E140E65AE2D1CF8CEB98E00E948A88CD
:10A5D0000E94C6740E94408480910906882309F471
:10A5E000B6CFDF91CF911F910F91FF90EF90DF9049
:10A5F000CF900895CF93DF93EC01CB01BA010F9474
:10A60000D1672AE037ED43E25CE30F946D6968831C
:10A6100079838A839B83DF91CF910895CF93DF93D2
:10A62000EC01CB01BA010F94D167688379838A83E7
:10A630009B83DF91CF910895CF93DF93EC01CB0102
:10A64000BA010F94D16720E030E048EC52E40F9457
:10A650006D69688379838A839B83DF91CF910895A5
:10A66000CF93DF93EC01CB01BA010F94D16720E0C7
:10A6700030E048EC52E40F946D690F94A36768834F
:10A6800079838A839B83DF91CF910895CF93DF9362
:10A69000EC01CB01BA010F94D1672AE037ED43E218
:10A6A0005CE30F946D69688379838A839B83DF9170
:10A6B000CF9108956AEF72E589E993E50C94E0740F
:10A6C0006EE073E586EF93E50C94E0746CE173E55E
:10A6D00086EB93E50C94E07460E373E582E194E526
:10A6E0000C94E07466E473E58CE793E50C94E074F5
:10A6F0000D94B1180D94F818CF93DF9300D01F92EA
:10A70000CDB7DEB70F94D1672AE037ED43E25CE3C3
:10A710000F946D6969837A838B839C83CE01019644
:10A720000E94809F0F900F900F900F90DF91CF911C
:10A730000895CF93DF9300D01F92CDB7DEB70F946B
:10A74000D1672AE037ED43E25CE30F946D696983DA
:10A750007A838B839C83CE0101960E941A9D0F9071
:10A760000F900F900F90DF91CF910895CF93DF93CB
:10A7700000D01F92CDB7DEB70F94D16720E030E054
:10A7800048EC52E40F946D6969837A838B839C83D0
:10A79000CE0101960E94C89E0F900F900F900F90CF
:10A7A000DF91CF910895CF92DF92EF92FF926B01EC
:10A7B0007C0120E030E0A9010F942F6787FD05C0E0
:10A7C00020E030E040E05FE304C020E030E040E023
:10A7D0005FEBC701B6010F9456660F949E67CB01DD
:10A7E000FF90EF90DF90CF900C94B89C0F94D167BE
:10A7F000DACFCF93DF9300D01F92CDB7DEB70F949F
:10A80000A3670F94CF6769837A838B839C83CE0180
:10A8100001960E94C89E0F900F900F900F90DF91AD
:10A82000CF9108950F94D16720E030E048EC52E4D6
:10A830000F946D69DECFCF93DF931F921F92CDB738
:10A84000DEB789839A830E94257340E050E0BA0105
:10A8500089819A810F900F90DF91CF910C94A17410
:10A860000F931F93CF93DF9361E081E00E94877580
:10A87000C0912F06D0E0C11119C08091F805811157
:10A8800004C00E94647F8111C5C080912402882386
:10A8900009F45DC081E09091F805911180E004E039
:10A8A00024E040EB5AE26D2F23DA51C0C130D1F4DD
:10A8B0008091F805813021F40E94647F8111B2C03B
:10A8C00080912402882309F442C081E09091F80528
:10A8D000913009F080E003E02EE347EA5AE26D2F61
:10A8E00007DA35C0C230C9F48091F805823021F40E
:10A8F0000E94647F81119FC080912402882339F1D6
:10A9000081E09091F805923009F080E003E02EE3B9
:10A910004AE95AE26D2FECD91AC0C330C1F48091D4
:10A92000F805833021F40E94647F81118DC08091ED
:10A930002402882361F081E09091F805933009F0BA
:10A9400080E003E02EE345E95AE26D2FD1D90E9461
:10A950008A7481111CC0C430E1F48091F805843000
:10A9600021F40E94647F811178C0809124028823A1
:10A9700009F47CC081E09091F805943009F080E002
:10A9800003E02EE34CE85AE26D2FB2D96FC014E019
:10A9900001C015E0C1131AC08091F8058C1304C0E2
:10A9A0000E94647F811164C080912402882369F031
:10A9B00081E09091F8059C1380E003E02EE340E8ED
:10A9C0005AE26D2F95D91C2F01C01C2F81E0810FF9
:10A9D000C81317C08091F8058C1304C00E94647FCF
:10A9E00081114FC080912402882359F081E0909119
:10A9F000F8059C1380E003E02EE347E75AE26D2F51
:10AA000077D9DF5FCF5FD53009F035CF1E5F109368
:10AA1000F7053FC00E94CC7480910906882309F491
:10AA200034CF37C083EF96E506DF8091090688238F
:10AA300009F446CF2EC082E99CE5FDDE809109062F
:10AA4000882309F459CF25C08AE09AE5F4DE809185
:10AA50000906882309F46BCF1CC08BEB98E5EBDE6D
:10AA600080910906882309F480CF13C015E0AECF8A
:10AA700080E19AE7E0DE80910906882309F494CF0B
:10AA800008C081EC95E5D7DE80910906882309F49A
:10AA9000A9CFDF91CF911F910F9108952F923F92EF
:10AAA0004F925F926F927F928F929F92AF92BF92DE
:10AAB000CF92DF92EF92FF920F931F93CF93DF938A
:10AAC000CDB7DEB727970FB6F894DEBF0FBECDBF68
:10AAD0001C017F836E839C2C8D2CA982CA01B90135
:10AAE0000F949E679B01AC01EE81FF8160817181B3
:10AAF000828193812A833B834C835D830F949E677D
:10AB00002A813B814C815D815B016C01A21AB30AF1
:10AB1000C40AD50AC801B7010F949E672A813B81F8
:10AB20004C815D817B018C01E21AF30A040B150B49
:10AB3000F981FF938F929F9280E6882E83E5982E6D
:10AB40006E817F81C1010E9447730F900F900F901B
:10AB500027960FB6F894DEBF0FBECDBFDF91CF9121
:10AB60001F910F91FF90EF90DF90CF90BF90AF902B
:10AB70009F908F907F906F905F904F903F902F901D
:10AB800008956F927F928F929F92AF92BF92CF92D1
:10AB9000DF92EF92FF920F931F93CF93DF9300D03A
:10ABA0001F92CDB7DEB761E081E00E9487756090AB
:10ABB0002F06712C611019C08091F805811104C015
:10ABC0000E94647F811194C080912402882309F43B
:10ABD00086C081E09091F805911180E004E024E0C6
:10ABE0004EE85CE2672D84D87AC081E068122BC001
:10ABF0008091F805813021F40E94647F811180C02A
:10AC000080912402882309F46AC011E08091F8053C
:10AC1000813009F010E080914F0E9091500EA0917C
:10AC2000510EB091520E89839A83AB83BC83CE01BF
:10AC300001960E941A9D00E09C014AE75CE2672DA4
:10AC4000812F85D84CC082E0681224C08091F8051D
:10AC5000823021F40E94647F811183C0809124029C
:10AC6000882309F43CC011E08091F805823009F096
:10AC700010E06091970B7091980B8091990B9091D7
:10AC80009A0B91DD00E09C0146E65CE2672D812F86
:10AC90005ED825C083E0681222C08091F805833019
:10ACA00021F40E94647F811174C080912402882362
:10ACB000B1F011E08091F805833009F010E0609167
:10ACC0009B0B70919C0B80919D0B90919E0B6BDD6B
:10ACD00000E09C0146E55CE2672D812F38D8739433
:10ACE000639485E0781266CF84E08093F70568C0AE
:10ACF0000E94CC7480910906882309F465CF60C056
:10AD000020E030E048EC52E460914F0E7091500E1C
:10AD10008091510E9091520E0F946D690F949E6721
:10AD20001F921F921F922AE5822E23E5922E5B012D
:10AD30006C011CE3E12E16E8F12E01E010E020E0AA
:10AD400030E0A9016FE47EE084E89CE20E94477352
:10AD50000F900F900F9080910906882309F450CF2F
:10AD60002FC081E00E94597FA12CC12CD12CE12C55
:10AD7000F12C08E413E420E030E0A90167E97BE06E
:10AD800080E79CE28BDE80910906882309F466CF78
:10AD900017C081E00E94597FA12CC12CD12CE12C3D
:10ADA000F12C08E413E420E030E0A9016BE97BE03A
:10ADB0008EE59CE273DE80910906882309F475CF45
:10ADC0000F900F900F900F90DF91CF911F910F91E7
:10ADD000FF90EF90DF90CF90BF90AF909F908F90BB
:10ADE0007F906F900895AF92CF92DF92EF92FF9293
:10ADF0000F931F93CF93DF9361E081E00E948775EB
:10AE0000D0912F06C0E0D1111AC08091F8058111B0
:10AE100004C00E94647F811103C1809124028823B1
:10AE200009F4F5C081E09091F805911180E004E00B
:10AE300024E044E45CE26C2F0E94784EE8C0D130FC
:10AE400029F58091F805813021F40E94647F8111F9
:10AE5000EFC080912402882309F4D9C011E08091C9
:10AE6000F805813009F010E06091010F7091020F38
:10AE70008091030F9091040F96DC00E09C0146E363
:10AE80005CE26C2F812F0E94A74EC1C0D23029F501
:10AE90008091F805823021F40E94647F8111E2C024
:10AEA00080912402882309F4B2C011E08091F80552
:10AEB000823009F010E06091050F7091060F8091CB
:10AEC000070F9091080F6FDC00E09C0148E25CE204
:10AED0006C2F812F0E94A74E9AC0D33029F5809104
:10AEE000F805833021F40E94647F8111D5C08091E0
:10AEF0002402882309F48BC011E08091F805833087
:10AF000009F010E06091090F70910A0F80910B0F0A
:10AF100090910C0F48DC00E09C014AE15CE26C2F50
:10AF2000812F0E94A74E73C0D43029F58091F80577
:10AF3000843021F40E94647F8111C8C08091240272
:10AF4000882309F464C011E08091F805843009F089
:10AF500010E060910D0F70910E0F80910F0F909186
:10AF6000100F21DC00E09C014CE05CE26C2F812F93
:10AF70000E94A74E4CC0D53029F58091F805853048
:10AF800021F40E94647F8111BBC080912402882338
:10AF900009F43DC011E08091F805853009F010E01A
:10AFA00060911D0F70911E0F80911F0F9091200FC7
:10AFB000FADB00E09C0142E05CE26C2F812F0E94F2
:10AFC000A74E25C0D63019F58091F805863021F4BA
:10AFD0000E94647F8111ADC0809124028823B9F062
:10AFE00011E08091F805863009F010E06091210FA2
:10AFF0007091220F8091230F9091240FD4DB00E0F9
:10B000009C014EEE5BE26C2F812F0E94A74ECF5F1A
:10B01000DF5FC53009F0F7CE87E08093F705A1C068
:10B020000E94CC7480910906882309F4F6CE99C059
:10B0300081E00E94597FA12CC12CD12CE12C10EC75
:10B04000F12E09E714E420E030E040E85FE361E03E
:10B050007FE08DE39CE222DD80910906882309F4DC
:10B06000F8CE7FC081E00E94597FA12CC12CD12C49
:10B07000E12C10ECF12E09E714E420E030E040E888
:10B080005FE365E07FE08FE29CE208DD80910906E6
:10B09000882309F405CF65C081E00E94597FA12C67
:10B0A000C12CD12CE12C10ECF12E09E714E420E0A6
:10B0B00030E040E85FE369E07FE081E29CE2EEDCC3
:10B0C00080910906882309F412CF4BC081E00E94C9
:10B0D000597FA12CC12CD12CE12C10ECF12E09E7C9
:10B0E00014E420E030E040E85FE36DE07FE083E1DE
:10B0F0009CE2D4DC80910906882309F41FCF31C07B
:10B1000081E00E94597FA12CC12CD12CE12C10ECA4
:10B11000F12E09E714E420E030E0A9016DE17FE0C1
:10B1200087E09CE2BBDC80910906882309F42DCFDF
:10B1300018C081E00E94597FA12CC12CD12CE12C98
:10B1400010ECF12E09E714E420E030E0A90161E2FF
:10B150007FE088EF9BE2A2DC80910906882309F456
:10B160003BCFDF91CF911F910F91FF90EF90DF9038
:10B17000CF90AF900895AF92CF92DF92EF92FF926F
:10B180000F931F93CF93DF9361E081E00E94877557
:10B19000D0912F06C0E0D1111AC08091F80581111D
:10B1A00004C00E94647F8111B4C08091240288236E
:10B1B00009F4A7C081E09091F805911180E004E0C6
:10B1C00024E04EE05BE26C2F0E94784E9AC0D130B2
:10B1D00029F58091F805813021F40E94647F811166
:10B1E000A0C080912402882309F48BC011E08091D3
:10B1F000F805813009F010E06091F10E7091F20EC7
:10B200008091F30E9091F40ECEDA00E09C014AEFAB
:10B210005AE26C2F812F0E94A74E73C0D23029F5BD
:10B220008091F805823021F40E94647F811195C0DD
:10B2300080912402882309F464C011E08091F8050C
:10B24000823009F010E06091F50E7091F60E809159
:10B25000F70E9091F80EA7DA00E09C0146EE5AE254
:10B260006C2F812F0E94A74E4CC0D33029F58091BE
:10B27000F805833021F40E94647F81118AC0809197
:10B280002402882309F43DC011E08091F805833041
:10B2900009F010E06091F90E7091FA0E8091FB0EAA
:10B2A0009091FC0E80DA00E09C0142ED5AE26C2F96
:10B2B000812F0E94A74E25C0D43019F58091F80542
:10B2C000843021F40E94647F81117FC08091240228
:10B2D0008823B9F011E08091F805843009F010E07E
:10B2E0006091FD0E7091FE0E8091FF0E9091000F07
:10B2F0005ADA00E09C014EEB5AE26C2F812F0E943B
:10B30000A74ECF5FDF5FC53009F045CFC093F7058B
:10B3100077C00E94CC7480910906882309F445CF38
:10B320006FC081E00E94597FA12C6AE7C62E63E5B9
:10B33000D62EE12C1CE3F12E0CE116E420E030E0E7
:10B3400040EA50E461EF7EE084E09BE2A7DB80917D
:10B350000906882309F445CF53C081E00E94597F34
:10B36000A12C4AE7C42E43E5D42EE12C1CE3F12E98
:10B370000CE116E420E030E040EA50E465EF7EE0C6
:10B3800080EF9AE28BDB80910906882309F450CF85
:10B3900037C081E00E94597FA12C2AE7C22E23E505
:10B3A000D22EE12C1CE3F12E0CE116E420E030E07B
:10B3B00040EA50E469EF7EE08CED9AE26FDB809129
:10B3C0000906882309F45BCF1BC081E00E94597FE6
:10B3D000A12C8AE7C82E83E5D82EE12C1CE3F12EA0
:10B3E0000CE116E420E030E040EA50E46DEF7EE04E
:10B3F00088EC9AE253DB80910906882309F466CF32
:10B40000DF91CF911F910F91FF90EF90DF90CF9040
:10B41000AF9008956F927F928F929F92AF92BF925A
:10B42000CF92DF92EF92FF920F931F93CF93DF9310
:10B4300000D01F92CDB7DEB761E081E00E94877532
:10B4400060902F06712C61101AC08091F80581114F
:10B4500004C00E94647F8111BFC0809124028823B0
:10B4600009F4B2C081E09091F805911180E004E008
:10B4700024E040E65BE2672D0E94784EA5C021E003
:10B48000621225C08091F805813021F40E94647F0A
:10B490008111AAC080912402882309F495C011E08B
:10B4A0008091F805813009F010E06091AD0E709147
:10B4B000AE0E8091AF0E9091B00E75D900E09C0158
:10B4C00040E55BE2672D812F0E94A74E7DC082E0A0
:10B4D000681225C08091F805823021F40E94647FB3
:10B4E00081119CC080912402882309F46DC011E071
:10B4F0008091F805823009F010E06091B10E7091F2
:10B50000B20E8091B30E9091B40E4DD900E09C0123
:10B5100040E45BE2672D812F0E94A74E55C023E0D7
:10B5200062122CC08091F805833021F40E94647F60
:10B5300081118EC080912402882309F445C011E056
:10B540008091F805833009F010E08091B50E90915C
:10B55000B60EA091B70EB091B80E89839A83AB83D3
:10B56000BC83CE0101960E94809F00E09C0140E3D5
:10B570005BE2672D812F0E94A74E26C084E06812EF
:10B5800023C08091F805843021F40E94647F8111EA
:10B5900099C0809124028823B9F011E08091F805C8
:10B5A000843009F010E06091B90E7091BA0E80916C
:10B5B000BB0E9091BC0EF7D800E09C0140E25BE22C
:10B5C000672D812F0E94A74E7394639425E0721219
:10B5D0003ACF7092F7058FC00E94CC748091090613
:10B5E000882309F43ACF87C081E00E94597FA12CBB
:10B5F000C12CD12CE12C10E8F12E07E714E420E057
:10B6000030E040E85FE36DEA7EE088E59BE246DA01
:10B6100080910906882309F43DCF6DC081E00E9426
:10B62000597FA12CC12CD12CE12C10E8F12E07E779
:10B6300014E420E030E040E85FE361EB7EE088E482
:10B640009BE22CDA80910906882309F44BCF53C082
:10B6500081E00E94597F20E030E048EC52E46091A4
:10B66000B50E7091B60E8091B70E9091B80E0F94F2
:10B670006D690F949E675B016C012AE0A21AB10804
:10B68000C108D1081F921F921F9292E7892E93E55D
:10B69000992E1EEAE12E12E8F12E01E010E02AE0D8
:10B6A00030E040E050E065EB7EE088E39BE20E9402
:10B6B00047730F900F900F9080910906882309F42B
:10B6C00039CF19C081E00E94597FA12CC12CD12C07
:10B6D000E12C10E8F12E07E714E420E030E040E828
:10B6E0005FE369EB7EE088E29BE2D8D980910906AE
:10B6F000882309F44ECF0F900F900F900F90DF9199
:10B70000CF911F910F91FF90EF90DF90CF90BF905E
:10B71000AF909F908F907F906F9008952F923F925F
:10B720004F925F926F927F928F929F92AF92BF9251
:10B73000CF92DF92EF92FF920F931F93CF93DF93FD
:10B74000CDB7DEB727970FB6F894DEBF0FBECDBFDB
:10B750001C017F836E83CA01B901E982FA820B83DF
:10B760001C839C2C8D2CAD822AE037ED43E25CE3F8
:10B770000F946D690F949E672B013C012AE037ED11
:10B7800043E25CE3EE81FF8160817181828193817C
:10B790000F946D690F949E675B016C01A418B50846
:10B7A000C608D7082AE037ED43E25CE3C801B701D9
:10B7B0000F946D690F949E677B018C01E418F50866
:10B7C00006091709FD81FF938F929F9286E6882EC6
:10B7D00083E5982EA30192016E817F81C1010E94B1
:10B7E00047730F900F900F9027960FB6F894DEBF17
:10B7F0000FBECDBFDF91CF911F910F91FF90EF90C2
:10B80000DF90CF90BF90AF909F908F907F906F9080
:10B810005F904F903F902F9008952F923F924F92BC
:10B820005F926F927F928F929F92AF92BF92CF92D0
:10B83000DF92EF92FF920F931F93CF93DF93CDB7D9
:10B84000DEB727970FB6F894DEBF0FBECDBF1C0141
:10B850007F836E83E982FA820B831C839C2C8D2C60
:10B86000AD82CA01B9010F94CF672AE037ED43E2F8
:10B870005CE30F946D690F949E672B013C01EE8190
:10B88000FF8160817181828193810F94CF672AE06B
:10B8900037ED43E25CE30F946D690F949E675B01A3
:10B8A0006C01A418B508C608D708C801B7010F94E1
:10B8B000CF672AE037ED43E25CE30F946D690F94A4
:10B8C0009E677B018C01E418F50806091709FD81C4
:10B8D000FF938F929F928CE6882E83E5982EA3018A
:10B8E00092016E817F81C1010E9447730F900F907A
:10B8F0000F9027960FB6F894DEBF0FBECDBFDF9135
:10B90000CF911F910F91FF90EF90DF90CF90BF905C
:10B91000AF909F908F907F906F905F904F903F90EF
:10B920002F9008959F92AF92BF92CF92DF92EF92A5
:10B93000FF920F931F93CF93DF9300D01F92CDB749
:10B94000DEB761E081E00E94877590902F06B12CF0
:10B9500091101AC08091F805811104C00E94647F83
:10B96000811152C180912402882309F444C181E0ED
:10B970009091F805911180E004E024E04CED5BE249
:10B980006B2D0E94784E37C181E098122CC08091B7
:10B99000F805813021F40E94647F81113DC18091BE
:10B9A0002402882309F427C111E08091F805813031
:10B9B00009F010E08091110F9091120FA091130FD8
:10B9C000B091140F89839A83AB83BC83CE01019617
:10B9D0000E94C89E00E09C0140ED5BE26B2D812F30
:10B9E0000E94A74E08C182E098122CC08091F805F1
:10B9F000823021F40E94647F811128C18091240249
:10BA0000882309F4F8C011E08091F805823009F02C
:10BA100010E08091150F9091160FA091170FB09123
:10BA2000180F89839A83AB83BC83CE0101960E9451
:10BA3000C89E00E09C014CEB5BE26B2D812F0E94C5
:10BA4000A74ED9C083E098122CC08091F8058330AE
:10BA500021F40E94647F811113C180912402882304
:10BA600009F4C9C011E08091F805833009F010E0B5
:10BA70008091190F90911A0FA0911B0FB0911C0F7C
:10BA800089839A83AB83BC83CE0101960E94C89EB2
:10BA900000E09C014AEA5BE26B2D812F0E94A74ED9
:10BAA000AAC084E0981228C08091F805843021F45F
:10BAB0000E94647F8111FEC080912402882309F4D2
:10BAC0009AC011E08091F805843009F010E060918F
:10BAD000DD0E7091DE0E8091DF0E9091E00E0F94DE
:10BAE000CF670E94F95300E09C014CE95BE26B2DAB
:10BAF000812F0E94A74E7FC085E0981228C08091B8
:10BB0000F805853021F40E94647F8111F0C0809196
:10BB10002402882309F46FC011E08091F805853074
:10BB200009F010E06091E10E7091E20E8091E30E59
:10BB30009091E40E0F94CF670E94F95300E09C01AE
:10BB40004EE85BE26B2D812F0E94A74E54C086E029
:10BB5000981228C08091F805863021F40E94647FF5
:10BB60008111E2C080912402882309F444C011E0CD
:10BB70008091F805863009F010E06091E50E709133
:10BB8000E60E8091E70E9091E80E0F94CF670E9429
:10BB9000F95300E09C0140E85BE26B2D812F0E948D
:10BBA000A74E29C087E0981226C08091F8058730FB
:10BBB00021F40E94647F8111D4C0809124028823E3
:10BBC000D1F011E08091F805873009F010E0609124
:10BBD000E90E7091EA0E8091EB0E9091EC0E0F94AD
:10BBE000CF670E94F95300E09C0142E75BE26B2DB6
:10BBF000812F0E94A74EB394939485E0B812A8CEEB
:10BC000088E08093F705C9C00E94CC748091090632
:10BC1000882309F4A7CEC1C081E00E94597FA12CDE
:10BC2000C12CD12CE12C1CE5F12E01EC17E420E015
:10BC300030E040E251E461E17FE086ED9BE26EDDC1
:10BC400080910906882309F4AACEA7C081E00E944A
:10BC5000597FA12CC12CD12CE12C1CE5F12E01EC3B
:10BC600017E420E030E048EC52E465E17FE086EC48
:10BC70009BE254DD80910906882309F4BFCE8DC074
:10BC800081E00E94597FA12CC12CD12CE12C1CE514
:10BC9000F12E01EC17E420E030E048EC52E469E1D9
:10BCA0007FE083EB9BE23ADD80910906882309F46B
:10BCB000D4CE73C081E00E94597FA12C68E7C62EC4
:10BCC00063E5D62E18EBE12E12E8F12E01E010E02C
:10BCD00024E630E040E050E06DED7EE083EA9BE258
:10BCE0009CDD80910906882309F4E6CE56C081E0E8
:10BCF0000E94597FA12C48E7C42E43E5D42E18EBAF
:10BD0000E12E12E8F12E01E010E024E630E040E000
:10BD100050E061EE7EE085E99BE27FDD80910906DF
:10BD2000882309F4F4CE39C081E00E94597FA12C08
:10BD300028E7C22E23E5D22E18EBE12E12E8F12ED1
:10BD400001E010E02AE030E040E050E065EE7EE007
:10BD500087E89BE262DD80910906882309F402CF1F
:10BD60001CC081E00E94597FA12C88E7C82E83E582
:10BD7000D82E18EBE12E12E8F12E01E010E024E6B7
:10BD800030E040E050E069EE7EE089E79BE245DD8F
:10BD900080910906882309F410CF0F900F900F901F
:10BDA0000F90DF91CF911F910F91FF90EF90DF9057
:10BDB000CF90BF90AF909F9008950F93CF93DF9354
:10BDC00061E081E00E948775C0912F06D0E0C1112B
:10BDD00018C08091F805811104C00E94647F811110
:10BDE000B5C080912402882361F081E09091F8052C
:10BDF000911180E004E024E046EA5DE26D2F0E94AC
:10BE0000784E8091250E8770873009F058C0C13078
:10BE1000D9F48091F805813021F40E94647F81116A
:10BE20009DC080912402882309F4C0C081E09091D4
:10BE3000F805913009F080E003E02EE34FE95DE280
:10BE40006D2F0E94784EB2C0C230D9F48091F805AF
:10BE5000823021F40E94647F81118AC08091240283
:10BE6000882309F4A3C081E09091F805923009F08D
:10BE700080E003E02EE348E95DE26D2F0E94784EFA
:10BE800095C0C330D1F58091F805833021F40E942C
:10BE9000647F811177C080912402882309F486C0D1
:10BEA00081E09091F805933009F080E003E02EE303
:10BEB00041E95DE26D2F0E94784E84E03EC0C130C2
:10BEC000F1F48091F805813021F40E94647F8111A2
:10BED00063C080912402882309F46AC081E09091B4
:10BEE000F805913009F080E000E22EE343E85DE2DE
:10BEF0006D2F0E94784E82E020C084E001C082E075
:10BF0000C8131BC08091F8058C1304C00E94647F85
:10BF1000811150C080912402882371F081E09091BA
:10BF2000F8059C1380E003E02EE349E75DE26D2F06
:10BF30000E94784E8C2F01C08C2FDF5FCF5FD530F1
:10BF400009F045CF8F5F8093F7053DC00E94CC7408
:10BF500080910906882309F444CF35C080EB93E62D
:10BF60000E941B5480910906882309F45ACF2BC0E4
:10BF700085EB93E60E941B5480910906882309F4FF
:10BF80006DCF21C08AEB93E60E941B548091090675
:10BF9000882309F480CF17C08DE89DE20E94457385
:10BFA00080910906882309F494CF0DC084E0C5CFA1
:10BFB00082E0C3CF8FEB93E60E941B548091090669
:10BFC000882309F4A7CFDF91CF910F910895CF92E5
:10BFD000DF92EF92FF92CF93C82F0E9439316B010D
:10BFE0007C0124EA30E74DE75FE3609146067091FB
:10BFF000470680914806909149060F942F6787FD68
:10C0000005C04AEF50E060E070E003C040E050E05F
:10C01000BA01C40ED51EE61EF71EC0924206D0928B
:10C020004306E0924406F0924506C0932502CF9164
:10C03000FF90EF90DF90CF9008953F924F925F92E4
:10C040006F927F928F929F92AF92BF92CF92DF9228
:10C05000EF92FF920F931F93CF93DF93CDB7DEB78D
:10C060002A970FB6F894DEBF0FBECDBF9A87898797
:10C07000362E0E94647F882329F010925F060E946A
:10C08000CC74E8C020915506309156064091570671
:10C09000509158062D833E834F835887232B242BA2
:10C0A000252B09F49EC034E0339E80011124F80151
:10C0B000ED5EF14F408051806280738020E030E07F
:10C0C0004AE754E4C301B2010F9455664B015C0189
:10C0D00020E030E04AE754E4C301B2010F94566611
:10C0E0006B017C0180914F028823D1F141E034162D
:10C0F00039F13416A0F052E0351232C08090F30DC1
:10C100009090F40DA090F50DB090F60DC0904B02FC
:10C11000D0904C02E0904D02F0904E0221C08090F1
:10C12000EB0D9090EC0DA090ED0DB090EE0DC09049
:10C130004302D0904402E0904502F090460210C0C5
:10C140008090EF0D9090F00DA090F10DB090F20D59
:10C15000C0904702D0904802E0904902F0904A0215
:10C160006D817E818F8198850F94D16720914606DD
:10C170003091470640914806509149060F946D69E9
:10C180009B01AC01C301B2010F9456660D5E114FC5
:10C19000D8016D937D938D939C9313972D813E8150
:10C1A0004F81588557FF0DC0A50194010F942F674B
:10C1B00087FF12C0D8018D929D92AD92BC921397C9
:10C1C0000BC0A70196010F94326918162CF4F801E0
:10C1D000C082D182E282F382832DF9DE81E08093F6
:10C1E000240210925506109256061092570610928D
:10C1F000580680912402882369F124E0329EF001E0
:10C200001124ED5EF14F80819181A281B3818983F8
:10C210009A83AB83BC832DEC3CEC4CEC5DE36091EA
:10C2200046067091470680914806909149060F9402
:10C23000326987FD05C0CE0101960E94B89D05C0F8
:10C2400060E2CE0101960E94309EBC0189859A85EC
:10C250000E94034F2A960FB6F894DEBF0FBECDBFE3
:10C26000DF91CF911F910F91FF90EF90DF90CF90D2
:10C27000BF90AF909F908F907F906F905F904F9006
:10C280003F90089560E08EE19EE2D7CE61E087E1C5
:10C290009EE2D3CE62E080E19EE2CFCECF93DF93E9
:10C2A00000D01F92CDB7DEB70E94647F882329F0AB
:10C2B00010925F060E94CC745DC06091550670912B
:10C2C00056068091570690915806611571058105B3
:10C2D000910569F10F94D167209146063091470688
:10C2E00040914806509149060F946D699B01AC013D
:10C2F00060911F0E7091200E8091210E9091220E60
:10C300000F94566660931F0E7093200E8093210E3B
:10C310009093220E83E05BDE81E0809324021092F2
:10C3200055061092560610925706109258068091A4
:10C3300024028823F9F02091E2053091E305409131
:10C34000E4055091E50560911F0E7091200E8091DB
:10C35000210E9091220E0F94556669837A838B8308
:10C360009C83CE0101960E94B89DBC018FEA9DE29C
:10C370000E94034F0F900F900F900F90DF91CF917D
:10C38000089521E020935F06609346067093470668
:10C39000809348069093490640E050E0BA018091AE
:10C3A000E0059091E1050C94A17460E070E080E2FA
:10C3B00091E4E7CF60E070E080E89FE3E2CF6DECCE
:10C3C0007CEC8CEC9DE3DDCFFF920F931F93CF931A
:10C3D000DF93F82E7093E1056093E00561E081E062
:10C3E0000E948775D0912F06C0E091E081E0F81699
:10C3F000A9F1F81628F082E0F81609F45DC08AC0A9
:10C40000D111FBC09923D9F08091F8051816BCF022
:10C410004091550650915606609157067091580606
:10C420004F5F5F4F6F4F7F4F4093550650935606B7
:10C4300060935706709358068F5F8093F80580913C
:10C440002402882309F44AC100E010E021E041E021
:10C4500069E07EE28C2F0E94194E40C1D111CDC0FF
:10C460009923D9F08091F8051816BCF04091550633
:10C470005091560660915706709158064F5F5F4F76
:10C480006F4F7F4F40935506509356066093570663
:10C49000709358068F5F8093F8058091240288235B
:10C4A00009F41CC100E010E021E041E062E07EE21E
:10C4B0008C2F0E94194E12C1D1119FC09923D9F01F
:10C4C0008091F8051816BCF040915506509156061B
:10C4D00060915706709158064F5F5F4F6F4F7F4FC7
:10C4E000409355065093560660935706709358062E
:10C4F0008F5F8093F80580912402882309F4EEC0B1
:10C5000000E010E021E041E06BEF7DE28C2F0E9423
:10C51000194EE4C040911F0E5091200E6091210EE3
:10C520007091220E4093E2055093E3056093E40579
:10C530007093E505D1112CC09923D9F08091F805AD
:10C540001816BCF04091550650915606609157065A
:10C55000709158064F5F5F4F6F4F7F4F4093550666
:10C560005093560660935706709358068F5F8093DA
:10C57000F80580912402882309F4E8C000E010E067
:10C5800021E041E061EF7DE28C2F0E94194EDEC078
:10C5900083E0F81232C06091590C70915A0C80916E
:10C5A0005B0C90915C0C2091160C211126C00F940D
:10C5B0009E67209130023091310262177307ECF4CC
:10C5C000D130C9F48091F805813021F40E94647F54
:10C5D00081118EC080912402882369F081E09091BE
:10C5E000F805913009F080E004E024E041EE5DE2DE
:10C5F0006C2F0E94784E82E072C0D130D9F48091C5
:10C60000F805813021F40E94647F811179C0809106
:10C610002402882309F462C081E09091F8059130EA
:10C6200009F080E004E024E047ED5DE26C2F0E9419
:10C63000784E54C0D230D9F48091F805823021F47C
:10C640000E94647F811164C080912402882309F4D0
:10C6500045C081E09091F805923009F080E003E058
:10C660002EE34DEC5DE26C2F0E94784E37C0D33044
:10C67000D1F48091F805833021F40E94647F811108
:10C6800051C080912402882349F181E09091F805FE
:10C69000933009F080E003E02EE344EC5DE26C2F80
:10C6A0000E94784E1BC0D430C9F48091F8058430C4
:10C6B00021F40E94647F81113FC08091240288236D
:10C6C00069F081E09091F805943009F080E003E092
:10C6D0002EE349EB5DE26C2F0E94784E85E0CF5F40
:10C6E000DF5F90E0C53009F081CE8093F70532C05E
:10C6F0000E94CC7480910906882309F46BCF2AC06C
:10C700000E94CC7480910906882309F480CF22C04E
:10C7100085ED91E60E941B5480910906882309F457
:10C7200093CF18C08AED91E60E941B5480910906B0
:10C73000882309F4A6CF0EC08FED91E60E941B540A
:10C7400080910906882309F4B8CF04C083E0F81269
:10C75000C5CF21CFDF91CF911F910F91FF90089509
:10C760004FEF62E471E680E02FCE4FEF66E471E6B2
:10C7700081E02ACE4FEF6AE471E682E025CE4FEFEA
:10C780006EE471E683E020CE0F93CF93DF9361E0F8
:10C7900081E00E948775D0912F06C0E0D1111AC0A8
:10C7A0008091F805811104C00E94647F81118BC0C3
:10C7B00080912402882309F47EC081E09091F805DD
:10C7C000911180E004E024E044E75DE26C2F0E94D8
:10C7D000784E71C0D130D9F48091F805813021F4C0
:10C7E0000E94647F811177C080912402882309F41C
:10C7F00062C081E09091F805913009F080E003E09B
:10C800002EE34AE65DE26C2F0E94784E54C0D2308F
:10C81000D9F48091F805823021F40E94647F81115F
:10C8200064C080912402882309F445C081E090917E
:10C83000F805923009F080E000E22EE34CE55DE27D
:10C840006C2F0E94784E37C0D330D1F48091F80518
:10C85000833021F40E94647F811151C080912402B1
:10C86000882349F181E09091F805933009F080E048
:10C8700000E22EE345EB5CE26C2F0E94784E1BC079
:10C88000D430C9F48091F805843021F40E94647F8B
:10C8900081113FC080912402882369F081E090914A
:10C8A000F805943009F080E000E22EE340EA5CE213
:10C8B0006C2F0E94784ECF5FDF5FC53009F06ECFDE
:10C8C000C093F7052FC00E94CC748091090688237D
:10C8D00009F46ECF27C08DED9EE50E941B54809118
:10C8E0000906882309F480CF1DC086E69DE20E94D8
:10C8F000457380910906882309F493CF13C082EC15
:10C900009CE20E94457380910906882309F4A6CF12
:10C9100009C081EB9CE20E9445738091090688233F
:10C9200009F4B8CFDF91CF910F910895CF93DF93A2
:10C93000EC01CB01BA010F94D1670F949E67798304
:10C940006883DF91CF91089566E974E687E395E601
:10C950000C94E0740F931F93CF93DF9361E081E019
:10C960000E948775C0912F06D0E081E0C1112CC0D4
:10C970008823D9F08091F8051816BCF0409155062F
:10C980005091560660915706709158064F5F5F4F61
:10C990006F4F7F4F4093550650935606609357064E
:10C9A000709358068F5F8093F80580912402882346
:10C9B00009F441C000E010E020E041E06DE77FE2D3
:10C9C0008D2F0E94194E37C0C130D1F48091F805E7
:10C9D000813021F40E94647F811137C0809124024C
:10C9E000882349F181E09091F805913009F080E0C9
:10C9F00000E22EE342E75FE26D2F0E94784E1BC0FB
:10CA0000C230C9F48091F805823021F40E94647F1D
:10CA1000811122C080912402882369F081E09091E5
:10CA2000F805923009F080E000E22EE34EE55FE287
:10CA30006D2F0E94784EDF5FCF5F80E0D53009F028
:10CA400095CF83E08093F7050DC0C0939F0B809135
:10CA50000906882319F206C0C0939F0B809109062E
:10CA60008823C1F2DF91CF911F910F9108950F9408
:10CA7000D1670F949E67CB010C94B89CEF92FF9204
:10CA80000F931F93CF93DF93CDB7DEB72B970FB6DE
:10CA9000F894DEBF0FBECDBF7C014091E705842F27
:10CAA000042E000C990B2091E805223051F0233020
:10CAB00019F02CEA3FE20AC047FF06C028EB3FE22C
:10CAC00005C02AEC3FE202C021EC3FE29F934F9366
:10CAD0003F932F938E010F5F1F4F1F930F930F9460
:10CAE0007C6F40912C0250912D024F5051099701BB
:10CAF0000F900F900F900F900F900F904E155F05B5
:10CB00000CF49A013093560C2093550C80E00E944F
:10CB1000BDC4C8010E94A4762B960FB6F894DEBF60
:10CB20000FBECDBFDF91CF911F910F91FF90EF907E
:10CB30000895E091E705EE0FFF0BEB5AF34F80816C
:10CB400091819CCF5F926F927F928F929F92AF92D2
:10CB5000BF92CF92DF92EF92FF920F931F93CF93EA
:10CB6000DF93582E8093E8056093E70561E081E04C
:10CB70000E948775D0912F06C0E081E029E9622EDE
:10CB800025E6722ED11138C08823D9F08091F8059E
:10CB90001816BCF040915506509156066091570604
:10CBA000709158064F5F5F4F6F4F7F4F4093550610
:10CBB0005093560660935706709358068F5F809384
:10CBC000F80580912402882309F492C022E05216CD
:10CBD00049F083E0581203C06EE87FE205C06EE7BB
:10CBE0007FE202C06EE97FE200E010E021E041E078
:10CBF0008C2F0E94194E7CC0D130D9F48091F80559
:10CC0000813021F40E94647F81117BC080912402D5
:10CC1000882309F46DC081E09091F805913009F006
:10CC200080E004E024E049E050E36C2F0E94784E5D
:10CC30005FC0D230D9F48091F805823021F40E948F
:10CC4000647F811166C080912402882309F450C05A
:10CC500081E09091F805923009F080E000E22EE347
:10CC60004DEF5FE26C2F0E94784E42C0D330D1F47A
:10CC70008091F805833021F40E94647F811154C0B3
:10CC8000809124028823A1F181E09091F8059330EE
:10CC900009F080E000E22EE341EF5FE26C2F0E949A
:10CCA000784E26C0D43021F58091F805843021F4E7
:10CCB0000E94647F811143C0809124028823C1F0C7
:10CCC00011E08091F805843009F010E0E091E7056B
:10CCD000EE0FFF0BEB5AF34F808191810E94B89CBD
:10CCE00000E09C0143ED5FE26C2F812F0E94A74E74
:10CCF000CF5FDF5F80E0C53009F044CFC093F70518
:10CD000051C00E94CC7480910906882309F47ECF1B
:10CD100049C08091F3059091F405B0DE8091090639
:10CD2000882309F490CF3EC08091F5059091F605D7
:10CD3000A5DE80910906882309F4A2CF33C081E0E3
:10CD40000E94597F6091E705660F770B6B5A734F0E
:10CD5000FB01A080B180C501BB0CAA0BBB0B5C0121
:10CD60006D01F8E7AF1AB108C108D1081F927F9290
:10CD70006F9284EA882E84E6982E1AEAE12EF12C2E
:10CD800000E010E028E730E040E050E082EE9FE273
:10CD90000E9447730F900F900F908091090688238F
:10CDA00009F48ACFDF91CF911F910F91FF90EF90FF
:10CDB000DF90CF90BF90AF909F908F907F906F90BB
:10CDC0005F90089560E081E0BDCE8F929F92AF9218
:10CDD000BF92CF92DF92EF92FF920F931F93CF9368
:10CDE000DF934C015B016A0160E085E00E9487757A
:10CDF000D0912F06F12C82E0E82ED1111AC080913B
:10CE00002402882321F180912302823041F0833073
:10CE100019F463E37FE205C061E27FE202C063E4EC
:10CE20007FE200E010E021E041E08F2D0E94194EEA
:10CE30000EC0D13061F480912402882341F000E0DB
:10CE400010E020E041E0B4018F2D0E94194EA114A2
:10CE5000B10481F0D23081F480912402882309F456
:10CE60006EC000E010E020E041E0B5018F2D0E948F
:10CE7000194E65C0C2E001C0C3E0C114D10491F0F5
:10CE8000DC130FC080912402882351F000E010E0F1
:10CE900020E041E0B6018F2D0E94194ECD2F01C038
:10CEA000CD2FCF5F21E030E0A114B10411F420E0D8
:10CEB00030E081E090E0C114D10411F480E090E012
:10CEC000820F931F029781F0DC130DC08091240222
:10CED000882349F000E010E020E041E06CE57FE2CB
:10CEE0008F2D0E94194ECF5FDC1314C08091240255
:10CEF000882371F000E010E021E040E061E57FE28E
:10CF00008F2D0E94194E6091E6058F2D0E94C04D15
:10CF1000E0922402F394DF5F85E0F8126ECFCF5FDA
:10CF2000C093F705DF91CF911F910F91FF90EF9084
:10CF3000DF90CF90BF90AF909F908F900895C3E007
:10CF4000C114D10409F0ADCFADCF48E15FE268E094
:10CF50007FE28FEF9EE239CF40E050E06FEE7EE25D
:10CF600086EE9EE232CF40E050E067ED7EE288EC54
:10CF70009EE22BCF40E050E069EB7EE28CEA9EE23D
:10CF800024CF40EA5EE26FE87EE28FE79EE21DCFAB
:10CF900040E050E061E77EE288E69EE216CF40E0A6
:10CFA00050E068E57EE28BE49EE20FCF40E050E087
:10CFB0006EE37EE28DE39EE208CF40E050E06EE259
:10CFC0007EE285E29EE201CF6111609323024093ED
:10CFD000E605082E000C990BAA0BBB0B8B309105B4
:10CFE00080F5FC018827EA56FF4F8F4F0D94B76AF2
:10CFF0008CEA97E61CC08FEC97E619C081EC97E6A7
:10D0000016C088EC97E613C08DED97E610C086ED4C
:10D0100097E60DC08AEB97E60AC083EB97E607C058
:10D0200010929F0B8AEA94E602C085EA97E6009781
:10D0300041F021E020935F0640E050E0BA010C94FB
:10D04000A1740C94C67480914A06882321F0109232
:10D050005F060E94CC740C94274D9091C90893FBF5
:10D06000882780F993FF06C081E09091F90691111D
:10D0700001C080E008950F93CF93DF9361E081E0DA
:10D080000E948775D0912F06C0E0D1111AC08091FF
:10D09000F805811104C00E94647F811152C0809103
:10D0A0002402882309F444C081E09091F80591118D
:10D0B00080E004E024E044ED50E36C2F0E94784EC1
:10D0C00037C0D130D1F48091F805813021F40E942D
:10D0D000647F81113EC080912402882349F181E060
:10D0E0009091F805913009F080E003E02EE343ECE5
:10D0F00050E36C2F0E94784E1BC0D230C9F480914F
:10D10000F805823021F40E94647F81112CC0809147
:10D110002402882369F081E09091F805923009F0AB
:10D1200080E003E02EE345EB50E36C2F0E94784E45
:10D13000CF5FDF5FC53009F0A8CF83E08093F705AC
:10D140001AC00E94CC7480910906882309F4A7CFE5
:10D1500012C083E298E60E941B548091090688233E
:10D1600009F4B9CF08C089E59FE60E941B5480915D
:10D170000906882361F2DF91CF910F91089540E075
:10D1800061E080E021DF8BEF90E30F94E1550D9497
:10D19000030863DF882319F08091C90882FD0C948D
:10D1A0009ABF87EF90E30F94E155F9CF10929C1846
:10D1B000109270028091C90880628093C9080E9411
:10D1C000A2BF6FEF89EE90E30E943F810C94C6747A
:10D1D0000F93CF93DF9361E081E00E948775D09138
:10D1E0002F06C0E08C2F8D0FC9F48091F8058111B6
:10D1F00004C00E94647F811133C08091240288237F
:10D2000041F181E09091F805911180E004E024E083
:10D2100044EE50E36C2F0E94784E1BC08130C9F45D
:10D220008091F805813021F40E94647F81111FC034
:10D2300080912402882369F081E09091F805913073
:10D2400009F080E000E22EE349ED50E36C2F0E94EC
:10D25000784ECF5FC53031F682E08093F7050CC081
:10D260000E94CC7480910906882339F205C09EDFA4
:10D27000809109068823E1F2DF91CF910F91089503
:10D28000EF92FF920F931F93CF93DF9361E081E0C2
:10D290000E948775C0912F0610E0C11118C08091BF
:10D2A000F805811104C00E94647F811195C18091AD
:10D2B0002402882361F081E09091F805911180E0CB
:10D2C00004E024E049EA50E3612F0E94784E0E9476
:10D2D0008A74D82F9091C90893FBEE24E0F893FF4D
:10D2E00003C0BBDEF82E01C0F12CDD2309F459C0C8
:10D2F000C130D9F48091F805813021F40E94647F17
:10D30000811172C180912402882309F499C181E0BE
:10D310009091F805913009F080E000E22EE34DE9AC
:10D3200050E3612F0E94784E8BC1C230D9F48091B6
:10D33000F805823021F40E94647F81115CC18091E4
:10D340002402882309F47CC181E09091F805923091
:10D3500009F080E003E02EE342E950E3612F0E94F0
:10D36000784E6EC1C33009F057C08091F805833004
:10D3700021F40E94647F811148C180912402882396
:10D3800009F45EC181E09091F805933009F080E0E6
:10D3900003E02EE34DE850E3612F0E94784ED4E085
:10D3A0005BC0C130D9F48091F805813021F40E942E
:10D3B000647F811134C180912402882309F442C121
:10D3C00081E09091F805913009F080E000E22EE3D1
:10D3D00040E850E3612F0E94784E34C1C230F1F42E
:10D3E0008091F805823021F40E94647F81111EC172
:10D3F00080912402882309F425C181E09091F805E9
:10D40000923009F080E003E02EE347E750E3612F1C
:10D410000E94784ED3E020C0D4E001C0D3E0CD1309
:10D420001BC08091F8058C1304C00E94647F811199
:10D430000BC180912402882371F081E09091F8055E
:10D440009C1380E003E02EE34BE650E3612F0E9443
:10D45000784EDC2F01C0DC2F81E08D0FC81318C07F
:10D460008091F8058C1304C00E94647F8111F6C07E
:10D4700080912402882361F081E09091F8059C134B
:10D4800080E003E02EE34DE550E3612F0E94784EEB
:10D4900082E08D0F4091550C5091560C9091160CD6
:10D4A000911107C020913002309131024217530789
:10D4B000DCF0C81333C08091F8058C1304C00E94BF
:10D4C000647F8111D5C080912402882339F181E0E5
:10D4D0009091F8059C1380E000E22EE345E450E3D0
:10D4E000612F0E94784E1AC0C81318C08091F805A9
:10D4F0008C1304C00E94647F8111C4C080912402F7
:10D50000882361F081E09091F8059C1380E003E0AE
:10D510002EE345E350E3612F0E94784EDD5FCD138B
:10D5200018C08091F8058C1304C00E94647F81119B
:10D53000B3C080912402882361F081E09091F805C6
:10D540009C1380E003E02EE347E250E3612F0E944A
:10D55000784E91E09D0FEE20E9F0F11035C0C9132F
:10D5600031C08091F8058C1304C00E94647F811142
:10D570009DC080912402882329F181E09091F805D3
:10D580009C1380E003E02EE349E150E3612F0E9409
:10D59000784E18C0C91316C08091F8058C1302C0CC
:10D5A0000E94647F80912402882361F081E0909141
:10D5B000F8059C1380E000E22EE34EE050E3612F7B
:10D5C0000E94784E92E09D0F1F5FCF5F153009F0EB
:10D5D00064CE9093F70573C00E94CC7480910906C5
:10D5E000882309F464CE6BC0CADD809109068823C4
:10D5F00009F488CE64C088EE98E60E941B5480919E
:10D600000906882309F49BCE5AC087EA9CE60E944B
:10D610001B5480910906882309F4AFCE50C0B9DDB0
:10D6200080910906882309F4C6CE49C084EC93E6AC
:10D630000E941B5480910906882309F4D9CE3FC06B
:10D64000D4E00ACFD3E008CF87E890E70E941B54CC
:10D6500080910906882309F4ECCE31C087EF91E769
:10D660000E941B5480910906882309F401CF27C02A
:10D6700085E590E30E94457380910906882309F4AB
:10D6800022CF1DC082EE96E60E941B5480910906AF
:10D69000882309F433CF13C08BE398E60E941B5410
:10D6A00080910906882309F444CF09C08CE092E5F3
:10D6B0000E941B5480910906882309F45ACFDF91F8
:10D6C000CF911F910F91FF90EF9008956091530CAF
:10D6D00070E080E00C94DFBF60915E0270915F02A9
:10D6E000072E000C880B990B0F94D1672AE037EDB9
:10D6F00043E25CE30F946D6960935A0270935B029E
:10D7000080935C0290935D020895CF93DF93EC01C8
:10D71000CB01BA010F94D1670F94A3676883DF919F
:10D72000CF91089540E050E0BA0185E59CE60E9463
:10D73000A1741092E9051092EA051092EB0510927F
:10D74000EC0581E080935F06089540E050E0BA0167
:10D7500089E59CE60E94A1741092E9051092EA0501
:10D760001092EB051092EC0581E080935F0608951E
:10D7700065E87BE68EEB9BE60C94E0740F94D16732
:10D780000F94A367862F0C94209CEF92FF920F9327
:10D790001F93CF93DF9300D01F92CDB7DEB7082F32
:10D7A0007B010E94647F882329F010925F060E940B
:10D7B000CC7470C08091550690915606A091570682
:10D7C000B09158060097A105B105D1F11092550608
:10D7D00010925606109257061092580621E0209398
:10D7E0002402E02FF0E02091240E30E0002E02C051
:10D7F000359527950A94E2F720FF0AC0EE0FFF1F28
:10D80000E35EF34F20813181280F391F318320835C
:10D81000092E000CAA0BBB0B4091E9055091EA05BB
:10D820006091EB057091EC05840F951FA61FB71F43
:10D830008093E9059093EA05A093EB05B093EC057E
:10D8400080912402882331F184E0089F8001112413
:10D850000354114F6091E9057091EA058091EB0541
:10D860009091EC050F94D1679B01AC01F8016081A8
:10D870007181828193810F946D6969837A838B832F
:10D880009C8360E2CE0101960E94309EBC01C701DC
:10D890000E94034F0F900F900F900F90DF91CF9148
:10D8A0001F910F91FF90EF9008956AE771E380E078
:10D8B0006CCF6FE671E381E068CF4F925F926F9219
:10D8C0007F928F929F92AF92BF92CF92DF92EF9210
:10D8D000FF920F931F93CF93DF93F901D8019E2CF2
:10D8E0009A01550F440B550BEB01A880B9806501D7
:10D8F000BB0CEE08FF0856016701A21AB30AC40A5E
:10D90000D50A2F01FF0F6608770883017201E21A1A
:10D91000F30A040B150B9F92BF93AF93E4EA8E2E8C
:10D92000E4E69E2EB4D60F900F900F90DF91CF912A
:10D930001F910F91FF90EF90DF90CF90BF90AF902D
:10D940009F908F907F906F905F904F9008956F920F
:10D950007F928F929F92AF92BF92CF92DF92EF927F
:10D96000FF920F931F93CF93DF9361E081E00E94BA
:10D970008775D0912F06C0E026E6622E2BE6722E28
:10D98000D1111AC08091F805811104C00E94647FF2
:10D99000811121C180912402882309F413C181E0FF
:10D9A0009091F805911180E004E024E04AE651E30B
:10D9B0006C2F0E94784E06C1D13011F58091F80588
:10D9C000813021F40E94647F81110CC18091240276
:10D9D000882309F4F7C011E08091F805813009F03F
:10D9E00010E080915402909155020E94B89C00E092
:10D9F0009C014EE551E36C2F812F0E94A74EE2C09F
:10DA0000D23011F58091F805823021F40E94647FB4
:10DA10008111FAC080912402882309F4D3C011E057
:10DA20008091F805823009F010E08091550C9091BA
:10DA3000560C0E94B89C00E09C0140E551E36C2F1D
:10DA4000812F0E94A74EBEC0D33011F58091F805FA
:10DA5000833021F40E94647F8111EBC08091240205
:10DA6000882309F4AFC011E08091F805833009F0F4
:10DA700010E080914B0C90914C0C0E94B89C00E0FF
:10DA80009C0148E451E36C2F812F0E94A74E9AC05D
:10DA9000D43001F58091F805843021F40E94647F30
:10DAA0008111DCC080912402882309F48BC011E02D
:10DAB0008091F805843009F010E08091530C0E94A9
:10DAC000209C00E09C0144E351E36C2F812F0E94D5
:10DAD000A74E78C0D53011F58091F805853021F436
:10DAE0000E94647F8111DEC080912402882309F4A2
:10DAF00069C011E08091F805853009F010E080914F
:10DB00005E0290915F020E94B89C00E09C014AE294
:10DB100051E36C2F812F0E94A74E54C0D630D9F408
:10DB20008091F805863021F40E94647F8111CCC079
:10DB300080912402882309F445C081E09091F80582
:10DB4000963009F080E003E02EE34FE151E36C2FC3
:10DB50000E94784E37C0D730D1F48091F8058730D5
:10DB600021F40E94647F8111BCC08091240288232B
:10DB700049F181E09091F805973009F080E003E0E9
:10DB80002EE344E151E36C2F0E94784E1BC0D83045
:10DB9000C9F48091F805883021F40E94647F8111D6
:10DBA000ADC080912402882369F081E09091F8054E
:10DBB000983009F080E003E02EE345E051E36C2F5C
:10DBC0000E94784ECF5FDF5FC53009F0D9CE89E083
:10DBD0008093F7059FC0E0D680910906882309F459
:10DBE000D9CE98C0E12C00E010E027EE33E04AE007
:10DBF00050E064E572E084E691E35FDE809109061F
:10DC0000882309F4E3CE86C081E00E94597FE12C8D
:10DC10000FE916E722E231E040E050E065E57CE004
:10DC200087E591E34ADE80910906882309F4F2CE64
:10DC300071C081E00E94597FE12C02EA16E727E8D3
:10DC400030E040E050E06BE47CE08CE491E335DED2
:10DC500080910906882309F401CF5CC081E00E940D
:10DC6000597FA090530CB12CC12CD12C1F927F92C4
:10DC70006F9288EB882E8BE6982EE12CF12C870191
:10DC8000EA9420E030E0A90163E57CE08EE391E3D3
:10DC9000FED40F900F900F9080910906882309F40D
:10DCA00001CF38C0E12C0CE61BE627EE33E04AE05A
:10DCB00050E06EE572E08FE291E3FFDD80910906AE
:10DCC000882309F411CF26C0C0D440E050E0BA0147
:10DCD00082E99BE636D680910906882309F428CF8D
:10DCE00019C0B3D440E050E0BA0185EA9BE629D6DA
:10DCF00080910906882309F438CF0CC0A6D440E0EF
:10DD000050E0BA018FEF95E71CD680910906882371
:10DD100009F447CFDF91CF911F910F91FF90EF90C2
:10DD2000DF90CF90BF90AF909F908F907F906F903B
:10DD300008954F925F926F927F92AF92BF92CF926F
:10DD4000DF92EF92FF92CF93DF93EB01FC016081B2
:10DD50007181828193812CE3C22ED12CE12CF12C94
:10DD6000A70196010F94796AB62EA72ECA01B901B0
:10DD7000A70196010F94796A6B017C01CA01B90170
:10DD800028E130E040E050E00F94796A2B013C013B
:10DD9000C9016DE671E00F94526A61157105D9F001
:10DDA000AF92BF92DF92CF925F924F929F938F93E9
:10DDB0007F936F938DEA91E39F938F93DF93CF933C
:10DDC0000F947C6F8DB79EB70E960FB6F8949EBFDA
:10DDD0000FBE8DBF61C00097C9F0AF92BF92DF92B6
:10DDE000CF925F924F929F938F938DE991E39F9390
:10DDF0008F93DF93CF930F947C6FEDB7FEB73C9674
:10DE00000FB6F894FEBF0FBEEDBF46C041145104DB
:10DE100061047104B9F0AF92BF92DF92CF925F922A
:10DE20004F9281E991E39F938F93DF93CF930F9468
:10DE30007C6F8DB79EB70A960FB6F8949EBF0FBE43
:10DE40008DBF2AC0C114D104E104F104A9F0AF923E
:10DE5000BF92DF92CF9289E891E39F938F93DF93F4
:10DE6000CF930F947C6FEDB7FEB738960FB6F8944A
:10DE7000FEBF0FBEEDBF10C0AF92BF9285E891E329
:10DE80009F938F93DF93CF930F947C6F0F900F909E
:10DE90000F900F900F900F90DF91CF91FF90EF9028
:10DEA000DF90CF90BF90AF907F906F905F904F903A
:10DEB00008952F923F924F925F926F927F928F922E
:10DEC0009F92AF92BF92CF92DF92EF92FF920F9309
:10DED0001F93CF93DF93CDB7DEB76F970FB6F8944C
:10DEE000DEBF0FBECDBF0E94647F882311F054D5E2
:10DEF000F0C02090710C3090720C8091730C909156
:10DF0000740C9F8F8E8F8091750C9091760CA091E0
:10DF1000770CB091780C8A8F9B8FAC8FBD8F40901F
:10DF2000790C50907A0C60907B0C70907C0C8090F7
:10DF30007D0C90907E0CA0907F0CB090800C60E0E7
:10DF400085E0E5D5E0902F06F12CDE0111966D01FC
:10DF5000E1100DC0809124028823E1F0C1010E94EC
:10DF6000EE9C8C0120E040E062E172E310C0B1E081
:10DF7000EB1210C080912402882361F08E8D9F8D5A
:10DF80000E94EE9C8C0120E040E066E072E38F2D61
:10DF90000E94194E8A8D9B8DAC8DBD8D8E8B9F8B73
:10DFA000A88FB98FB601CE014696C3DE92E0E91282
:10DFB0000BC0809124028823B1F000E010E020E043
:10DFC00040E064EF71E30CC0A3E0EA120CC0809162
:10DFD0002402882341F0860120E040E061EF71E3F4
:10DFE0008F2D0E94194E4E8A5F8A688E798EB601F7
:10DFF000CE0146969EDEB4E0EB120BC08091240267
:10E000008823B1F000E010E020E040E06FED71E324
:10E010000CC085E0E8120CC080912402882341F0F6
:10E02000860120E040E06CED71E38F2D0E94194ED7
:10E0300020E030E048EC52E4C501B4010F943667AB
:10E040000F949E67CB016AE070E00F94666A9F931D
:10E050008F9320E030E04AE754E4C501B4010F9407
:10E0600036670F949E679F938F937F936F93A4ED72
:10E07000B1E3BF93AF93DF92CF920F947C6F0FB653
:10E08000F894DEBF0FBECDBFB6E0EB120BC080919F
:10E0900024028823B1F000E010E020E040E064ECCE
:10E0A00071E30CC087E0E8120CC080912402882341
:10E0B00041F0860120E040E061EC71E38F2D0E9489
:10E0C000194EF394E39495E0F91242CF88E08093DF
:10E0D000F7056F960FB6F894DEBF0FBECDBFDF9188
:10E0E000CF911F910F91FF90EF90DF90CF90BF9055
:10E0F000AF909F908F907F906F905F904F903F90E8
:10E100002F9008951092540C0E9457C53FC42F922F
:10E110003F924F925F926F927F928F929F92AF92B7
:10E12000BF92CF92DF92EF92FF920F931F93CF9304
:10E13000DF9361E081E0EBD420902F06312C66E67E
:10E14000462E6BE6562EC2EAD6E77FE9672E76E7C3
:10E15000772E21101AC08091F805811104C00E9409
:10E16000647F8111AFC080912402882309F477C0B5
:10E1700081E09091F805911180E004E024E043E50E
:10E1800052E3632D0E94784E6AC081E0281222C0BB
:10E190008091F805813021F40E94647F811199C03B
:10E1A00080912402882309F45AC011E08091F80577
:10E1B000813009F010E08091550C9091560C0E942E
:10E1C000B89C00E09C0145E452E3632D812F0E943E
:10E1D000A74E45C092E0291221C08091F8058230F7
:10E1E00021F40E94647F81119DC0809124028823C4
:10E1F000B1F111E08091F805823009F010E08091D2
:10E200004B0C90914C0C0E94B89C00E09C014DE39B
:10E2100052E3632D812F0E94A74E21C083E0281274
:10E220001EC08091F805833021F40E94647F811123
:10E23000A1C080912402882391F011E08091F8051B
:10E24000833009F010E08091530C0E94209C00E084
:10E250009C0149E252E3632D812F0E94A74E8091D9
:10E26000550C9091560C20914B0C30914C0C232B5B
:10E2700011F4892BF1F094E0291219C08091F8056E
:10E28000843021F40E94647F811198C0809124021F
:10E29000882369F081E09091F805943009F080E0DE
:10E2A00000E22EE340E252E3632D0E94784E85E0C7
:10E2B00001C084E03394239495E039124ACF8093CF
:10E2C000F70582C069D380910906882309F44BCFF2
:10E2D0007BC081E00E94597FA090550CB090560CF5
:10E2E0000B2C000CCC08DD081F927F926F9244EA41
:10E2F000842E44E6942E12E2E12EFF24F39400E0F3
:10E3000010E020E030E0A90165E57CE08CE492E3D8
:10E31000BED10F900F900F9080910906882309F4C9
:10E320003FCF52C081E00E94597FA0904B0CB0902B
:10E330004C0C0B2C000CCC08DD081F92DF93CF9304
:10E3400024EA822E24E6922E17E8E12EF12C00E03A
:10E3500010E020E030E0A9016BE47CE081E492E38E
:10E3600096D10F900F900F9080910906882309F4A1
:10E370003CCF2AC081E00E94597FA090530CB12C61
:10E38000C12CD12C1F925F924F9288EB882E8BE686
:10E39000982EE12CF12C8701EA9420E030E0A901CD
:10E3A00063E57CE083E392E372D10F900F900F90CE
:10E3B00080910906882309F43CCF06C0A3DE809132
:10E3C0000906882309F462CFDF91CF911F910F9145
:10E3D000FF90EF90DF90CF90BF90AF909F908F9085
:10E3E0007F906F905F904F903F902F9008950F9384
:10E3F0001F93CF93DF9361E081E089D3D0912F0603
:10E40000C0E0D11117C08091F805811104C00E94AD
:10E41000647F81119EC080912402882309F43EC04C
:10E4200081E09091F805911180E004E024E047EA52
:10E4300052E331C0D130B9F48091F805813021F434
:10E440000E94647F81118CC080912402882331F165
:10E4500081E09091F805913009F080E003E02EE32F
:10E4600045E952E318C0D230C9F48091F8058230F2
:10E4700021F40E94647F811180C08091240288234E
:10E4800069F081E09091F805923009F080E003E0B6
:10E490002EE346E852E36C2F0E94784E3BD2182FB1
:10E4A000D330D9F48091F805833021F40E94647F41
:10E4B000811170C080912402882309F47EC081E01C
:10E4C0009091F805933009F080E000E22EE347E7F1
:10E4D00052E36C2F0E94784E70C0811171C0D4300D
:10E4E000B9F48091F805843021F40E94647F811191
:10E4F00058C080912402882319F181E09091F80599
:10E50000943009F080E000E22EE349E652E315C0C2
:10E51000D530B1F48091F805853009F449C0809177
:10E520002402882369F081E09091F805953009F084
:10E5300080E000E22EE348E552E36C2F0E94784E23
:10E5400086E0CF5FDF5FC53009F05BCF8093F705D2
:10E5500042C022D280910906882309F45CCF3BC0D7
:10E5600074D040E050E0BA0180E394E5EAD18091B4
:10E570000906882309F468CF2EC067D040E050E038
:10E58000BA018FEF95E7DDD180910906882309F460
:10E5900074CF21C0E1D380910906882309F48ACF82
:10E5A0001AC0DDD380910906882309F4A2CF13C0D5
:10E5B0000E94647F811106C0B2CF112309F4C0CF3D
:10E5C00084E0BFCF0E947FEA81E005D380910906F5
:10E5D000882309F4A4CFDF91CF911F910F91089563
:10E5E000CF93DF93EC01CB01BA010F94D1670F9465
:10E5F0009E676883DF91CF910895CF93DF93EC01FD
:10E60000CB01BA010F94D16720E030E040E251E441
:10E610000F946D690F94A36779836883DF91CF911D
:10E6200008950F94D1670F949E67862F0C94469C93
:10E630000F94D16720E030E040E251E40F946D691F
:10E640000F94A367CB010C94759C80910A068630C9
:10E65000D8F496E0899FF0011124E55FF94F2091ED
:10E6600050063091510631832083409155065091D8
:10E67000560660915706709158064283538364830F
:10E6800075838F5F80930A0608950D94E1552F924C
:10E690003F924F925F926F927F928F929F92AF9232
:10E6A000BF92CF92DF92EF92FF920F931F93CF937F
:10E6B000DF9300D000D0CDB7DEB71C012B833C83A5
:10E6C0004D835E8369837A83C0DF83E08093240275
:10E6D000309208062092070669817A8170930606B7
:10E6E000609305062B813C814D815E81209301065C
:10E6F000309302064093030650930406E092FD0512
:10E70000F092FE050093FF0510930006A0925506B7
:10E71000B0925606C0925706D09258069092510673
:10E72000809250068C8D9D8D9093FC058093FB0507
:10E730008E8D8093FA0526960FB6F894DEBF0FBE35
:10E74000CDBFDF91CF911F910F91FF90EF90DF90A0
:10E75000CF90BF90AF909F908F907F906F905F9081
:10E760004F903F902F9008954F925F926F927F92BB
:10E770008F929F92AF92BF92CF92DF92EF92FF92D1
:10E780000F931F93FB01722F602FA12FBE2D242FFB
:10E7900030E040E050E0A080CA2CD12CE12CF12CDC
:10E7A00056016701A21AB30AC40AD50A472E512C92
:10E7B000612C712C83017201E21AF30A040B150B10
:10E7C000BF93AF936F9368EB862E6BE6962EBF01D7
:10E7D0005EDF0F900F900F901F910F91FF90EF90C1
:10E7E000DF90CF90BF90AF909F908F907F906F9071
:10E7F0005F904F9008952F923F924F925F926F9249
:10E800007F928F929F92AF92BF92CF92DF92EF92C0
:10E81000FF920F931F93CF93DF9300D01F921F920D
:10E82000CDB7DEB71C017D836C8349010A831B834E
:10E83000E982BA0180E090E00F94CF672DEC3CECC8
:10E840004CEC5DE30F946D690F949E672B013C01C6
:10E85000EC81FD816081718180E090E00F94CF6751
:10E860002DEC3CEC4CEC5DE30F946D690F949E67CE
:10E870005B016C01A418B508C608D708B40180E094
:10E8800090E00F94CF672DEC3CEC4CEC5DE30F94E3
:10E890006D690F949E677B018C01E418F5080609E9
:10E8A0001709F981FF938B818F93EA81EF9382E8B7
:10E8B000882E85E7982EA30192016C817D81C1018C
:10E8C000E6DE0F900F900F900F900F900F900F902B
:10E8D0000F90DF91CF911F910F91FF90EF90DF90FC
:10E8E000CF90BF90AF909F908F907F906F905F90F0
:10E8F0004F903F902F900895FB01908181E08927F0
:10E90000808383E0809324024115510511F0FA01C0
:10E910001994089580912B0F9091280F891B8F7067
:10E9200071F49091C90892FB882780F992FD08C084
:10E9300081E090918F18913019F080E0089581E086
:10E940000895209150063091510628173907E9F0B3
:10E950009093510680935006409355065093560667
:10E960006093570670935806885B9E4721F4109277
:10E970005F0610920A060E94BF4D82E08093240237
:10E9800081E08093090610925A06089540E050E015
:10E99000BA0188EB9EE7D5CFE0910A06EE2379F025
:10E9A000E150E0930A0686E0E89FF0011124E55F5C
:10E9B000F94F40E050E0BA0180819181C2CFE6CFAB
:10E9C0000F931F93CF93DF93FC01EB0180915506CA
:10E9D00090915606A0915706B0915806B7FF08C00F
:10E9E000109255061092560610925706109258062D
:10E9F0008091FD059091FE05A091FF05B091000664
:10EA000040915506509156066091570670915806F0
:10EA100084179507A607B70744F48093550690938B
:10EA20005606A0935706B093580680912402882377
:10EA300001F18091010690910206A0910306B09128
:10EA40000406409155065091560660915706709104
:10EA500058068C019D01040F151F261F371FC90181
:10EA6000B8011995BC0180910706909108060E9493
:10EA7000034F80914A06811108C08091FA058823CE
:10EA8000B9F180912402882399F180910506909133
:10EA900006060097B1F00091010610910206209140
:10EAA0000306309104064091550650915606609138
:10EAB000570670915806400F511F621F731FFE01C9
:10EAC0001995E091FB05F091FC05309741F080919C
:10EAD000FA05811103C080914A06811119950E949F
:10EAE000647F882329F0DF91CF911F910F9154CF3C
:10EAF000DF91CF911F910F91089560EF72E781E14F
:10EB000093E75ECF6DEF72E788E193E759CF282F47
:10EB100010924F068091550690915606A091570687
:10EB2000B091580681309048A105B10540F010928F
:10EB3000550610925606109257061092580680916C
:10EB40005906882331F0809155068093F80510927C
:10EB500009068091F7051816FCF4082E000C990B95
:10EB6000821B91092091F805022E000C330B281707
:10EB7000390794F097FF02C080E090E08093F80599
:10EB8000092E000CAA0BBB0B8093550690935606DA
:10EB9000A0935706B09358068091F8056623C1F0FC
:10EBA00090912F06891714F480932F0620912F0639
:10EBB000022E000C330B2C5F3F4F482F082E000C09
:10EBC000550B2417350734F4845080932F0608958D
:10EBD00080932F060895882361F063E972E084E64C
:10EBE00090E00F9419616AEB72E084E690E00D9476
:10EBF000196168EB71E084E190E00D9419618F92E6
:10EC00009F92AF92BF92CF92DF92EF92FF920E94BB
:10EC1000647F882359F010925F06FF90EF90DF9099
:10EC2000CF90BF90AF909F908F90B6CE81E08093B1
:10EC30005F06C0905506D0905606E0905706F090BB
:10EC40005806C114D104E104F10409F450C0109233
:10EC50005506109256061092570610925806B601A5
:10EC60000D2C000C880B990B0F94D1672091C50EC9
:10EC70003091C60E4091C70E5091C80E0F946D6929
:10EC80002091E10D3091E20D4091E30D5091E40DA2
:10EC90000F9456664B015C0120E030E040E050EC00
:10ECA0000F94326987FD23C020E030E040EA50E451
:10ECB000C501B4010F942F671816CCF08091240E73
:10ECC00082FF0AC08091210C9091220CC80ED91E9F
:10ECD000D092220CC092210C8092E10D9092E20D14
:10ECE000A092E30DB092E40D82E080932402809123
:10ECF00024028823D9F081EE9DE00E941A9DBC0178
:10ED00008CEA92E30E94034F6091E10D7091E20D55
:10ED10008091E30D9091E40DFF90EF90DF90CF9004
:10ED2000BF90AF909F908F900C94A84FFF90EF9062
:10ED3000DF90CF90BF90AF909F908F90089580E02C
:10ED40000C94BDC40C940AC521E02093F9050F94DE
:10ED5000E6551092F90508950E94F0E53CCF0E9417
:10ED600037F739CF6091650D7091660D82E39DE0B4
:10ED70000C94A33B60912A0D70912B0D87EF9CE0C2
:10ED80000C94A33B6091EF0C7091F00C8CEB9CE029
:10ED90000C94A33B6091B40C7091B50C81E89CE09D
:10EDA0000C94A33B8F929F92AF92BF92CF92DF922F
:10EDB000EF92FF92CF936091F10E7091F20E8091DD
:10EDC000F30E9091F40E0F94A3674B015C01C09178
:10EDD0006B0D82E39DE00E94183DDC0120E136E0EE
:10EDE00041EC50E00F94CE6A6B017C01AC2FB0E097
:10EDF000A50194010F94CE6A2227362F472F582F52
:10EE0000C701B6010F94796ABA01A901662777276D
:10EE100082E39DE0CF91FF90EF90DF90CF90BF9085
:10EE2000AF909F908F900C946C3D8F929F92AF9279
:10EE3000BF92CF92DF92EF92FF92CF936091F50E47
:10EE40007091F60E8091F70E9091F80E0F94A367D3
:10EE50004B015C01C091300D87EF9CE00E94183D92
:10EE6000DC0120E136E041EC50E00F94CE6A6B010A
:10EE70007C01AC2FB0E0A50194010F94CE6A22274B
:10EE8000362F472F582FC701B6010F94796ABA0160
:10EE9000A9016627772787EF9CE0CF91FF90EF903D
:10EEA000DF90CF90BF90AF909F908F900C946C3D6F
:10EEB0008F929F92AF92BF92CF92DF92EF92FF928A
:10EEC000CF936091F90E7091FA0E8091FB0E9091A4
:10EED000FC0E0F94A3674B015C01C091F50C8CEB09
:10EEE0009CE00E94183DDC0120E136E041EC50E05E
:10EEF0000F94CE6A6B017C01AC2FB0E0A5019401A8
:10EF00000F94CE6A2227362F472F582FC701B601FC
:10EF10000F94796ABA01A901662777278CEB9CE0E8
:10EF2000CF91FF90EF90DF90CF90BF90AF909F90E8
:10EF30008F900C946C3D8F929F92AF92BF92CF9224
:10EF4000DF92EF92FF92CF936091FD0E7091FE0ED3
:10EF50008091FF0E9091000F0F94A3674B015C010D
:10EF6000C091BA0C81E89CE00E94183DDC0120E1D0
:10EF700036E041EC50E00F94CE6A6B017C01AC2F7F
:10EF8000B0E0A50194010F94CE6A2227362F472FB7
:10EF9000582FC701B6010F94796ABA01A9016627F3
:10EFA000772781E89CE0CF91FF90EF90DF90CF90A2
:10EFB000BF90AF909F908F900C946C3D60916C0DC2
:10EFC00082E39DE00C94E53D6091310D87EF9CE07C
:10EFD0000C94E53D60916A0D82E39DE00C946040E5
:10EFE00060912F0D87EF9CE00C9460406091F40CD1
:10EFF0008CEB9CE00C9460406091B90C81E89CE043
:10F000000C9460400F931F93CF93DF9361E081E0F6
:10F010007EDDD0912F06C0E081E0D1112CC0882385
:10F02000D9F08091F8051816BCF040915506509122
:10F03000560660915706709158064F5F5F4F6F4FAD
:10F040007F4F409355065093560660935706709332
:10F0500058068F5F8093F80580912402882309F475
:10F06000AAC000E010E020E041E06DE373E38C2FE4
:10F070000E94194EA0C0D130D1F48091F8058130A2
:10F0800019F422D78111A1C080912402882309F4A8
:10F0900092C081E09091F805913009F080E004E0A1
:10F0A00024E041E353E36C2F0E94784E84C0D230B9
:10F0B000F9F48091F805823019F406D781118CC0DB
:10F0C00080912402882309F476C080916A0D811111
:10F0D00003C028E233E302C02CE233E381E09091E5
:10F0E000F805923009F080E001E046E253E360C0A9
:10F0F000D330F9F48091F805833019F4E5D6811105
:10F1000078C080912402882309F455C080912F0D86
:10F11000811103C02DE133E302C021E233E381E03A
:10F120009091F805933009F080E001E04BE153E362
:10F130003FC0D430F1F48091F805843019F4C4D67E
:10F14000811164C0809124028823A9F18091F40C7C
:10F15000811103C022E133E302C026E133E381E001
:10F160009091F805943009F080E001E040E153E32C
:10F170001FC0D53001F58091F805853019F4A4D66B
:10F18000811151C0809124028823A9F08091B90C8B
:10F19000811103C026E033E302C02AE033E381E0BB
:10F1A0009091F805953009F080E001E043E053E3E9
:10F1B0006C2F0E94A74ECF5FDF5F80E0C53009F063
:10F1C0002CCF86E08093F7053AC0E6DB80910906F4
:10F1D000882309F459CF33C04AEE57E76AE67DE049
:10F1E0008FE293E389DB80910906882309F468CFD5
:10F1F00026C040EF57E76FE27DE084E293E37CDBDB
:10F2000080910906882309F47CCF19C046EF57E79F
:10F2100064EF7CE089E193E36FDB8091090688234A
:10F2200009F490CF0CC04CEF57E769EB7CE08DE020
:10F2300093E362DB80910906882309F4A3CFDF9171
:10F24000CF911F910F9108954F925F926F927F928D
:10F250008F929F92AF92BF92CF92DF92EF92FF92E6
:10F260000F931F93CF93DF9361E081E050DCD09147
:10F270002F06C0E044EE642E47E7742E5EED452E67
:10F2800057E7552ED11119C08091F805811103C09F
:10F290001BD6811156C080912402882309F448C0EE
:10F2A00081E09091F805911180E004E024E049E5C7
:10F2B00053E36C2F0E94784E3BC0D130D1F4809143
:10F2C000F805813019F400D6811142C080912402E2
:10F2D000882371F111E08091F805813009F010E088
:10F2E00080916C0D0E94469C00E09C0145E553E333
:10F2F0001BC0D230E9F48091F805823019F4E4D5CE
:10F30000811152C080912402882391F011E08091F4
:10F31000F805823009F010E08091310D0E94469C82
:10F3200000E09C0141E553E36C2F812F0E94A74E22
:10F33000CF5FDF5FC53009F0A5CF83E08093F7058D
:10F340005EC02ADB80910906882309F4A4CF57C048
:10F35000A0906C0D8A2DAA0C990BAA0BBB0B5C011B
:10F360006D0120E4A20EB11CC11CD11C1F925F9242
:10F370004F922DE7822E25E7922E1FE7E12EF12CEA
:10F3800000E010E020EC3FEF4FEF5FEF6CE67DE038
:10F3900087E593E37CD90F900F900F908091090639
:10F3A000882309F493CF2BC0A090310D8A2DAA0C8D
:10F3B000990BAA0BBB0B5C016D0120E4A20EB11CE2
:10F3C000C11CD11C1F927F926F928DE7882E85E71A
:10F3D000982E1FE7E12EF12C00E010E020EC3FEF2B
:10F3E0004FEF5FEF61E37DE083E593E350D90F904A
:10F3F0000F900F9080910906882309F483CFDF9145
:10F40000CF911F910F91FF90EF90DF90CF90BF9021
:10F41000AF909F908F907F906F905F904F900895E6
:10F420000F93CF93DF9361E081E071DBD0912F06E2
:10F43000C0E0D11116C08091F805811103C044D5F8
:10F4400081117BC080912402882309F46EC081E081
:10F450009091F805911180E004E024E04BEF52E335
:10F4600061C0D130B9F48091F805813019F42CD500
:10F4700081116AC080912402882309F456C081E07A
:10F480009091F805913009F080E003E02EE34CEE16
:10F4900052E348C0D230B9F48091F805823019F4B3
:10F4A00013D581115BC080912402882309F43DC0EB
:10F4B00081E09091F805923009F080E003E02EE3BE
:10F4C0004BED52E32FC0D330B1F48091F805833077
:10F4D00019F4FAD481114CC080912402882329F1B7
:10F4E00081E09091F805933009F080E003E02EE38D
:10F4F00049EC52E317C0D430C1F48091F805843050
:10F5000019F4E2D481113EC080912402882369F06D
:10F5100081E09091F805943009F080E003E02EE35B
:10F520004BEB52E36C2F0E94784ECF5FDF5FC5300C
:10F5300009F07FCFC093F7052EC02EDA809109061F
:10F54000882309F47FCF27C08FEC9AE70E941B54D1
:10F5500080910906882309F48DCF1DC08EEC9BE7AE
:10F560000E941B5480910906882309F49CCF13C084
:10F5700084E299E70E941B5480910906882309F4CC
:10F58000ABCF09C082E098E70E941B548091090626
:10F59000882309F4B9CFDF91CF910F910895EF92AD
:10F5A0000F931F93CF93DF9361E081E0B0DAD091A6
:10F5B0002F06C0E0D11119C08091F805811103C058
:10F5C00083D4811197C080912402882309F48AC0D2
:10F5D00081E09091F805911180E004E024E045E994
:10F5E00053E36C2F0E94784E7DC0D130E9F48091B6
:10F5F000F805813019F468D4811183C08091240208
:10F60000882309F46FC011E08091F805813009F07A
:10F6100010E08091650D9091660D0E94759C00E050
:10F620009C0141E953E35AC0D230E9F48091F805D6
:10F63000823019F449D4811176C080912402882344
:10F6400009F450C011E08091F805823009F010E013
:10F6500080912A0D90912B0D0E94759C00E09C01D9
:10F660004DE853E33BC0D330E1F48091F80583309B
:10F6700019F42AD4811169C080912402882391F160
:10F6800011E08091F805833009F010E08091EF0CD3
:10F690009091F00C0E94759C00E09C0149E853E3B6
:10F6A0001DC0D430F9F48091F805843019F40CD4DD
:10F6B00081115DC0809124028823A1F011E0809126
:10F6C000F805843009F010E08091B40C9091B50CED
:10F6D0000E94759C00E09C0143E853E36C2F812F4E
:10F6E0000E94A74ECF5FDF5FC53009F063CFC093A4
:10F6F000F7054EC051D980910906882309F463CFDC
:10F7000047C0E12C02EB16E728EB3BE044E650E073
:10F7100065E67DE083E993E36ED88091090688234E
:10F7200009F46CCF35C0E12C0AEB16E728EB3BE07F
:10F7300044E650E06AE27DE08FE893E35CD8809194
:10F740000906882309F479CF23C0E12C02EC16E7DF
:10F7500028EB3BE044E650E06FEE7CE08BE893E37F
:10F760004AD880910906882309F486CF11C0E12C7C
:10F770000AEC16E728EB3BE044E650E064EB7CE063
:10F7800086E893E338D880910906882309F492CF5C
:10F79000DF91CF911F910F91EF900895EF920F930A
:10F7A0001F93CF93DF9361E081E0B1D9D0912F0611
:10F7B000C0E0D11119C08091F805811103C084D334
:10F7C00081118FC080912402882309F482C081E0D6
:10F7D0009091F805911180E004E024E047E753E3BD
:10F7E0006C2F0E94784E75C0D130D9F48091F80505
:10F7F000813019F469D381117BC080912402882360
:10F8000009F467C011E08091F805813009F010E03B
:10F8100080916B0D0E94209C00E09C0143E753E324
:10F8200054C0D230D9F48091F805823019F44CD309
:10F8300081116FC080912402882309F44AC011E02D
:10F840008091F805823009F010E08091300D0E941F
:10F85000209C00E09C014FE653E337C0D330D1F445
:10F860008091F805833019F42FD3811163C0809102
:10F870002402882371F111E08091F805833009F0AA
:10F8800010E08091F50C0E94209C00E09C014BE66A
:10F8900053E31BC0D430E9F48091F805843019F4A7
:10F8A00013D3811158C080912402882391F011E074
:10F8B0008091F805843009F010E08091BA0C0E9424
:10F8C000209C00E09C0145E653E36C2F812F0E94B1
:10F8D000A74ECF5FDF5FC53009F06BCFC093F70550
:10F8E0004AC05AD880910906882309F46BCF43C0D7
:10F8F000E12C02ED16E72FEF40E06BE67DE085E7B7
:10F9000093E30E94B47380910906882309F475CFAC
:10F9100032C0E12C05E117E72FEF40E060E37DE026
:10F9200081E793E30E94B47380910906882309F468
:10F9300081CF21C0E12C08E517E72FEF40E065EF0C
:10F940007CE08DE693E30E94B473809109068823DE
:10F9500009F48DCF10C0E12C0BE917E72FEF40E041
:10F960006AEB7CE088E693E30E94B4738091090619
:10F97000882309F498CFDF91CF911F910F91EF90D9
:10F980000895FC0180810895FC01849108954F92AF
:10F990005F926F927F928F929F92AF92BF92CF921F
:10F9A000DF92EF92FF920F931F93CF93DF936C013F
:10F9B0007B015A012901672B31F088248394912C13
:10F9C000C0E0D0E019C0F8011182108227C03701D1
:10F9D000680C791C76946794E3012197A201BE011B
:10F9E000C601F50119951816190654F0892BC9F0AE
:10F9F0004301FFEF8F1A9F0AE814F90440F702C091
:10FA00007E01FACFCE15DF0530F4CE0102968816BE
:10FA1000990620F02196F801D183C0838FEF9FEFE4
:10FA200005C0F801D183C08380E090E0DF91CF91E1
:10FA30001F910F91FF90EF90DF90CF90BF90AF900C
:10FA40009F908F907F906F905F904F9008958F92CE
:10FA50009F92AF92BF92CF92DF92EF92FF920F935D
:10FA60001F93CF93DF93EC016B017A01FB01199592
:10FA700087FD06C0082F10E020E030E0219620C16D
:10FA8000982F907E903CC1F4082F0F7110E020E079
:10FA900030E04801590186E0880C991CAA1CBB1C67
:10FAA0008A95D1F7CE010196F60119958F739501CC
:10FAB0008401082B229604C1982F907F903E19F55F
:10FAC0008F70882E912CA12CB12C16E0880C991CDB
:10FAD000AA1CBB1C1A95D1F7CE010196F601199507
:10FAE0008F73882A06E0880C991CAA1CBB1C0A95F7
:10FAF000D1F7CE010296F60119958F739501840115
:10FB0000082B2396DDC0982F987F903F81F5877052
:10FB1000882E912CA12CB12CF6E0880C991CAA1CE3
:10FB2000BB1CFA95D1F7CE010196F60119958F739A
:10FB3000882AA6E0880C991CAA1CBB1CAA95D1F7A0
:10FB4000CE010296F60119958F73882AB6E0880CCB
:10FB5000991CAA1CBB1CBA95D1F7CE010396F601DD
:10FB600019958F7395018401082B2496A9C0982FAD
:10FB70009C7F983FE9F58370882E912CA12CB12CA5
:10FB800056E0880C991CAA1CBB1C5A95D1F7CE01D3
:10FB90000196F60119958F73882A66E0880C991CE6
:10FBA000AA1CBB1C6A95D1F7CE010296F6011995E5
:10FBB0008F73882A76E0880C991CAA1CBB1C7A9546
:10FBC000D1F7CE010396F60119958F73882AE6E0E6
:10FBD000880C991CAA1CBB1CEA95D1F7CE0104968F
:10FBE000F60119958F7395018401082B259668C03D
:10FBF000982F9E7F9C3F09F04AC08170882E912CDF
:10FC0000A12CB12C86E0880C991CAA1CBB1C8A95DF
:10FC1000D1F7CE010196F60119958F73882A96E0E7
:10FC2000880C991CAA1CBB1C9A95D1F7CE01029690
:10FC3000F60119958F73882A26E0880C991CAA1C56
:10FC4000BB1C2A95D1F7CE010396F60119958F7347
:10FC5000882A36E0880C991CAA1CBB1C3A95D1F75F
:10FC6000CE010496F60119958F73882A46E0880C18
:10FC7000991CAA1CBB1C4A95D1F7CE010596F6012A
:10FC800019958F7395018401082B269619C0982F1A
:10FC9000907C903849F4082F007C003871F421964C
:10FCA000CE01F6011995F7CF082F0E7F0D3F28F0F2
:10FCB0002196CE01F6011995F7CF00E010E09801EA
:10FCC000E114F10429F0F7010083118322833383C7
:10FCD000CE01DF91CF911F910F91FF90EF90DF90B8
:10FCE000CF90BF90AF909F908F9008951F93CF9328
:10FCF000DF9300D01F92CDB7DEB710E0AE014F5FAB
:10FD00005F4F61EC7CE7A3DE49815A816B817C8186
:10FD1000452B462B472B11F01F5FF0CF812F0F9003
:10FD20000F900F900F90DF91CF911F9108951F9327
:10FD3000CF93DF9300D01F92CDB7DEB710E0AE01B6
:10FD40004F5F5F4F64EC7CE782DE49815A816B81B3
:10FD50007C81452B462B472B11F01F5FF0CF812F65
:10FD60000F900F900F900F90DF91CF911F910895FA
:10FD700010924F0680914A0610924A06882349F055
:10FD800040E050E0BA0180E499E60E94A1740C942E
:10FD90008C4D20915402309155024091550650915E
:10FDA00056066091570670915806C901840F951F39
:10FDB0002436310571F4473051056105710514F0A1
:10FDC000069732C04A3F5F4F6F4F7F4F54F50696FC
:10FDD0002BC02436310524F48536910514F504C072
:10FDE0008436910524F41DC08A3091053CF0883E8C
:10FDF00043E094072CF087EE93E002C08AE090E0A5
:10FE00002817390761F0909355028093540210929D
:10FE100055061092560610925706109258060C94EA
:10FE2000564984E690E0E3CF8A30910504F78AE0F2
:10FE300090E0E9CFCF93DF931F92CDB7DEB78091EB
:10FE40007A08811103C08CEB98E02FC0211103C008
:10FE50008AE798E02AC08DE0815048F0440F411DA8
:10FE6000E82FF0E0E454F74F90814927F5CF8091D7
:10FE700041068417A9F0409341068AE798E0698318
:10FE800035DF90E06981861B910997FF02C080E011
:10FE900090E0809352061092530688E080932602E9
:10FEA0008091530690E08658974F0F90DF91CF9145
:10FEB000089580934F0610924B0610924C061092B4
:10FEC0004D0610924E06089580914A0610924A06F9
:10FED0000895CF92DF92EF92FF920F931F930E94AB
:10FEE000393100913D0610913E0620913F06309138
:10FEF00040066B017C01C01AD10AE20AF30AF7FC42
:10FF000013C020913C06209520933C06DC01CB01D8
:10FF10008A549C4FAF4FBF4F80933D0690933E064F
:10FF2000A0933F06B093400681E090913C0691116A
:10FF300001C080E01F910F91FF90EF90DF90CF9074
:10FF400008958091C90882FF09C083FF04C0809191
:10FF5000F906811106C020E02093620680916206B6
:10FF600008958091840690918506A0918606B091AF
:10FF700087060097A105B10571F3BC01CD016D594C
:10FF80007F4F8F4F9F4F24E630E040E050E00F94CA
:10FF9000796A6091800670918106809182069091C5
:10FFA00083060F94796AD8CFCF9393E0909324027D
:10FFB0008111109261060E943931DC01CB018C5015
:10FFC0009E4FAF4FBF4F80935B0690935C06A0930C
:10FFD0005D06B0935E0668E873E182E090E00F94FE
:10FFE0001961C6E0C15049F00F94AE6062E070E064
:10FFF00080E090E00E946A31F5CFCF910895AF92F2
:020000021000EC
:10000000BF92CF92DF92EF920F931F93CF93DF9324
:1000100000D01F92CDB7DEB7809125028F3F09F443
:1000200044C00E943931009142061091430620914C
:10003000440630914506DC01CB01801B910BA20BDD
:10004000B30BB7FD32C09091280F80912B0F8F5FBB
:100050008F70981751F1E091250284E0E802F001D9
:100060001124E059FC4F20E030E040E752E4608189
:100070007181828193810F94366769837A838B8340
:100080009C83A12CB12C6501E12C8E010F5F1F4FC9
:100090002FE13EE04BE15EE067E17EE083E19EE040
:1000A0000F94CC168FEF809325020F900F900F9036
:1000B0000F90DF91CF911F910F91EF90DF90CF9034
:1000C000BF90AF9008950F931F930E943931009114
:1000D0005B0610915C0620915D0630915E06DC01A6
:1000E000CB01801B910BA20BB30BB7FD11C080910C
:1000F000030181FB992790F981E089279091030101
:1001000092FF82609091000196FF84608093610667
:100110008091610681709091610691FD826090915D
:100120003006891741F18130A9F028F0823041F082
:10013000833059F01EC0913089F09230A9F019C077
:10014000992361F0933081F014C0913069F09230BE
:1001500081F404C0992341F0933059F490915406EE
:1001600091509093540605C0909154069F5F9093D0
:100170005406809330061F910F910895CF93DF931B
:100180000E948C4DE4E0F1E080818D7F8083C5E0AA
:10019000D1E088818095827043E051E0DA018C9350
:1001A00080818B7F80838881809584708C9321E00F
:1001B00031E0D9018C918F7B8C93809102018095E5
:1001C00080748093000180818E7F808388818095F8
:1001D0008170FA01808382E08093600674DF109260
:1001E0005406DF91CF910C94F9AB81E090916306B6
:1001F000911101C080E00895CF93DF9320917A069A
:1002000021111EC0FC0101900020E9F73197EF0198
:10021000C81BD90BC731D10534F031972081207C20
:100220002038D9F3F4CFBC01DD27AE0183E696E098
:100230000F94626FCD59D94F188283E080932402C6
:10024000DF91CF910895CF93DF93CDB7DEB78E8145
:1002500090917A06891780F080937A069E01275F35
:100260003F4F4F81588566E170E083E696E00F943A
:10027000AB6F83E080932402DF91CF9108950F93B9
:100280001F93CF93DF938C0167FF03C010927A0610
:1002900060E080917A0690E0262F062E000C330B4A
:1002A000281739070CF160937A06C8010F94C46EC1
:1002B000F801E80FF91FEF01C01BD10BC731D105C1
:1002C00034F031978491807C8038D9F3F4CFDD27E6
:1002D000AE01B80183E696E00F94E56ECD59D94F93
:1002E000188283E080932402DF91CF911F910F91B8
:1002F00008954F925F926F927F928F929F92AF92EA
:10030000BF92CF92DF92EF92FF920F931F93CF9302
:1003100076DED9DE8091610682FF15C080913B06B2
:10032000811113C091E090933B0620919C182111FC
:1003300003C08091F905892780934A0610929C1882
:1003400081E032DE02C010923B068091030180956D
:100350008170C09160068C17B9F080936006882385
:1003600009F48EC164EF71E080E090E00E94DC9BB4
:100370000E94038DC23009F07EC10E94D38D83E0BC
:10038000809324020E948C4D0E9439316B017C01C4
:100390008091370690913806A0913906B0913A06BF
:1003A000A7019601281B390B4A0B5B0B57FF05C0B1
:1003B00080915A06882309F43DC2D701C6018C59A1
:1003C0009F4FAF4FBF4F8093370690933806A0934F
:1003D0003906B0933A0660915406062E000C770B4E
:1003E00077FF03C0719561957109062E000C770B9C
:1003F000880B990B0F94D1672B013C0120E030E072
:1004000040E050E40F94326987FF05C080914A06AE
:10041000811183C093C080914F06882309F456C090
:1004200080904B0690904C06A0904D06B0904E06E2
:1004300081149104A104B104E1F120E030E040E036
:100440005FE3C301B2010F946D692B013C01C70149
:10045000B601681979098A099B090F94CF679B0136
:10046000AC01C301B2010F94366720E030E04AE7E7
:1004700054E40F946D694B015C0120E030E040EAE8
:1004800052E40F94326987FF0FC020E030E040EF64
:1004900051E4C501B4010F94326987FD0AC02AE016
:1004A00030E040E050E009C024E630E040E050E0B9
:1004B00004C021E030E040E050E0C0924B06D09212
:1004C0004C06E0924D06F0924E0604C021E030E06A
:1004D00040E050E0A09154060A2E000CBB0B0F9494
:1004E000D86A22E030E040E050E00F949B6A8091AF
:1004F000550690915606A0915706B0915806820F66
:10050000931FA41FB51F8093550690935606A09382
:100510005706B093580610925406D701C601885664
:10052000954CAF4FBF4F8093330690933406A09302
:100530003506B093360681E0809324022091500660
:10054000309151064EE7283B340741F48091260252
:10055000882309F4A8C08150809326022C5032458C
:1005600071F48091530690915206891740F490914E
:100570002602992309F4A7C09150909326028091F6
:100580006F0081FB222720F981FF05C080916F0059
:100590008D7F80936F0080913B0E90913C0EA091D7
:1005A0003D0EB0913E0E222329F020916F00226073
:1005B00020936F003AE0B695A795979587953A9561
:1005C000D1F7009721E0A207B10520F08FEF9FEF50
:1005D000A0E0B0E09695879520912402211105C0F6
:1005E00030915A06311122C139C0009739F040913B
:1005F0003106509132064817590780F580915A0606
:10060000811103C0223008F076C0C1E0809150060D
:1006100090915106885B9E4709F0C0E08C2F0E94A4
:100620005849CC2309F473C0A3DB10924A060E94F8
:100630003931DC01CB018C199D09AE09BF0900914C
:1006400031061091320620E030E0081719072A071A
:100650003B0720F490933206809331068091500638
:1006600090915106885B9E4709F4A3C080915F0674
:1006700081119FC0CAC060E085ED93E300DE7FCEAC
:10068000BAD5C23009F47BCE60E088EC93E3F7DDA5
:100690008091500690915106885B9E4709F46FCE79
:1006A0000E94C6746CCE8CE0809326028091310645
:1006B000909132060197909332068093310681E043
:1006C000809324024BCF96E09093260291E0909382
:1006D00024028F5F80935306D701C6018856954C3C
:1006E000AF4FBF4F8093330690933406A0933506E7
:1006F000B093360644CF243030F0243009F085CF53
:100700001092240282CF81E0809324027ECF8091D8
:100710005A06811114C08091DF04811107C081E065
:100720008093DF0486EA94E00E94F93586EA94E03B
:100730000E94303681E08093590680935A0683E008
:100740000E94A54C61E086EA94E00E945236E09156
:100750005006F091510619951092590680915A064B
:10076000882309F462CF86EA94E00E94343691E04F
:10077000811101C090E090935A06992309F455CF56
:100780000E943931DC01CB018C199D09AE09BF09EA
:10079000C0903106D0903206E12CF12CC816D90653
:1007A000EA06FB0608F046C09093320680933106B5
:1007B00041C058E9C50E5AE3D51EE11CF11CC09298
:1007C0003306D0923406E0923506F09236068091D8
:1007D0005A0681112FC080912402813099F0833014
:1007E00049F5CF911F910F91FF90EF90DF90CF903F
:1007F000BF90AF909F908F907F906F905F904F9041
:100800000C94BF4D1092240215C080913306909134
:100810003406A0913506B0913606C81AD90AEA0AFC
:10082000FB0AF7FCD4CF0E94C674D1CF009709F41D
:10083000ECCEDDCECF911F910F91FF90EF90DF9026
:10084000CF90BF90AF909F908F907F906F905F9070
:100850004F90089561E013DD0C94C674CF93DF933D
:100860001F921F92CDB7DEB789839A8387DC898177
:100870009A81F0DF0F900F90DF91CF910C94914D02
:100880008091C90882FD05C080918F18823061F483
:1008900010C080917A08811103C08CEB98E002C0EF
:1008A0008AE798E061E0A8CC813031F081EA93E3F7
:1008B00005C08BEB93E302C08FEA93E36FEFDFCCCD
:1008C00088EB9EE79093510680935006089561E06F
:1008D000FC0180810E945E338FEF0C945CA4CF9367
:1008E000DF93EC018A810E941DA460E08881DF9182
:1008F000CF910C945E338F929F92AF92BF92EF9202
:10090000FF920F931F93CF93DF93EC018B017A013A
:100910000E9439314B015C012CE2820E21E0921ED3
:10092000A11CB11C0E9436A48B838F3F61F40E94EE
:100930003931DC01CB0188199909AA09BB09B7FD36
:10094000F1CF81E10DC08E3F51F4B701C8010E9483
:100950003DA40E9436A40E9436A411E003C08FE09B
:10096000898310E0CE01B3DF812FDF91CF911F91FA
:100970000F91FF90EF90BF90AF909F908F90089550
:10098000CF92DF92EF92FF926A017B010E94393190
:10099000C60ED71EE81EF91E0E9436A48F3F61F0D6
:1009A0000E943931DC01CB018C199D09AE09BF09C8
:1009B000B7FDF2CF80E001C081E0FF90EF90DF90C3
:1009C000CF900895EF92FF921F93CF93DF9300D0C3
:1009D0001F92CDB7DEB77C01162F29833A834B8354
:1009E0005C837DDF48E552E060E070E0C701C8DF6E
:1009F000812F80640E945CA48C810E945CA48B8106
:100A00000E945CA48A810E945CA489810E945CA4EB
:100A1000112311F087E801C085E90E945CA41C3015
:100A200011F40E9436A410E00E9436A4F7018383DB
:100A300087FF04C01F3F11F01F5FF6CF0F900F908C
:100A40000F900F90DF91CF911F91FF90EF9008953D
:100A50008F929F92AF92BF92CF92DF92EF92FF92CE
:100A60000F931F93CF93DF93EC01162F1C821982F3
:100A700048830E9439316B017C0120EDC20E27E0D2
:100A8000D21EE11CF11CA89561E088810E945E33B2
:100A900061E088810E9422330E942EA485E08A832F
:100AA0000E941DA40AE08FEF0E945CA40150D9F7B8
:100AB000A89520E030E0A90160E0CE0183DF8B83C0
:100AC000813061F00E943931DC01CB018C199D0924
:100AD000AE09BF09B7FDEDCF81E055C0A8952AEA60
:100AE00031E040E050E068E0CE016CDF853011F489
:100AF00081E009C004E00E9436A48B830150D9F73D
:100B00008A3A51F482E08C83A8958C81823081F0FE
:100B1000812C912C540111C00E943931DC01CB0190
:100B20008C199D09AE09BF09B7FDD9CF82E02BC052
:100B3000812C912CA12C80E4B82E20E030E0A9017A
:100B400067E3CE013FDFA501940169E2CE013ADF00
:100B50008B83882361F00E943931DC01CB018C1931
:100B60009D09AE09BF09B7FDE8CF8AE00CC08C81B2
:100B70008230D1F420E030E0A9016AE3CE0122DF27
:100B8000882329F088E08983CE01A1DE16C00E9467
:100B900036A4807C803C11F483E08C830E9436A4D0
:100BA0000E9436A40E9436A4CE0191DE173018F4BC
:100BB0001A8381E003C088E1898380E0DF91CF91CF
:100BC0001F910F91FF90EF90DF90CF90BF90AF906B
:100BD0009F908F9008950F931F93CF93DF93EC0115
:100BE00089018C81833039F089E0440F551F661FDD
:100BF000771F8A95D1F79A01AB0161E1CE01E2DE60
:100C0000811109C040E052E0B801CE01DF91CF91DF
:100C10001F910F9170CE84E08983CE0158DE80E071
:100C2000DF91CF911F910F910895CF93DF93EC0146
:100C3000862FBA010E9461A48FEF0E945CA48FEFFF
:100C40000E945CA40E9436A48B83982F9F719530DC
:100C500031F083E18983CE013ADE80E001C081E09A
:100C6000DF91CF9108950F931F93CF93DF93EC0102
:100C700089018C81833039F089E0440F551F661F4C
:100C8000771F8A95D1F79A01AB0168E1CE019ADE10
:100C900081111EC0A8016EEFCE01C7DF8823E1F0ED
:100CA00048E552E060E070E0CE016ADE882371F032
:100CB00020E030E0A9016DE0CE0184DE81110AC0A0
:100CC0000E9436A4811106C011E007C087E103C06D
:100CD00086E001C086E1898310E0CE01F8DD812F36
:100CE000DF91CF911F910F910895CF93DF931F92C2
:100CF000CDB7DEB720919E1830919F18CE01019696
:100D00002115310519F0821B930B02C0845A9841BA
:100D10000F90DF91CF910895FC01238121110C9454
:100D20002B9708958091C908847F8B7F8093C90891
:100D3000109280061092810610928206109283060D
:100D400010928406109285061092860610928706ED
:100D50001092F506109234078EE091E0E5E3F7E09B
:100D6000DF019C011D9221503040E1F78FEF80930D
:100D700079080895FC0120E03EE2DB014C9140320D
:100D800041F0283011F430833196DB014C914083DF
:100D900031962F5F6F5F7F4F2B3079F71082089568
:100DA0002F923F924F925F926F927F928F929F927B
:100DB000AF92BF92CF92DF92EF92FF920F931F9369
:100DC000CF93DF93CDB7DEB7C356D1090FB6F894F2
:100DD000DEBF0FBECDBF8C015B014A014DB65EB6D2
:100DE000312C7E0187E5E80EF11C9BE1292E4AE7B4
:100DF00058E0BE016F5F7F4FC5010E949B9518169A
:100E00000CF005C18C85282F2871203109F074C0A1
:100E100090917F069150923008F46EC06DB67EB608
:100E2000BE016F5F7F4FC701A5DF0115110521F0DE
:100E3000F8018081811173C021E081E090E0F70129
:100E400001900020E9F73197EE19FF09E80FF91F2B
:100E500032968DB79EB78E1B9F0B0FB6F8949EBF30
:100E60000FBE8DBFEDB7FEB731966F01211102C0E5
:100E7000B80102C060E873E0C6010F944D6FB7017E
:100E8000C6010F94376F60E873E0C6010F94376FA7
:100E90001CAE1FAE21E0A701B501CE01CC960E9489
:100EA000279981110DC080917F06811109C00E9490
:100EB0002FA085EC95E30E9421A0C7010E94EDA21E
:100EC000FE01FC96DE019196822D01900D928A958D
:100ED000E1F740E050E0BE016F5D7F4FC60160DF8B
:100EE000CE01819619DFCE01CC9616DF0FB6F894AD
:100EF0007EBE0FBE6DBE7BCF9981992309F487C05A
:100F0000953E09F474CF9E3209F471CF90917A081E
:100F10009E3209F46CCF8A7009F069CF0AC0F801DB
:100F200001900020E9F73197CF01801B910B20E061
:100F300086CF81E0203109F080E09091C90880FBE4
:100F400094F99093C908811108C08985873409F004
:100F50004ECF8A858E3709F44ACF80917F06813043
:100F600021F068F08230B9F142CF80917D069091F6
:100F70007E06019690937E0680937D0638CFBE0153
:100F80006F5F7F4F8CEB98E0F5DE0115110511F0D6
:100F9000680105C08CEBC82E88E0D82E08C0F60189
:100FA00081916F018823B1F30E9496A2F8CFF601D8
:100FB00081916F01882319F00E9496A2F8CF80E2F8
:100FC0000E9496A26D8D7E8D8F8D98A14AE050E093
:100FD0000E94A9A30CCFBE016F5F7F4F8CEB98E0FE
:100FE000C9DE8114910441F06CEB78E0C4010F94E8
:100FF000246F892B51F40BC0832D90E020917B0648
:1010000030917C068217930711F03394F0CE0FB61F
:10101000F8945EBE0FBE4DBECD59DF4F0FB6F894AB
:10102000DEBF0FBECDBFDF91CF911F910F91FF901B
:10103000EF90DF90CF90BF90AF909F908F907F9078
:101040006F905F904F903F902F900895CF93DF93D4
:10105000CDB7DEB76B970FB6F894DEBF0FBECDBF2E
:1010600010927F0640E050E0BA018EE598E00E94C1
:101070004A968BE1EEE5F8E0DE01119601900D92C3
:101080008A95E1F740E050E0BE016F5F7F4F80E05E
:1010900090E086DECE0101963FDE6B960FB6F894A7
:1010A000DEBF0FBECDBFDF91CF9108950F931F9389
:1010B000CF93DF93CDB7DEB72D970FB6F894DEBF91
:1010C0000FBECDBF8091F906882391F0BE016F5FFE
:1010D0007F4F86EF96E00E94BD938E010F5F1F4FFA
:1010E000F80181918F01882339F00E9496A2F8CFF0
:1010F0008BEB95E30E9421A08AE00E9496A22D9698
:101100000FB6F894DEBF0FBECDBFDF91CF911F9118
:101110000F910895CF92DF92EF92FF920F931F935A
:10112000CF93DF93CDB7DEB7EDB6FEB6DC010D9001
:101130000020E9F79D01281B390B2C5F3F4F4DB76D
:101140005EB7421B530B0FB6F8945EBF0FBE4DBF88
:101150000DB71EB70F5F1F4F9F938F9385E795E3E2
:101160009F938F931F930F930F947C6F680154E0AC
:10117000C50ED11C0F900F900F900F900F900F90F5
:10118000F6018081882349F0082E000C990B0F94FA
:10119000A86EF60181936F01F3CFC8010F94E65555
:1011A00081E795E30F94E1550FB6F894FEBE0FBEAC
:1011B000EDBEDF91CF911F910F91FF90EF90DF90E7
:1011C000CF9008958091C90883FF03C08460809305
:1011D000C90808951092960B8091C9088F7D8B7F66
:1011E0008093C9080E942D68882321F086EF96E03D
:1011F0000C942B970895EEDF8091C908877F809328
:10120000C90808950F931F93CF93DF938B01EA01D1
:10121000DB016D917C910E94BD93D801ED91FC9111
:101220009081888191110EC08936B0F48FE280835D
:10123000F8018081918101969183808388818F5FFD
:1012400088830AC0893680F73196D801ED93FC93E4
:1012500088818F5F8883E1CFDF91CF911F910F91BC
:1012600008950F931F93CF93DF9300D0CDB7DEB7D0
:101270009C012F5F3F4F3B832A832FE2FC01208399
:1012800081E0898310E00BE180913407181770F436
:10129000019FC0011124AE014F5F5F4FBE016E5F21
:1012A0007F4F8B5C984FAEDF1F5FEECF89818B3510
:1012B00070F4AE014F5F5F4FBE016E5F7F4F86EFF0
:1012C00096E0A0DF8A819B8101979B838A83EA81D4
:1012D000FB8110820F900F900F90DF91CF911F91A3
:1012E0000F9108958091C90882FF1FC082E494E3A2
:1012F0000E9421A0609180067091810680918206F3
:10130000909183064AE050E00E9498A38FE20E94E9
:1013100096A26091840670918506809186069091D0
:1013200087064AE050E00C94A9A381E394E30C946F
:1013300021A0EF92FF920F931F93CF93DF938C0125
:10134000FC0101900020E9F73197EF01C81BD90B90
:101350001092F6066EE470E00F94426F7C010097E5
:1013600029F4FE013197E00FF11F0EC060E270E03A
:101370000F94426F8C010F5F1F4F6AE270E0C7014C
:101380000F94426FFC0131978DE081838AE0828364
:101390001382B80186EF96E00E94BA9B8091F60610
:1013A000882361F00E9432A08AE194E3DF91CF911B
:1013B0001F910F91FF90EF900C9421A0DF91CF919E
:1013C0001F910F91FF90EF90089586EF96E00E9495
:1013D000E09686EF96E00E942B978091C9088D7F5A
:1013E0008E7F8093C9081092800610928106109219
:1013F00082061092830681E080938F0B08950F93ED
:101400001F93CF93DF93CDB7DEB76B970FB6F894EA
:10141000DEBF0FBECDBF8B0122E020937F069093ED
:101420007C0680937B0640E050E0BA0183E498E0BC
:101430000E944A968BE1E3E4F8E0DE011196019008
:101440000D928A95E1F7A801BE016F5F7F4F80E0A2
:1014500090E0A6DCCE0101965FDC6B960FB6F894A7
:10146000DEBF0FBECDBFDF91CF911F910F910895C9
:10147000CF93DF93CDB7DEB76B970FB6F894DEBF8F
:101480000FBECDBF81E080937F0610927E06109242
:101490007D0640E050E0BA0183E498E00E944A965D
:1014A0008BE1E3E4F8E0DE01119601900D928A955C
:1014B000E1F740E050E0BE016F5F7F4F80E090E0D9
:1014C0006FDCCE01019628DC80917D0690917E062E
:1014D0006B960FB6F894DEBF0FBECDBFDF91CF91F4
:1014E00008952F923F924F925F926F927F928F92C8
:1014F0009F92AF92BF92CF92DF92EF92FF920F93A3
:101500001F93CF93DF93CDB7DEB76C970FB6F894E8
:10151000DEBF0FBECDBF5C014C8F2DB63EB619822B
:101520001C82FB0180819E012F5F3F4F49018F325A
:1015300039F083E498E0F501918380838B0162C0E8
:101540008EE598E0F501918380838B010F5F1F4F3B
:101550000115110509F456C04DB65EB66FE270E094
:10156000C8010F94426F3C010817190708F04AC0E0
:101570007C01E01AF10AFF24C70101962DB73EB79E
:10158000281B390B0FB6F8943EBF0FBE2DBF8DB789
:101590009EB701966C01A701B8010F94626FF60126
:1015A000EE0DFF1D10823C8D332319F0C6010E9401
:1015B000EDA2F5016081718121E0A601C4010E94C4
:1015C0002799811113C0B6018DEF93E30E9435A0D6
:1015D0008EE20E9496A28AE00E9496A20FB6F8942C
:1015E0005EBE0FBE4DBE00E010E00CC0F501918262
:1015F000808283010F5F1F4F0FB6F8945EBE0FBE4F
:101600004DBEA6CFC40188DBC8010FB6F8943EBE1C
:101610000FBE2DBE6C960FB6F894DEBF0FBECDBFC9
:10162000DF91CF911F910F91FF90EF90DF90CF90BE
:10163000BF90AF909F908F907F906F905F904F90F2
:101640003F902F9008950F931F93CF93DF931F9296
:101650001F92CDB7DEB72091C90823FF27C0BC0178
:1016600040E0CE0101963DDF8C010097F9F0BC010E
:1016700089819A810E94019AB801882381F08CE6C1
:1016800094E30E9435A08AE00E9496A21092800600
:1016900010928106109282061092830607C084E59C
:1016A00094E30E9435A08EE20E9496A20F900F90C4
:1016B000DF91CF911F910F910895EF92FF920F93B9
:1016C0001F93CF93DF9300D0CDB7DEB72091C90829
:1016D00023FF07C1F42EE62E8C010E942D6888237B
:1016E00009F451C0FF2009F45BC08091F5068823FE
:1016F00059F00E9432A08CE295E30E9421A080E084
:1017000090E00F945364EDC088E896E0AADDE09184
:10171000F50684E0E89FF0011124EF50F94F809125
:10172000800690918106A0918206B0918306808305
:101730009183A283B3830E942FA0B80183E195E334
:101740000E9435A08091F50699E6899FB001112489
:101750006857794F88E095E30E9435A04091800654
:1017600050918106609182067091830682E095E334
:101770000E9496A08AE00E9496A28091F5068F5F53
:101780008093F50625C0FF2039F00E942FA082EF3C
:1017900094E30E9421A01CC01092F50622E001C033
:1017A00021E02B830E942FA08DEE94E30E9421A0C4
:1017B0002B81213009F492C081EE94E30E9421A094
:1017C000B80189ED94E30E9435A08AE00E9496A2B8
:1017D00001DD40E0B801CE01019683DE8C01009767
:1017E00009F47FC069817A81EE2009F44BC021E0C1
:1017F000AC0186EF96E00E942799882309F43EC049
:101800008091070790910807A0910907B0910A07F6
:101810008093840690938506A0938606B0938706EE
:101820001092800610928106109282061092830612
:10183000B8018BEC94E30E9435A04091840650914E
:101840008506609186067091870683EC94E30E947A
:1018500096A08AE00E9496A284EB94E30E9421A0C5
:10186000B80180E090E0CBDD80917A08811102C060
:10187000C80102C08AE798E060E02DC0B80180EAA4
:1018800094E30BC026E5AC0186EF96E00E94279911
:1018900081110CC0B8018CE894E30E9435A08EE25F
:1018A0000E9496A28AE00E9496A21BC08091C9085D
:1018B00081608093C908B80180E090E0A0DD1092BB
:1018C0008F0BB8018AE794E30E9435A08AE00E945A
:1018D00096A260E0C8010E94FC8003C087EE94E3FA
:1018E0006DCF0F900F900F90DF91CF911F910F91BF
:1018F000FF90EF9008952091C90822602093C908B5
:1019000040E060E0DACE0F931F93CF93DF93CDB723
:10191000DEB76B970FB6F894DEBF0FBECDBF8C015C
:1019200019821C8280914608811103C06EE578E01F
:1019300002C063E478E021E0A801CE0101960E9494
:1019400027998823F1F08BE1FE013196A3E4B8E0FA
:1019500001900D928A95E1F7A0913407AA30D8F44E
:1019600081E08A0F809334078BE18A9FD001112494
:10197000AB5CB84FE3E4F8E001900D928A95E1F793
:101980000AC00E942FA0B80187EE93E30E9435A001
:101990008AE00E9496A2CE010196BED96B960FB640
:1019A000F894DEBF0FBECDBFDF91CF911F910F9195
:1019B0000895809134078823C9F0815080933407BB
:1019C000882359F090E001972BE1289FF001299F8F
:1019D000F00D1124EB5CF84F02C0EEE5F8E08BE16E
:1019E000A3E4B8E001900D928A95E1F78091340765
:1019F00008958BE1EEE5F8E0A3E4B8E001900D92E4
:101A00008A95E1F708958091C908877F8093C90876
:101A100080916108882321F08EE598E00E942B9741
:101A200045E360E08FE297E013D8811105C00E9482
:101A30002FA08DEA95E32AC041E06FE277E081E1D3
:101A400097E07BD481110DC040E06FE277E081E147
:101A500097E073D4811105C00E9432A089E995E313
:101A600015C061E177E08EE598E0E3D6811105C00D
:101A70000E9432A088E895E309C08091C908886077
:101A80008093C9080E942FA08CE795E30E9421A0B3
:101A9000B0DF83E0809324020895AF92BF92CF928B
:101AA000DF92EF92FF921F93CF93DF93CDB7DEB714
:101AB000A8970FB6F894DEBF0FBECDBF809179080E
:101AC00087FD61C08091C90882FD5DC083FF9BDFF7
:101AD0008091C90883FF54C080917908082E000CBA
:101AE000990BC0969F938F9381E194E39F938F937B
:101AF0006E0181E2C80ED11CDF92CF920F947C6FF1
:101B000040E050E0BA018EE598E00E944A960F90BE
:101B10000F900F900F900F900F90FE0131967F0164
:101B200040E050E0B7018EE598E00E949B951816C2
:101B30003CF5F70101900020E9F731971E2F1E199F
:101B4000115068F05701A10EB11C17FDBA94F501B0
:101B5000808190E00F94A86EF5018083F1CF8A8593
:101B60008E37F1F245E050E0B601C7010F94546F93
:101B7000892BB1F6C601CEDA809179088F5F01C05A
:101B80008FEF80937908A8960FB6F894DEBF0FBE4A
:101B9000CDBFDF91CF911F91FF90EF90DF90CF905D
:101BA000BF90AF9008951092790823CF61CC0F9425
:101BB000030886EF96E00E942B978091F506882314
:101BC00029F181508093F50629E6829FC0011124F6
:101BD00041E061E08857994F70DDE091F50684E0BF
:101BE000E89FF0011124EF50F94F4081518162814B
:101BF00073814093800650938106609382067093B0
:101C0000830686EF96E00E944A96DCCAE3DA0E94D9
